:1000000000000220218C0000498C00004B8C000075
:100010004D8C00004F8C0000518C0000000000004F
:10002000000000000000000000000000538C0000F1
:10003000558C000000000000578C0000598C000017
:100040005B8C000079600000E58F0000598B000098
:100050004D8B00005B8C00005B8C00005B8C000013
:10006000114000005B8C00005B8C00005B8C00008A
:100070005B8C00005B8C00005B8C00005B8C0000E4
:100080005B8C0000699000005B8C00005B8C0000C2
:100090005B8C00005B8C00005B8C00005B8C0000C4
:1000A0005B8C00005B8C00005B8C00005B8C0000B4
:1000B0005B8C00005B8C0000000000000000000072
:1000C0005B8C00005B8C00005B8C00005B8C000094
:1000D0005B8C00005B8C00005B8C00005B8C000084
:1000E0005B8C000000000000000000000000000029
:1000F000000000005B8C0000000000005B8C000032
:1001000000000000000000000000000000000000EF
:1001100000000000000000000000000000000000DF
:1001200000000000000000000000000000000000CF
:1001300000000000000000000000000000000000BF
:1001400000000000000000000000000000000000AF
:10015000000000000000000000000000000000009F
:10016000000000000000000000000000000000008F
:10017000000000000000000000000000000000007F
:10018000000000000000000000000000000000006F
:10019000000000000000000000000000000000005F
:1001A000000000000000000000000000000000004F
:1001B000000000000000000000000000000000003F
:1001C000000000000000000000000000000000002F
:1001D000000000000000000000000000000000001F
:1001E000000000000000000000000000000000000F
:1001F00000000000000000000000000000000000FF
:1002000010B5054C237833B9044B13B10448AFF350
:1002100000800123237010BD440200200000000074
:10022000ACE7000008B5034B1BB103490348AFF32B
:10023000008008BD0000000048020020ACE700007C
:10024000154B002B08BF134B9D46A3F5803A0021A8
:100250008B460F461348144A121A0BF099F90F4BAC
:10026000002B00D098470E4B002B00D09847002061
:10027000002104000D000D48002802D00C48AFF307
:1002800000800BF03DF92000290008F003FF0BF07F
:1002900011F900BF0000080000000220000000006B
:1002A00000000000440200209C900120000000009B
:1002B0000000000010F0010310D104280CD90368DD
:1002C000C3F30F1343B1013B9B001A1DC1180979F9
:1002D00011B101339342F9D1184670470023FBE76F
:1002E000037883B11A0601D40130704703F0C003CC
:1002F000C02B08BF0130024610460132037803F0DC
:10030000C003802BF8D0704708B5002103780BB9E3
:10031000084608BDFFF7E4FF0131F7E738B50022D2
:1003200004460D46411C092004F0A6F940B16300C3
:10033000024643F0010342F8043F0023A34200DBDE
:1003400038BD55F8231042F8041F0133F6E70128A1
:1003500038B504DC1C20BDE8384001F075BA0D68E2
:10036000EA0701D41120F6E74868C30706D4042839
:1003700004D9036803F00F03042B01D00E20EAE731
:1003800003F0DEFF6D10002D044603DDFFF7BCFF18
:10039000A84206DA1220DEE72046FFF7A1FF013D62
:1003A0000446012DF8D120787F2808DDDF280ADCFB
:1003B0006378800100F4F86003F03F0318434000C5
:1003C00040F0010038BDEF280ADC637800039B0190
:1003D00080B203F47C630343A07800F03F00EDE7B4
:1003E000F72810DC637880041B0303F47C3300F4EB
:1003F000E0101843E37803F03F030343A078800143
:1004000000F47C60DAE74FF0FF30D8E7486838B591
:10041000C3070D4606D4042804D9036803F00F026D
:10042000092A04D00B20BDE8384001F00DBA446819
:10043000C3F30F1364105A1EA2420BD8032194FB7E
:10044000F1F16429A8BF64210329ACBF5918D91C54
:1004500004F04EF90368C3F30F13013B9C4208D22A
:10046000A31C013464002A6840F8232044F00104EE
:100470004460002038BD01282DE9F84304DC1C202D
:10048000BDE8F84301F0E0B902284E680CD08C6852
:10049000E70709D56410012CB8BF0124F50705D57D
:1004A0004FF0FF30BDE8F8830124F7E7042EF7D9B9
:1004B00033680D6803F00F02042A30D1E80706D430
:1004C000042D04D92B6803F00F03042B01D00E2058
:1004D000D6E73046FFF7EEFEA042E1DB304603F000
:1004E0002FFF0646284603F02BFF03780146002B1A
:1004F000D6D0601E30440BF01AFC01460028CFD045
:10050000012433780BB18E4203D3640044F0010020
:10051000C8E73046FFF7E4FE01340646F1E7092A52
:1005200038D177687F10BC42BADCE90729D4042DA2
:1005300027D92B6803F00F03042B22D1284603F0A0
:10054000FFFE804604F1010956F82900854203D1D7
:10055000600040F00100A5E7C2070ED404280CD9C2
:10056000036803F00F03042B07D103F0E9FE0146F3
:1005700040460BF0A3FB0028C7D0B9454C46E1DD4F
:100580008EE7631C56F82320AA42BED0BB421C460D
:10059000F7DD85E7032A83D1C3F30F17C3F3417354
:1005A000C3EB8707BC423FF77BAFEB0728D4042D92
:1005B00026D9286800F00F03032B17D1C0F30F13BF
:1005C000C0F3417005F10408C0EB83003F1A013C01
:1005D00040440336BC423FF763AF3219434683427F
:1005E00019460FD315D1601C4000B2E7042B07D188
:1005F000284603F0A5FE80462846FFF75BFEE5E7A8
:100600000F203DE712F8015F09788D4203F10103E5
:10061000E5D00134DEE7000001282DE9F0470E4661
:1006200004DC1C20BDE8F04701F00EB90868C207E1
:1006300006D4042804D9036803F00F03042B01D067
:100640000E20EFE74B6813F00109F9D1042BF7D91D
:100650001B6803F00F03042BF2D103F071FE044674
:10066000706803F06DFE82460BF032FB804670B975
:100670002046FFF749FE05460122A918092003F08C
:10068000FBFF354F386098B90020BDE8F087514630
:1006900020460BF04CFB231A5D425D4120466F1C47
:1006A0000028E9D0514640440BF041FB3D46F6E7B7
:1006B0006B0043F001034360B8F1000F19D12046ED
:1006C000FFF70EFE4D45064601DC3868DDE7311BBD
:1006D000204604F052F80028D6D009F102023B6807
:1006E00043F822003046FFF7FBFD09F101093446CB
:1006F000E8E7012D02D133688360C6E75146204602
:100700000BF015FB01268146B9F1000F14D0B5425C
:10071000DBDBA9EB0401204604F02FF80028B3D05E
:100720003B68013609EB080443F826005146204691
:100730000BF0FDFA8146E7E7B542C6DB20460BF039
:10074000C7FA0146204604F018F800289CD001366C
:100750003B6843F82600B8E7546D012008B503F064
:10076000D3FD400040F0010008BDC30711D40428A8
:100770000FD9026802F00F03032B0AD101F0030323
:10078000C3F104035B0703F0C04322F0C0421343EC
:1007900003607047002838B504DC1C20BDE83840F1
:1007A00001F052B80C68E50701D40D20F6E70128E6
:1007B0001CD04B68DA07F8D55B10FF2B01D913204A
:1007C000ECE71A0442EA03621A4342EA0322641085
:1007D00024EAE474E11C8910032003F04DFF054670
:1007E00010B12146FFF7C1FF284638BD0022EEE7D1
:1007F00001282DE9F0470546884604DC1C20BDE8A9
:10080000F04701F021B84C6814F0010701D10D2028
:10081000F5E7022802D08B68DA07F8D5D8F800602F
:10082000F30700F1A980042E40F2A680326864101C
:10083000012C02F00F03B8BF0124092B28D17668E0
:10084000022D4FEA660605D0D8F808305B109E42AC
:10085000A8BF1E46351B0135012225EAE575A918FA
:10086000092003F009FF074648B16D00034645F033
:100870000105D8F8002043F8045FA64202DA3846A2
:10088000BDE8F087013452F8241043F8041FF4E760
:10089000042B43D1304603F053FDFFF735FD022D05
:1008A000824605D0D8F808305B109842A8BF9A4617
:1008B000A24504DA0020BDE8F04703F057BF3046F8
:1008C00003F03EFD0546A74222DB304603F038FD2B
:1008D000A94606462846FFF703FD0134A245054612
:1008E000F8DAA0EB0905284603F040FF0746002888
:1008F000C5D003F025FD0446D8F8000003F020FD24
:10090000A9EB060101442A4620460AF01DFEB6E77F
:100910002846FFF7E5FC01370546D4E7032B2BD12A
:10092000C2F30F13022DC2F34172C2EB830205D052
:10093000D8F808305B109A42A8BF1A46A24206DADD
:10094000002211460320BDE8F04703F095BE151BB9
:100950000423291D002291FBF3F1032003F08CFEF8
:10096000074600288BD001352946FFF7FEFEE11C23
:100970002A4631440430C8E7212040E70028F8B572
:1009800004DC1C20BDE8F84000F05EBF0C6814F0E9
:10099000010711D06410FF2C01D91320F2E70022C7
:1009A0000121032003F068FE054618B10121FFF77D
:1009B000DCFE04712846F8BD042CEED9256805F04C
:1009C0000F05042D19D12046FFF774FC3A46C11CCF
:1009D000064691FBF5F1032003F04EFE0546002884
:1009E000E8D03146FFF7C1FE204603F0A9FC3246AD
:1009F0000146281D0AF0A8FDDCE7092D1DD1666817
:100A000076100423F11C3A4691FBF3F1032003F026
:100A100033FE05460028CDD03146FFF7A6FE04344C
:100A2000B742C7DA54F8043FDA0704D55B10FF2B4E
:100A3000B3D8EA1913710137F2E7032DADD125467A
:100A4000B8E77F2902DC017001307047B1F5006F13
:100A50000CDA03468A1162F03F0203F8022B01F020
:100A60003F0161F07F01417018467047B1F5803F4A
:100A70000FDA0B1363F01F030370C1F3851301F04A
:100A80003F0163F07F0361F07F01437081700330A9
:100A90007047B1F5883F0DDAF0230370902343705F
:100AA0008B1101F03F0163F07F0361F07F018370E0
:100AB000C1700430704710B510F0010402D044102A
:100AC000204610BD042812D9026802F00F02042A41
:100AD00007D103F035FC0A222146BDE810400BF097
:100AE000BBB9032A03D10A2221460430F5E70D20C1
:100AF00000F0AAFEE4E7000000282DE9F7430F46C6
:100B000003DC1C2000F0A0FE16E00C6814F00105C8
:100B100006D1042C1FD9236803F00F03042B0DD139
:100B20002046FFF7C8FF6C4601462046FFF789FFC5
:100B3000011B204603F021FE044635E0092B0AD1B3
:100B40006668DFF8849076104FF00108B04504DD48
:100B500000F080FED8B12A20D4E708F1010854F84B
:100B60002800FFF7A8FF7F280BDDB0F5006F0ADB38
:100B7000B0F5803F09DB4845D4BF04200020054480
:100B8000E4E70120FBE70220F9E70320F7E7284626
:100B900003F0ECFD044638B1D7F8008003F0D0FB39
:100BA00001250746B54203DD204603B0BDE8F083CA
:100BB000013558F82500FFF77EFF01463846FFF75C
:100BC00040FF0746EEE700BFFF0F01000128F8B520
:100BD00007460D4604DC1C20BDE8F84000F034BE9A
:100BE0000868FFF768FF06466868FFF764FF022F92
:100BF000044606D0A868FFF75EFF051E02DC292028
:100C0000EAE70125A642D5BFA41B341B94FBF5F4EB
:100C100094FBF5F4D4BF013401344FF0000204F129
:100C200001014FF00900C8BF6D4203F025FD50B12E
:100C30006200034642F0010243F8042F6D00760083
:100C40000022944200DCF8BD46F0010143F8041F85
:100C500001322E44F5E710B5044611F0010011D120
:100C600004290ED90B6803F00F03042B09D10846A1
:100C700003F066FB014620460BF020F8B0FA80F046
:100C8000400910BD0020FCE70128F8B50D4604DC42
:100C90001C20BDE8F84000F0D7BD4E68F20706D42E
:100CA000042E04D9336803F00F02092A01D00B2067
:100CB000EFE7746809686410C3F30F13A34298BF89
:100CC00003F1FF3411F001070DD0481000283ADD80
:100CD000844238DB06EB8003844218DD9A6843F8CF
:100CE000042F0130F8E71A48FFF7B5FF40B10123A0
:100CF000BC4201DA0020F8BD013746F82730F7E79B
:100D000029681448FFF7A7FF50B1002CF2D0012248
:100D1000631C013C9440144346F823207460E9E7C7
:100D20002868C30711D404280FD9036803F00F0300
:100D3000042B0AD1FFF7BFFE0028C8D12968064856
:100D4000FFF789FF08B11220A3E71120A1E700BF38
:100D50004FCC000053CC000035DF0000002310B55D
:100D60000B70C3070C4606D50E4942102046BDE85D
:100D700010400AF067BF28B90B492046BDE8104073
:100D80000AF080BF042801D10849F6E709D90368B1
:100D900003F00F03042B04D103F0D2FA04490246F6
:100DA000E4E710BD0CD9000058CC00005ECC000078
:100DB00063CC00002DE9F04301288FB081460E4638
:100DC00007DC1C2000F040FD054628460FB0BDE8BA
:100DD000F0830B6813F0010440F0A180042B40F273
:100DE000D5801B6803F00F03092B40D1274656F826
:100DF000273013F0010806D1042B04D9186800F03D
:100E00000F00092801D02220DCE75B680137B945D3
:100E100004EB6304EBD10122A11803F02DFC05467D
:100E200008B90025D1E7640044F00104446042465B
:100E300000F1080456F822104B6808685B10C0F3F4
:100E40000F10984298BF00F1FF3304310020834215
:100E500007DC013223EAE373BA4204EB8304E9DBE3
:100E6000B3E751F804CF44F820C00130EFE7032B7B
:100E700040F08C80274656F8270010F00108C2D1B8
:100E80000428C0D9036803F00F02032A38D1C3F342
:100E90000F12C3F34173C3EB82031C440137B945FE
:100EA000E9D10423E11C002291FBF3F1032003F0BC
:100EB000E3FB05460028B4D02146FFF756FC00F1BD
:100EC000040956F82840E10720D4042C1ED92068D4
:100ED00000F00F03032B19D1C0F30F13C0F34170BF
:100EE000C0EB830003344B46A3EB0902824211DBC3
:100EF00008F101080028A8BF8144B845E1DB64E798
:100F0000042A80D1FFF7D6F90444C7E72046FFF74B
:100F1000D1F9E7E714F8012F03F8012BE4E70025E6
:100F20002C4656F82500C20732D4042830D903686D
:100F300003F00F02042A32D1FFF7BCF90444013553
:100F4000A945EED1204603F011FC054600283FF4E8
:100F500068AF041DB04606EB890958F8046BF30727
:100F600028D4042E26D9336803F00F02042A34D182
:100F70003046FFF79FF90746304603F0E1F93A465D
:100F8000014620460AF0E0FA3C4421E02546C8E745
:100F900001A9FFF7E3FE01A80AF09AFECEE7032AB3
:100FA0007FF431AFC3F30F12C3F34173C3EB82037A
:100FB0001C44C4E701A93046FFF7D0FE01A80AF09F
:100FC00087FE01A90646024620460AF0BDFA3444CF
:100FD000C145C2D100232370F7E6032AF8D1C3F339
:100FE0000F17C3F34173C3EB87073A46311DC8E7B8
:100FF0002DE9F04F002893B00F4607DC1C2000F0CD
:1010000023FC0546284613B0BDE8F08F0D6815F0A7
:10101000010806D1042D04D92B6803F00F03092B16
:1010200001D00B20EBE76E687610002E03DC404603
:1010300003F09CFBE5E7012826D04868C20723D4CB
:10104000042821D9036803F00F03042B1CD103F0FB
:1010500077F9044620460AF03BFE0435731E8146AC
:10106000009303FB00FB05EB860A55F8040FC3074A
:1010700071D404286FD9036803F00F02042A05D144
:10108000FFF718F983440AE0384CE3E7032A69D1F3
:10109000C3F30F12C3F34173C3EB82039B44AA450E
:1010A000E3D1584603F062FB05460028AAD0D7F8E2
:1010B00000A0B9F1000F03D0786803F041F90446AD
:1010C000284603F03DF90AF1040307460193019B0A
:1010D00053F804AF0193504603F032F91AF00103BC
:1010E0000146029302D1BAF1040F04D805A9504673
:1010F000FFF734FE05A9084603910AF0E9FDDDE992
:10110000023183468BB9BAF1040F0ED9DAF8000028
:1011100000F00F0CBCF1030F01BFC0F30F13C0F3BD
:1011200041700AF10401C0EB830B38465A460AF0BD
:101130000BFA5F44B9F1000F08D0009B434505DD71
:1011400038464A4621460AF0FFF94F4408F10108A3
:101150004645BCD156E705A9FFF700FE05A80AF0F1
:10116000B7FD8FE703F0ECF8F9E700BFABD1000063
:10117000021E10B513DD0B6813F001041CBF5C10D8
:1011800024EAE474012A00D04A68611C092003F0B3
:1011900073FA18B1640044F00104446010BD0024E7
:1011A0000122F2E70A6838B512F0010436D1042AA8
:1011B00034D91368496803F00F00092818D1506822
:1011C000C3F30F134010834298BF03F1FF30151D86
:1011D000A04205DC01330220984205DB002038BD27
:1011E00045F8041F0134F3E742F820100130F3E71B
:1011F000032813D1C80704D41320BDE8384000F0F9
:1012000023BB4910FF29F7D80432C3F30F1302EBB5
:1012100083039A42E2D202F8011BFAE70B2000F0A6
:1012200013FBDBE72DE9F0414E6816F00107884615
:1012300029D1042E27D9326802F00F03092B12D1CD
:101240007068C2F30F124510AA4200D8551ED8F894
:10125000008018F0010F1AD04FEA6804002C49DD15
:10126000A54220DA46E0042B04D13046FFF722F8ED
:101270000546ECE7032B08D1C2F30F10C2F341720D
:10128000C2EB8005E3E70025E1E73D46DFE74146A5
:101290003248FFF7E0FCA8B10AF06CFC90FBF5F3D4
:1012A00003FB1500441C002F55D1042E53D933687D
:1012B00003F00F03092B26D1013456F824402046B1
:1012C000BDE8F08141462648FFF7C5FCC8B9B8F132
:1012D000040F11D9D8F8003003F00F03042B0BD101
:1012E0004046FFF7E8FB041EB9D141461D48FFF711
:1012F000B2FC08B1122000E01120BDE8F04100F07E
:10130000A3BA2C46CFE7042B1DD1304603F018F8C2
:10131000012C05460FDCFEF7E3FF461B304603F0C9
:1013200025FA04460028CAD003F00AF832462946B6
:101330000AF00AF9C3E72B78013C002BDAD02846E3
:10134000FEF7CEFFE4E7032B05D13444E4786400D4
:1013500044F00104B3E70B20CFE700BF48CC000006
:1013600053CC000035DF00002DE9F0414C6814F04B
:10137000010788462ED1042C2CD923688E6803F0EF
:101380000F02092A13D16568C3F30F136D10AB4226
:1013900000D85D1ED8F800103448FFF75CFC68B335
:1013A000236803F00F03092B1ED1012317E0032A42
:1013B00010D1F20704D41320BDE8F04100F044BA84
:1013C0007710FF2FF7D8C3F30F15C3F34173C3EBA7
:1013D0008505DFE70B20EFE7013344F823609D42EA
:1013E000FADA0020BDE8F081032BFAD1033401239F
:1013F0009D42F6DB04F8017F0133F9E7D8F800805D
:1014000018F0010F0ED04FEA6800002822DD854257
:1014100020DB236803F00F03092B21D1013044F8AE
:101420002060DEE741461248FFF715FCB0B9B8F17D
:10143000040F11D9D8F8003003F00F03042B0BD19F
:101440004046FFF738FB0028E0D141460948FFF746
:1014500002FC08B11220AFE71120ADE72846D8E71B
:10146000032B04BF2418E770BBE700BF4FCC00007C
:1014700053CC000035DF0000086808B5C3071BD453
:10148000042819D9036803F00F02092A01D1406822
:1014900008BD032A09D1C3F30F12C3F34170C0EB97
:1014A0008200400040F00100F2E7042A04D102F07B
:1014B00047FFFEF729FFF4E70120E9E7024A034866
:1014C0000E2104F0C7BE00BFD8CB0000D0CB000077
:1014D000002070470420704701207047002003F06F
:1014E00045B9002070470020704700207047002059
:1014F0007047002070470020704700207047002090
:101500007047002070470000024A03480D2104F094
:10151000A1BE00BFF0CC000058CD0000704703789A
:1015200083B11A0601D40130704703F0C003C02B09
:1015300008BF0130024610460132037803F0C003B1
:10154000802BF8D070470000F8B511F00105064671
:101550001446084626D104293FD90B6803F00F032F
:10156000042B3AD1D30714D4042A36D9136803F0D4
:101570000F03042B31D102F0E3FE0546204602F0B2
:10158000DFFE014628460AF099FB00282DDB1ED11C
:1015900026E002F0D5FE29460A220AF05DFC054647
:1015A000601011E012F0010715D1042A15D9136853
:1015B00003F00F03042B10D110464D1002F0C0FEB3
:1015C0000A2239460AF048FC85420EDB08DD002E6F
:1015D00009DC00200CE04D10E2E7064B0F221A70E8
:1015E0000136022EF5D8042002E0701700F0040046
:1015F000F8BD00BF840200202DE9F0412E4F0646C1
:101600000024E500EB191B79032B0BD00134FF2CD0
:10161000F7D1304604F032FE002814BF04464FF0E4
:10162000FF3445E030460AF053FB31460246E0B253
:1016300004F0ACFE00283BD1EB5959681A1D8842D2
:10164000E4D052F8045FF02D00F10100F7D18000E2
:1016500008301A18D107D9D4042AD7D91B5803F057
:101660000F010429D2D1C3F30F13013302EB83001E
:10167000C507CBD40428C9D952F8233003F00F038F
:10168000042BC3D102F05CFE4FF00308054609218C
:1016900028460AF006FB0028B8D0B8F1010800F18E
:1016A0000105F4D1314628460AF041FB8542ADD10F
:1016B0002046BDE8F08100BF7086012010B510F013
:1016C000010402D04410204610BD042812D902683B
:1016D00002F00F02042A07D102F032FE0A2221464C
:1016E000BDE810400AF0B8BB032A03D10A22214604
:1016F0000430F5E7014B0D221A70E4E78402002064
:1017000010F0010210B516D1042802D90268C2F304
:101710000F1211F0010310D1042902D90B68C3F391
:101720000F13934216D1043000EB83020331904231
:1017300005D301200BE00022EBE70023F1E710F8CE
:10174000014B11F8013F1CB9B3FA83F0400910BDF9
:101750009C42ECD00020FAE72DE9F74F80468946FD
:101760009A46304F304E6AB102233B7001233360FA
:101770003368DFF8D0B00024FC54444504DB03B0E8
:10178000BDE8F08F3260F3E759F824003168C307F1
:1017900007EB0105C1F5487105D5244A43102846D9
:1017A0000AF01CFA04E0C8B9214A28460AF016FAE1
:1017B0001C480AF08DFA3060BAF1000F0CD008F125
:1017C000FF33A34208DDB0F5487F05D2431C202239
:1017D0003A540022FA5433600134CEE7042801D190
:1017E000144AE2E71BD9026802F00F03042B06D16A
:1017F000019102F0A5FD104A01990346CFE7092B9C
:1018000003D143685A465B10C9E7032B08D1C2F3E2
:101810000F13C2F34172C2EB8303084ABFE70123EF
:10182000074ABCE785020020A80500200CD900006B
:1018300058CC00005ECC00003BDF0000DFCF000092
:10184000EACF0000D0CF0000014B18700020704795
:1018500084020020024B1878003018BF0120704726
:101860008402002008B500231A46FFF775FF034BDA
:101870000348196805F004FA002008BDA8050020F7
:101880008502002010B502F099FA084C231D01468C
:101890001F2218460AF036FA0AF01AFA04308008B5
:1018A000000140F004002060204610BD60020020CE
:1018B0002DE9F04F85B000F1180104690291D0E9DB
:1018C0000232824601EB8404BC4F4169029800EB6E
:1018D0008109397803EB820529BB53F82230B84AD5
:1018E0001E1203F07F03043552F82330904643F074
:1018F000010318479AF8010005F0A0F900238AF8BF
:10190000003021E03B7873B92B681E1203F07F038F
:10191000043558F82330EAE7029A231D9A1AD82A88
:1019200026DD1A233B70DAF808209AF8023039785D
:101930009AF80100AA1A921043EA022205F084F9EB
:1019400000238AF800303B70DAF80830ED1A029B69
:10195000E41AA9EB0309AD10A4104FEAA903CAF8D1
:101960000C50CAF81040CAF8143005B0BDE8F08F2A
:1019700022461C463B781660002BD4D12B681E12E1
:1019800003F07F03043558F82330B0E7029A231D93
:101990009A1AD82A02DD1A233B70C4E721461C4656
:1019A0002B680B603B782A1D0BB11546BBE76B68B3
:1019B0001E1203F07F03083558F8233097E7029A88
:1019C000231D9A1AD82A02DD1A233B70ABE7224660
:1019D0001C463B7805EB86061660002BA3D12B68CE
:1019E0001E1203F07F03043558F823307FE7029A74
:1019F000231D9A1AD82A02DD1A233B7093E7224648
:101A00001C46704B53F8263013603B78002B8AD16C
:101A10002B681E1203F07F03043558F8233066E765
:101A2000684B54F8042D43F826203B78002B7FF4B4
:101A30007AAF2B681E1203F07F03043558F8233069
:101A400055E7DFF880B15BF82600FFF737FE3A78FC
:101A50005AB9009054F8040DFFF730FE009B18446B
:101A6000400040F001004BF826003B78002B7FF44B
:101A70005AAF2B681E1203F07F03043558F8233049
:101A800035E7029B221DD31AD82B02DD1A233B70A7
:101A900049E7029B21464B4534BF59F80C3C0123D2
:101AA0000B603B781446002B7FF43DAF2B681E1271
:101AB00003F07F03043558F8233018E7029B221DFA
:101AC000D31AD82B02DD1A233B702CE7029B4B451F
:101AD00018D259F80C3C06F180465B10C3EB8373B7
:101AE000033E334459F8233023603B781446002BDF
:101AF0007FF419AF2B681E1203F07F03043558F8EA
:101B00002330F4E618233B700023EDE7029B4B459E
:101B100018D259F80C3C54F8042D5B1006F180469D
:101B2000C3EB8373033E334449F823203B78002BF7
:101B30007FF4F9AE2B681E1203F07F03043558F8CA
:101B40002330D4E618233B70F0E7029B4B4529D2A3
:101B500059F80C3C06F180465B10033EC3EB8373DF
:101B6000334459F82300FFF7A9FD834654F8040DC8
:101B7000FFF7A4FD59F80C3C5B10C3EB837358448A
:101B80001E44400040F0010049F826003B78002B3D
:101B90007FF4C9AE2B681E1203F07F03043558F89A
:101BA0002330A4E618233B70F0E7029A231D9A1A0B
:101BB000D82A09DD1A233B70B5E600BF8402002055
:101BC000D0CD0000688E012022461C4659F82630F0
:101BD00013603B78002B7FF4A6AE2B681E1203F037
:101BE0007F03043558F8233081E654F8043D49F862
:101BF00026303B78002B7FF496AE2B681E1203F044
:101C00007F03043558F8233071E659F826004FEA6F
:101C1000600B54F8040DFFF751FD584440003B7829
:101C200040F0010049F82600002B7FF47CAE2B68C1
:101C30001E1203F07F03043558F8233057E6029B49
:101C4000A4EB8604A3420BD83B78002B7FF46BAE49
:101C50002B681E1203F07F03043558F8233046E644
:101C6000C84802F05DFB3B78002B7FF45CAE2B682C
:101C70001E1203F07F03043558F8233037E6002E98
:101C800005EB8605FFF660AE3B78002B7FF44BAE8C
:101C90002B681E1203F07F03043558F8233026E624
:101CA00054F8043D042B04D1002E05EB8605FFF605
:101CB0004BAE3B78002B7FF436AE2B681E1203F040
:101CC0007F03043558F8233011E654F8043D042B03
:101CD00004D0002E05EB8605FFF636AE3B78002BD0
:101CE0007FF421AE2B681E1203F07F03043558F8F1
:101CF0002330FCE554F8040CC307A4F1040B0BD506
:101D00004010013800280ADB400040F0010005EBDC
:101D10008605CBF8000017E6FFF7D0FCF1E73B782B
:101D20000BB15C46FFE52B681E1203F07F035C4697
:101D300058F823300435DAE5029A029B04F10C0BC3
:101D4000ABEB0202A9EB0303D82A4FEAA30302DD9F
:101D50001A233B70E7E5A146740004F4FF7646F0D1
:101D60000106C9F80060DAF808209AF80200AD1AF6
:101D7000AD1040EA052040005B0043F0010340F055
:101D80000100C9F80400C9F808303A788AF802E07E
:101D900051F83C30CAF808305C461AB103F1080526
:101DA000D946C0E503F10C059B681E1203F07F03C2
:101DB000D94658F823309AE5029B54F8046C4B45F9
:101DC0002FD1F70720D4042E17D9336803F00F035F
:101DD000042B13D1304602F0B3FA09F079FFB0F5C5
:101DE000487F28BF4FF448700630643004F014FB7D
:101DF00070B9043DDDF80890A6E507D0002E14BFA9
:101E00004FF400700720F0E70A20EEE70720ECE728
:101E100031469AF8010004F02EFF00238AF80030C2
:101E2000E8E759F80C3C58495A106FF00303534344
:101E30000C3B09EB030449F8036059F8083C5A10BD
:101E40008AF80220D2B2C3F3552351F83220CAF8DF
:101E5000082059F8041C4FEA6109029901EB89092D
:101E60003978043402EB830500297FF45CAD52F825
:101E700023301E1203F07F03043558F8233036E573
:101E800054F8040CFFF71AFC1E288346A4EB8604C2
:101E900025DC00280BDC3B78002B7FF444AD2B685D
:101EA0001E1203F07F03043558F823301FE501F0BC
:101EB00071FFABF1030B354E834401F06BFFA0EBD8
:101EC0000B00B042F9D83B78002B7FF42CAD2B6887
:101ED0001E1203F07F03043558F8233007E5012371
:101EE0008AF8003001F056FF0A385844CAF8040056
:101EF0002AE554F8040CFFF7E1FBA4EB8604061E68
:101F00000BDC3B78002B7FF40EAD2B681E1203F028
:101F10007F03043558F82330E9E41D4B9E4202DD6F
:101F20001D233B70FFE401238AF8003001F032FFEB
:101F30004FF47A7303FB06000A38D7E700233046D4
:101F4000A4EB8604134E1A462146FFF705FC3168C0
:101F5000114802F012FC114B316818600E4804F071
:101F60003BFD31680C4804F08BFE3B78002B7FF47E
:101F7000DAAC2B681E1203F07F03043558F82330C7
:101F8000B5E400BFFCCF0000708601203F420F0087
:101F900080EE3600A8050020850200200800002001
:101FA0003B78A4EB8604002B7FF4BDAC2B681E129B
:101FB00003F07F03043558F8233098E4504604F0CA
:101FC0008FFA3B78002B7FF4AEAC2B681E1203F027
:101FD0007F03043558F8233089E454F8043C002B7F
:101FE00044D154F80C0C10F0010B1ED04FEA600BDA
:101FF0004FEA4B0343F0010344F8083CBBF1000FE8
:1020000040F388804FEA4B0343F0010354F80C0C73
:1020100044F8043C54F8083CC107CBEB63032AD5D1
:1020200001335B0043F0010330E004281BD903684F
:1020300003F00F02092A01D14068D7E7042A09D129
:1020400002F07EF90378002BD2D0FFF768FA0BF18B
:10205000010BF7E7032A06D1C3F30F1BC3F3417348
:10206000C3EB8B0BC4E719233B705CE44FEA630BB3
:102070000BF1FF3BC2E7042849D9026802F00F02C6
:10208000092A11D103F1020B50F82B3049F8263000
:102090003B78002B7FF447AC2B681E1203F07F03C4
:1020A000043558F8233022E4042A2BD1039309EB9A
:1020B0008603009302F044F9039B83465E1C012EC5
:1020C00012DC5846FFF72BFAA0EB0B06304602F065
:1020D0004DFB034670B1039002F032F93246594687
:1020E00009F032FA039B05E09BF80030013E23B96A
:1020F00012223A70009A1360CAE75846FFF70FFAA7
:102100008346DCE7032A02D11844037989E71923BF
:102110003B7008E40435BBE7029A04EB86039B1A84
:10212000D82B11DC0122002E06F1FF3310DC3B78A6
:10213000002B7FF4F8AB2B681E1203F07F030435ED
:1021400058F82330FFF7D3BB1A233B70FFF7EBBBE4
:1021500022601E460434E6E7029A231D9B1AD82B00
:1021600003DD1A233B70FFF7DEBB029B4B452AD2EF
:1021700054F8040CFFF7A2FA002821DD59F80C3CB2
:102180005B1083421CDBC3EB8373184400F1804077
:102190000438A4EB860359F820201A606FF003007E
:1021A0003B7800FB06440434002B7FF4BCAB2B6867
:1021B0001E1203F07F03043558F82330FFF797BB56
:1021C00020233B70EAE71823FBE7C04B1A68A4EB17
:1021D00086036FF003001A603B7800FB064404346A
:1021E000002B7FF4A0AB2B681E1203F07F03043595
:1021F00058F82330FFF77BBB54F8043C042B3B78A2
:10220000A4F1040204BF05EB8605224613B114466F
:10221000FFF789BB2B681E1203F07F03144658F8A2
:1022200023300435FFF763BB54F8043D042B1CBF77
:10223000002323603B781CBF05EB86050434002B8C
:102240007FF471AB2B681E1203F07F03043558F83E
:102250002330FFF74CBB002EA4EB860115DC1C23BA
:102260003B7000226FF003003B780A6000FB0644DD
:102270000434002B7FF457AB2B681E1203F07F034E
:10228000043558F82330FFF732BB0B684FF0000CD1
:102290005B1051F82C0010F0010202D10D233B70AD
:1022A000E0E7401083420CF1010CA8BF03466645ED
:1022B000EFDC5B0043F00102D4E7002EA4EB8601C3
:1022C00015DC1C233B7000226FF003003B780A6092
:1022D00000FB06440434002B7FF425AB2B681E1250
:1022E00003F07F03043558F82330FFF700BB0B6879
:1022F0004FF0000C5B1051F82C0010F0010202D1DD
:102300000D233B70E0E7401083420CF1010CB8BF95
:1023100003466645EFDC5B0043F00102D4E754F866
:10232000081C11F0010F4FEA86031ED054F8042C4C
:10233000D0071AD55210B2EB610FA4EB0303D4BF40
:10234000002204221A606FF003003B7800FB064471
:102350000434002B7FF4E7AA2B681E1203F07F03DE
:10236000043558F82330FFF7C2BA54F8042C6FF044
:102370000100A4EB030BFFF7E7F8CBF80000E2E75E
:1023800054F8081C11F0010F4FEA86031ED054F8D0
:10239000042CD0071AD55210B2EB610FA4EB030343
:1023A000B4BF002204221A606FF003003B7800FBE8
:1023B00006440434002B7FF4B6AA2B681E1203F0E7
:1023C0007F03043558F82330FFF791BA54F8042CF2
:1023D0004FF0FF30A4EB030BFFF7B6F8CBF800008B
:1023E000E2E754E9020181424FEA860314D1E31A7D
:1023F00004221A606FF003003B7800FB06440434AB
:10240000002B7FF490AA2B681E1203F07F03043583
:1024100058F82330FFF76BBA0428A4EB030B01D85C
:10242000002315E0C307FBD4036803F00F03042B5C
:10243000F6D1CB07F4D40429F2D90B6803F00F03CB
:10244000042BEDD1FFF75CF900280CBF0023042317
:10245000CBF80030CEE754E9020181424FEA86030F
:1024600014D1E31A00221A606FF003003B7800FBDE
:1024700006440434002B7FF456AA2B681E1203F086
:102480007F03043558F82330FFF731BA0428A4EB52
:10249000030B01D8042315E0C307FBD4036803F042
:1024A0000F03042BF6D1CB07F4D40429F2D90B681F
:1024B00003F00F03042BEDD1FFF722F900280CBF26
:1024C00004230023CBF80030CEE700BF0800002033
:1024D00054F8081C11F0010F4FEA86031ED054F87F
:1024E000042CD0071AD55210B2EB610FA4EB0303F2
:1024F000CCBF002204221A606FF003003B7800FB7F
:1025000006440434002B7FF40EAA2B681E1203F03D
:102510007F03043558F82330FFF7E9B954F8042C49
:102520000120A4EB030BFFF70FF8CBF80000E3E763
:1025300054F8081C11F0010F4FEA86031ED054F81E
:10254000042CD0071AD55210B2EB610FA4EB030391
:10255000ACBF002204221A606FF003003B7800FB3E
:1025600006440434002B7FF4DEA92B681E1203F00E
:102570007F03043558F82330FFF7B9B954F8042C19
:102580000220A4EB030BFEF7DFFFCBF80000E3E72C
:1025900054F8043C042BA4EB860314BF042200224D
:1025A0001A606FF003003B7800FB06440434002BF4
:1025B0007FF4B9A92B681E1203F07F03043558F885
:1025C0002330FFF794B954F8080CFFF777F88346E7
:1025D00054F8040CFFF772F85844A4EB860340004B
:1025E00040F0010018606FF003003B7800FB0644E8
:1025F0000434002B7FF497A92B681E1203F07F038D
:10260000043558F82330FFF772B954F8080CFFF777
:1026100055F8834654F8040CFFF750F8ABEB000074
:10262000A4EB8603400040F0010018606FF0030047
:102630003B7800FB06440434002B7FF474A92B681C
:102640001E1203F07F03043558F82330FFF74FB90B
:1026500054F8080CFFF732F8834654F8040CFFF7DF
:102660002DF800FB0BF0A4EB8603400040F00100C6
:1026700018606FF003003B7800FB06440434002B25
:102680007FF451A92B681E1203F07F03043558F81C
:102690002330FFF72CB954F8040CFFF70FF88346EA
:1026A000B8B91F233B70A4EB86036FF00300C3F897
:1026B00000B03B7800FB06440434002B7FF433A9C0
:1026C0002B681E1203F07F03043558F82330FFF700
:1026D0000EB954F8080CFEF7F1FF90FBFBFB4FEA34
:1026E0004B0B4BF0010BDEE754F8040CFEF7E6FF52
:1026F0008346B8B91F233B70A4EB86036FF0030039
:10270000C3F800B03B7800FB06440434002B7FF490
:102710000AA92B681E1203F07F03043558F82330F2
:10272000FFF7E5B854F8080CFEF7C8FF90FBFBF381
:1027300003FB1B0B4FEA4B0B4BF0010BDCE754F890
:10274000040CFEF7BBFF0028B8BF4042A4EB860391
:10275000400040F0010018606FF003003B7800FB80
:1027600006440434002B7FF4DEA82B681E1203F00D
:102770007F03043558F82330FFF7B9B8012EA4EBD6
:10278000860B32D1DBF80000FEF798FF02460028E6
:10279000B4BF4FF0FF330123934202DC11461A46C7
:1027A0000B4601339B1A0392009309F0E3F9009B57
:1027B000039A90FBF3F101FB130313445B0043F016
:1027C0000103CBF800306FF003003B7800FB0644B8
:1027D0000434002B7FF4A7A82B681E1203F07F039C
:1027E000043558F82330FFF782B8022E0BD1DBF8FE
:1027F0000000FEF763FF0090DBF80400FEF75EFFC9
:10280000009B0246C8E764230122CAE7A4EB860BBB
:102810005946304602F007F93B78CBF800006FF0DC
:10282000030000FB06440434002B7FF47CA82B68D3
:102830001E1203F07F03043558F82330FFF757B812
:1028400054F8080CFEF73AFF834654F8040CFEF7E0
:1028500035FF0BEA0000A4EB8603400040F00100C6
:1028600018606FF003003B7800FB06440434002B33
:102870007FF459A82B681E1203F07F03043558F823
:102880002330FFF734B854F8080CFEF717FF8346DF
:1028900054F8040CFEF712FF4BEA0000A4EB860389
:1028A000400040F0010018606FF003003B7800FB2F
:1028B00006440434002B7FF436A82B681E1203F064
:1028C0007F03043558F82330FFF711B854F8080C8B
:1028D000FEF7F4FE834654F8040CFEF7EFFE8BEA95
:1028E0000000A4EB8603400040F0010018606FF088
:1028F00003003B7800FB06440434002B7FF413A84C
:102900002B681E1203F07F03043558F82330FEF7BE
:10291000EEBF54F8040CFEF7D1FEC043A4EB8603CF
:10292000400040F0010018606FF003003B7800FBAE
:1029300006440434002B7EF4F6AF2B681E1203F01D
:102940007F03043558F82330FEF7D1BF54F8080C44
:10295000FEF7B4FE834654F8040CFEF7AFFE0BFA04
:1029600000F0A4EB8603400040F0010018606FF017
:1029700003003B7800FB06440434002B7EF4D3AF05
:102980002B681E1203F07F03043558F82330FEF73E
:10299000AEBF54F8080CFEF791FE834654F8040CC1
:1029A000FEF78CFE4BFA00F0A4EB8603400040F0EB
:1029B000010018606FF003003B7800FB064404340C
:1029C000002B7EF4B0AF2B681E1203F07F0304359A
:1029D00058F82330FEF78BBF54F80C0CFEF76EFE50
:1029E000834654F8080CFEF769FE8BFB002354F86D
:1029F000040CCDE90023FEF761FEDDE90023C0F100
:102A0000200CB0F1200103FA0CFC22FA00F040EA9D
:102A10000C005CBF43FA01F10843A4EB860E4000B2
:102A200040F00100CEF800003B786FF0030000FB9F
:102A300006440434002B7EF476AF2B681E1203F09C
:102A40007F03043558F82330FEF751BFA4EB860B03
:102A500059463046FEF78CFB3B78CBF800006FF010
:102A6000030000FB06440434002B7EF45CAF2B68AB
:102A70001E1203F07F03043558F82330FEF737BFEA
:102A8000A4EB860421463046FEF78CFB3B78002BF6
:102A90007EF449AF2B681E1203F07F03043558F80B
:102AA0002330FEF724BFA4EB860B59463046FEF7D1
:102AB000B9FB3B78CBF800006FF0030000FB064445
:102AC0000434002B7EF42FAF2B681E1203F07F031B
:102AD000043558F82330FEF70ABFA4EB86042146DC
:102AE0003046FEF741FC3B78002B7EF41CAF2B6890
:102AF0001E1203F07F03043558F82330FEF7F7BEAB
:102B0000A4EB860B59463046FEF7B6FC3B78CBF873
:102B100000006FF0030000FB06440434002B7EF439
:102B200002AF2B681E1203F07F03043558F82330E0
:102B3000FEF7DDBE54F8040C01F002FC54F8083C2A
:102B4000DA072AD4042B0CD91B6803F00F03013BCE
:102B5000082B10D8DFE803F0052127230F0F0F0FF4
:102B60002500CC4909F0AAF8A4EB8603002814BF7D
:102B7000002204221A606FF003003B7800FB064439
:102B80000434002B7EF4CFAE2B681E1203F07F03BB
:102B9000043558F82330FEF7AABEBF49E2E7BF4923
:102BA000E0E7BF49DEE7BF49DCE7029B261DF31AD9
:102BB000D82B03DD1A233B70FEF7B5BE01F0F2F807
:102BC0002346400040F0010018603B783446002B5B
:102BD0007EF4A9AE2B681E1203F07F03043558F86B
:102BE0002330FEF784BE029B261DF31AD82B03DD8B
:102BF0001A233B70FEF797BE01F0CCF8AA4B224691
:102C000003EA40003B7840F0010034461060002B9E
:102C10007EF489AE2B681E1203F07F03043558F84A
:102C20002330FEF764BE029B261DF31AD82B03DD6A
:102C30001A233B70FEF777BE01F0B4F89B4B1B687C
:102C400098423DBFC3F5830303F63713C018C01A7B
:102C50004000234640F0010018603B783446002BCA
:102C60007EF461AE2B681E1203F07F03043558F822
:102C70002330FEF73CBE01F095F88C4B18603B7892
:102C8000A4EB8604002B7EF44EAE2B681E1203F0DC
:102C90007F03043558F82330FEF729BE03F0A8FB64
:102CA000B30068B9E41A3B78002B7EF43CAE2B6885
:102CB0001E1203F07F03043558F82330FEF717BEC9
:102CC000304627467A4EE41A01231A462146FEF77B
:102CD00043FD3068643003F09FFB18B9043D3C4667
:102CE000FEF732BE9AF801203168724803F0DBFF2C
:102CF00001238AF8003001F04DF86F4A33681268FA
:102D0000063302FB0300FFF7F1B803F071FBB300D9
:102D100068B9E41A3B78002B7EF405AE2B681E12CE
:102D200003F07F03043558F82330FEF7E0BD30464A
:102D300027465F4EE41A002201232146FEF70CFDD0
:102D40003068643003F068FB0028C7D0594803F0AE
:102D50002BFDCDE7FEF796FDA4EB860B3B78CBF879
:102D600000006FF0030000FB06440434002B7EF4E7
:102D7000DAAD2B681E1203F07F03043558F82330B8
:102D8000FEF7B5BD3B78A4EB8604002B7EF4CBADFB
:102D90002B681E1203F07F03043558F82330FEF72A
:102DA000A6BDA4EB860B584601F033F83B78CBF870
:102DB00000006FF0030000FB06440434002B7EF497
:102DC000B2AD2B681E1203F07F03043558F8233090
:102DD000FEF78DBDA4EB860B584601F01CF83B783E
:102DE000CBF800006FF0030000FB06440434002B16
:102DF0007EF499AD2B681E1203F07F03043558F85A
:102E00002330FEF774BDA4EB860B5946304600F024
:102E10008FFC3B78CBF800006FF0030000FB06440A
:102E20000434002B7EF47FAD2B681E1203F07F0369
:102E3000043558F82330FEF75ABDA4EB860420462B
:102E400000F0ECFF3B78002B7EF46DAD2B681E127A
:102E500003F07F03043558F82330FEF748BDA4EB98
:102E6000860B5946304600F0D7FB3B78CBF8000084
:102E70006FF0030000FB06440434002B7EF453ADD6
:102E80002B681E1203F07F03043558F82330FEF739
:102E90002EBD00BF0CD0000014D000001BD00000DD
:102EA00022D0000027D00000FEFFFF7FB0050020E9
:102EB000A80500208502002004000020A4EB860461
:102EC000204601F091F83B78002B7EF42CAD2B6866
:102ED0001E1203F07F03043558F82330FEF707BDB8
:102EE0000121304601F04EF83B78002B7EF41BADFB
:102EF0002B681E1203F07F03043558F82330FEF7C9
:102F0000F6BC0021304601F03DF83B78002B7EF402
:102F10000AAD2B681E1203F07F03043558F82330E6
:102F2000FEF7E5BCA4EB860B584600F0E3FF3B78C8
:102F3000CBF800006FF0030000FB06440434002BC4
:102F40007EF4F1AC2B681E1203F07F03043558F8B1
:102F50002330FEF7CCBCA4EB860B584600F0DEFF16
:102F60003B78CBF800006FF0030000FB064404340C
:102F7000002B7EF4D8AC2B681E1203F07F030435BF
:102F800058F82330FEF7B3BCA4EB8604204600F0CB
:102F900093FF3B78002B7EF4C6AC2B681E1203F027
:102FA0007F03043558F82330FEF7A1BCA4EB860458
:102FB000204604F085FB3B78002B7EF4B4AC2B68F4
:102FC0001E1203F07F03043558F82330FEF78FBC40
:102FD000A4EB860B584604F049FC3B78CBF8000084
:102FE0006FF0030000FB06440434002B7EF49BAC1E
:102FF0002B681E1203F07F03043558F82330FEF7C8
:1030000076BCA4EB8604204604F0AAFA3B78002B99
:103010007EF489AC2B681E1203F07F03043558F848
:103020002330FEF764BCA4EB860B584604F0B4FAD8
:103030003B78CBF800006FF0030000FB064404343B
:10304000002B7EF470AC2B681E1203F07F03043556
:1030500058F82330FEF74BBCA4EB860421463046DB
:1030600002F014F93B78002B7EF45DAC2B681E1245
:1030700003F07F03043558F82330FEF738BCA4EB87
:1030800086042146304601F0E7FE3B78002B7EF4B3
:103090004AAC2B681E1203F07F03043558F8233026
:1030A000FEF725BCA4EB86042146304601F0A8FFBC
:1030B0003B78002B7EF437AC2B681E1203F07F03A5
:1030C000043558F82330FEF712BCA4EB86042146E1
:1030D000304601F0BBFF3B78002B7EF424AC2B681C
:1030E0001E1203F07F03043558F82330FEF7FFBBB0
:1030F000A4EB860B5946304604F0CCFC3B78CBF869
:1031000000006FF0030000FB06440434002B7EF443
:103110000AAC2B681E1203F07F03043558F82330E5
:10312000FEF7E5BBA4EB860B5946304604F0BAFC2B
:103130003B78CBF800006FF0030000FB064404343A
:10314000002B7EF4F0AB2B681E1203F07F030435D6
:1031500058F82330FEF7CBBBA4EB860B594630461C
:1031600004F0A8FC3B78CBF800006FF0030000FBF4
:1031700006440434002B7EF4D6AB2B681E1203F0F9
:103180007F03043558F82330FEF7B1BBA4EB860B60
:103190005946304604F080F83B78CBF800006FF0D9
:1031A000030000FB06440434002B7EF4BCAB2B6808
:1031B0001E1203F07F03043558F82330FEF797BB47
:1031C000A4EB86042146304601F0E4FF3B78002B57
:1031D0007EF4A9AB2B681E1203F07F03043558F868
:1031E0002330FEF784BBA4EB86042146304601F071
:1031F00055FF3B78002B7EF496AB2B681E1203F034
:103200007F03043558F82330FEF771BBA4EB860B1F
:103210005946304601F0BCFE3B78CBF800006FF019
:10322000030000FB06440434002B7EF47CAB2B68C7
:103230001E1203F07F03043558F82330FEF757BB06
:10324000A4EB86042146304601F04CFE3B78002B6F
:103250007EF469AB2B681E1203F07F03043558F827
:103260002330FEF744BB002E40F38180012E54F83A
:1032700004BC40D11BF0010F4AD1BBF1040F47D968
:10328000DBF8003003F00F03042B41D1584601F066
:1032900057F8FEF7B1F903465A1CA4EB860466D032
:1032A000022E45D11BF0010F3BD1BBF1040F38D9E1
:1032B000DBF8002002F00F02092A32D1DBF804000B
:1032C000261FC0F347000122824224DD04EB800464
:1032D000FF2B2FD840EA03264FEA262E48495FFAF3
:1032E0008EFC01EBCC031B79032B3EF425AD0223AE
:1032F0003B70FEF718BB022E0AD154F8080CC10728
:1033000006D4042804D9036803F00F03042BBED0AD
:103310004FF0FF33C0E701325BF8221046F8041F7C
:10332000D2E70B233B70002323600434FEF7FBBA83
:103330000020CDE7029AA21AA4EB800B9210CAF8E3
:103340001020594698472F4A002313603B78CBF84A
:1033500000000BF10404002B7EF4E5AA2B681E127A
:1033600003F07F03043558F82330FEF7C0BA00237A
:1033700023603B78221D13B11446FEF7D4BA2B68A4
:103380001E1203F07F03144658F823300435FEF76D
:10339000AEBA029BE31A9B10A4EB8604CAF8103065
:1033A0002146304603F044FA3B78002B7EF4BBAA5A
:1033B0002B681E1203F07F03043558F82330FEF704
:1033C00096BA029BE31A9B10A4EB860BCAF8103046
:1033D0005946304603F02CFA3B78CBF800006FF0EA
:1033E000030000FB06440434002B7EF49CAA2B68E7
:1033F0001E1203F07F03043558F82330FEF777BA26
:1034000070860120546D01202DE9F84F224D0023D4
:10341000002B03F1FF3706DA01F04EFF03F018FB33
:1034200003F0F0FC19270026DFF878803046D8F842
:103430000020B24215DD2B68184C01339342A8BF1F
:1034400000232B60D5F80090F02303FB09F304EB75
:10345000030AE35CA346EBB1022B04D15046FEF70E
:1034600027FA3B46D4E7012B0ED108B900F092FCB5
:10347000F02303FB09F39B440949DBF80420821A7B
:103480008A429CBF0222E254F02303FB09F3E35C6F
:10349000022BE3D00136CAE700000020107D012096
:1034A0003F420F00AC0500200A4B4FF480721A60B7
:1034B000094B01211964D3F840250532C3F848258A
:1034C000C3F84C254FF44022C3F80423034B197072
:1034D000704700BF00E100E000800040D7050020F9
:1034E00004207047F8B5D1E9004514F001002DD053
:1034F00015F001002AD064101C2C3CD81F4F6D1011
:1035000041F288363B5DAE42A8BF2E46012B05D066
:103510000121204605F054FF01233B55184B1B7831
:103520000BB9FFF7C1FF002D4FF00003154A0EDC69
:10353000154940F2DC50FF25D65CB44204BF21F8A7
:103540001300D5540133042BF6D10420F8BDD15C0F
:103550008C4203D10C4A22F81360F6E70133042BA6
:10356000F5D10023D15CFF2901D1D454F2E7013316
:10357000042BF7D1E9E70020E8E700BFB8050020F9
:10358000D70500201C0000200E00002070B5D1E9F6
:10359000004514F001001BD015F0010018D0641094
:1035A0001D2C28BF1B24154E335D012B05D0012196
:1035B000204605F005FF01233355114B6D10A5F191
:1035C00010029A420F4B04D94FF0FF321A600420C8
:1035D00070BD1C600C4B0D4890FBF5F018800C4B37
:1035E0001B780BB9FFF760FF0A4B01229A64D3F8EE
:1035F00048251044C3F84805E9E700BFB805002096
:1036000090860100180000200C00002020A1070077
:10361000D70500200080004070B50C68E30704D493
:103620000D20FEF711F9012070BD64101C2C14D878
:10363000012814DD4B68042B14BF002502250A4E17
:10364000335DAB4204D02946204605F0B9FE35551E
:10365000204605F0FBFE012803D00020E4E700250A
:10366000EDE70420E0E700BFB805002070B50D6865
:103670000128CCBF4C68012415F0010042D014F0A1
:1036800001003FD06D10002D05DC1F4B0122C3F857
:103690000825002036E064101C2CFAD81B4E335D40
:1036A000012B05D00121204605F08AFE0123335568
:1036B0000A22174B93FBF5F3053393FBF2F3154AFC
:1036C000154952F824201548120242F00312C1F89D
:1036D00010250D4AC2F81005C2F814150121C2F8D0
:1036E0000415A2F5A83210690020C2F810054FF6A3
:1036F000FF708342A8BF0346C2F840350420C2F8D9
:103700000012116070BD00BF00F00140B80500203C
:1037100000B4C40410E300000060004040A1004079
:10372000002802DC1C20FEF78FB801207047000043
:10373000F8B50B68DA0707460D4604D40D20FEF7EE
:1037400083F8012007E05B10062B05D103F036FF5C
:10375000400040F00100F8BDF3D80C4A0C4E52F87E
:103760002340335D2BB10021204605F029FE0023C4
:103770003355012F06DD6B68042B03D1022120464F
:1037800005F01EFE204605F025FDE1E7A4D000006F
:10379000B805002010B510F0010402D044102046F6
:1037A00010BD042812D9026802F00F02042A07D1C2
:1037B00000F0C6FD0A222146BDE8104008F04CBBCF
:1037C000032A03D10A2221460430F5E70D20FEF733
:1037D0003BF8E4E70228F8B50C4604DC1C20BDE801
:1037E000F840FEF731B80868FFF7D4FF0646606876
:1037F000FFF7D0FF0546A0686E4CFFF7CBFF1C2DEE
:1038000094FBF0F400F2B5826B4F7B5D012B05D089
:103810000121284605F0D4FD01237B5500212846CF
:1038200005F0F8FD002C3CD02046013800BF00BF59
:1038300000BF00BF00BF00BF00BF00BF00BF00BF90
:1038400000BF00BF00BF00BF00BF00BF00BF00BF80
:1038500000BF00BF00BF00BF00BF00BF00BF00BF70
:1038600000BF00BF00BF00BF00BF00BF00BF00BF60
:1038700000BF00BF00BF00BF00BF00BF00BF00BF50
:1038800000BF00BF00BF00BF00BF00BF00BF00BF40
:1038900000BF00BF00BF00BF00BF00BF00BF00BF30
:1038A000C3D106F00101284605F0B4FD002C3CD040
:1038B0002046013800BF00BF00BF00BF00BF00BFEF
:1038C00000BF00BF00BF00BF00BF00BF00BF00BF00
:1038D00000BF00BF00BF00BF00BF00BF00BF00BFF0
:1038E00000BF00BF00BF00BF00BF00BF00BF00BFE0
:1038F00000BF00BF00BF00BF00BF00BF00BF00BFD0
:1039000000BF00BF00BF00BF00BF00BF00BF00BFBF
:1039100000BF00BF00BF00BF00BF00BF00BF00BFAF
:1039200000BF00BF00BF00BFC3D1C6F3400128469F
:1039300005F070FD002C41D02046013800BF00BFCB
:1039400000BF00BF00BF00BF00BF00BF00BF00BF7F
:1039500000BF00BF00BF00BF00BF00BF00BF00BF6F
:1039600000BF00BF00BF00BF00BF00BF00BF00BF5F
:1039700000BF00BF00BF00BF00BF00BF00BF00BF4F
:1039800000BF00BF00BF00BF00BF00BF00BF00BF3F
:1039900000BF00BF00BF00BF00BF00BF00BF00BF2F
:1039A00000BF00BF00BF00BF00BF00BF00BF00BF1F
:1039B000C3D103E040420F00B8050020C6F38001E8
:1039C000284605F027FD002C3CD02046013800BFDA
:1039D00000BF00BF00BF00BF00BF00BF00BF00BFEF
:1039E00000BF00BF00BF00BF00BF00BF00BF00BFDF
:1039F00000BF00BF00BF00BF00BF00BF00BF00BFCF
:103A000000BF00BF00BF00BF00BF00BF00BF00BFBE
:103A100000BF00BF00BF00BF00BF00BF00BF00BFAE
:103A200000BF00BF00BF00BF00BF00BF00BF00BF9E
:103A300000BF00BF00BF00BF00BF00BF00BF00BF8E
:103A400000BFC3D1C6F3C001284605F0E3FC002C3B
:103A50003CD02046013800BF00BF00BF00BF00BF00
:103A600000BF00BF00BF00BF00BF00BF00BF00BF5E
:103A700000BF00BF00BF00BF00BF00BF00BF00BF4E
:103A800000BF00BF00BF00BF00BF00BF00BF00BF3E
:103A900000BF00BF00BF00BF00BF00BF00BF00BF2E
:103AA00000BF00BF00BF00BF00BF00BF00BF00BF1E
:103AB00000BF00BF00BF00BF00BF00BF00BF00BF0E
:103AC00000BF00BF00BF00BF00BFC3D1C6F30011DD
:103AD000284605F09FFC002C3CD02046013800BF52
:103AE00000BF00BF00BF00BF00BF00BF00BF00BFDE
:103AF00000BF00BF00BF00BF00BF00BF00BF00BFCE
:103B000000BF00BF00BF00BF00BF00BF00BF00BFBD
:103B100000BF00BF00BF00BF00BF00BF00BF00BFAD
:103B200000BF00BF00BF00BF00BF00BF00BF00BF9D
:103B300000BF00BF00BF00BF00BF00BF00BF00BF8D
:103B400000BF00BF00BF00BF00BF00BF00BF00BF7D
:103B500000BFC3D1C6F34011284605F05BFC002C22
:103B60003CD02046013800BF00BF00BF00BF00BFEF
:103B700000BF00BF00BF00BF00BF00BF00BF00BF4D
:103B800000BF00BF00BF00BF00BF00BF00BF00BF3D
:103B900000BF00BF00BF00BF00BF00BF00BF00BF2D
:103BA00000BF00BF00BF00BF00BF00BF00BF00BF1D
:103BB00000BF00BF00BF00BF00BF00BF00BF00BF0D
:103BC00000BF00BF00BF00BF00BF00BF00BF00BFFD
:103BD00000BF00BF00BF00BF00BFC3D1C6F380114C
:103BE000284605F017FC002C3CD02046013800BFC9
:103BF00000BF00BF00BF00BF00BF00BF00BF00BFCD
:103C000000BF00BF00BF00BF00BF00BF00BF00BFBC
:103C100000BF00BF00BF00BF00BF00BF00BF00BFAC
:103C200000BF00BF00BF00BF00BF00BF00BF00BF9C
:103C300000BF00BF00BF00BF00BF00BF00BF00BF8C
:103C400000BF00BF00BF00BF00BF00BF00BF00BF7C
:103C500000BF00BF00BF00BF00BF00BF00BF00BF6C
:103C600000BFC3D1C6F3C011284605F0D3FB002C1A
:103C70003CD02046013800BF00BF00BF00BF00BFDE
:103C800000BF00BF00BF00BF00BF00BF00BF00BF3C
:103C900000BF00BF00BF00BF00BF00BF00BF00BF2C
:103CA00000BF00BF00BF00BF00BF00BF00BF00BF1C
:103CB00000BF00BF00BF00BF00BF00BF00BF00BF0C
:103CC00000BF00BF00BF00BF00BF00BF00BF00BFFC
:103CD00000BF00BF00BF00BF00BF00BF00BF00BFEC
:103CE00000BF00BF00BF00BF00BFC3D101212846F5
:103CF00005F090FB002C3CD02046013800BF00BFEF
:103D000000BF00BF00BF00BF00BF00BF00BF00BFBB
:103D100000BF00BF00BF00BF00BF00BF00BF00BFAB
:103D200000BF00BF00BF00BF00BF00BF00BF00BF9B
:103D300000BF00BF00BF00BF00BF00BF00BF00BF8B
:103D400000BF00BF00BF00BF00BF00BF00BF00BF7B
:103D500000BF00BF00BF00BF00BF00BF00BF00BF6B
:103D600000BF00BF00BF00BF00BF00BF00BF00BF5B
:103D7000C3D10020F8BD00BF04207047002802DC3A
:103D80001C20FDF761BD0B68DB0701D40D20F8E7AF
:103D900000207047024B01221A64D3F84005704797
:103DA00000800040044B01221A64D3F840054FF410
:103DB0007A73B0FBF3F07047008000400048704712
:103DC000C0D000001D20704770B5054D2B5C8B42A4
:103DD00004460E4602D005F0F3FA2E5570BD00BF22
:103DE000B805002070B50024084D2646635D012B00
:103DF00008D10021204605F00DFB0021204605F0EA
:103E0000DFFA665501341D2CF0D170BDB8050020D5
:103E100070470F2070473B207047000070B5046862
:103E2000E20702D54568EB0704D40D20BDE87040D9
:103E3000FDF70ABD64101C2C2FD8184E335D012BE2
:103E400018D00121204605F0BBFA01231B2C335565
:103E500010D1134BDA6E134B202AB8BF4FF0A0439A
:103E600002F01F0203EB8203D3F8002742F44072F2
:103E7000C3F800270C4BD3F8082132B1D3F818212E
:103E8000002AFBD00022C3F81821A5F34A012046DE
:103E90008910BDE8704005F041BA70BDB80500203A
:103EA00010E300000003005000C0014008B50846C0
:103EB000FFF7B4FF002008BD13B50A4A044692E894
:103EC000030022686B46042A83E8030019464FF07A
:103ED000020003D101F094F802B010BD01F0B6F871
:103EE000FAE700BF34D0000008B50846FFF7E4FF4A
:103EF000002008BD10B5084C63792BB100210520C6
:103F000005F05EFA00236371052005F09FFA002892
:103F10000CBF0420002010BDB805002010B5084CCF
:103F2000E37A2BB100210B2005F04AFA0023E3725B
:103F30000B2005F08BFA00280CBF0420002010BDD8
:103F4000B805002010B50B4A0B4C0C480C49002357
:103F5000C2F80035A2F5C832C2F8103501226260FD
:103F600042604A60C4F80035C0F80035C1F8003539
:103F700010BD00BF00F0014000C001400010024031
:103F8000002002401C2870B504460D4625D8134E6B
:103F9000335C012B04D0012105F012FA01233355C3
:103FA0001C2C12D1FFF7CEFF0D4B1A6F0D4B202AA0
:103FB000B8BF4FF0A04302F01F0203EB8203D3F817
:103FC000002742F44072C3F80027291C204618BF7E
:103FD0000121BDE8704005F01DBA70BDB805002094
:103FE00010E30000000300500368D90702D40D203D
:103FF000FDF72ABC41680A1F514251415810FFF792
:10400000C1BF08B50846FFF7EFFF002008BD00005C
:10401000F8B5324CD4F84831ABB10023D4F8485548
:10402000C4F848312E4B186800280CDB2D4A117853
:10403000B1FA81F14909117005F0ECF92A4B1B889E
:104040002B44C4F84835254BD3F84C21002A37D0EF
:104050000021264ED3F84C45C3F84C113378244D3B
:1040600033B12B68032B03D8224AD05C05F0D2F978
:104070002B68204F01335A4202F0030203F003037E
:1040800058BF53422B600022042B194619D001332C
:10409000F81810F8010CFF2801D10122F4E702B151
:1040A0002960012105F0B6F9012333702A68124B0B
:1040B00033F8122004F10C031344084AC2F84C35BB
:1040C000F8BD4FF0FF3304F58C44044A2B605C3498
:1040D00000233370C2F84C45F2E700BF0080004077
:1040E00018000020D60500200C000020D505002077
:1040F000B40500201C0000200E000020094B0A49D6
:1041000040F2DC521A805A809A80DA80074A0023F3
:104110001370074AFF20087048708870C8701360D9
:10412000704700BF0E0000201C000020D5050020B5
:10413000B4050020024B4FF0FF321A60704700BFF9
:1041400018000020024A03480D2102F083B800BF86
:104150003CD0000043DA000038B54FF4E131284884
:1041600004F0FCFD274B012200211A61C3F804155D
:104170000321C3F808150421C3F810151A604FF085
:1041800080430221C3F818159A604FF01023D3F82A
:104190000C32DB070FD51C4BC3F80425D3F80024E1
:1041A000002AFBD04FF010226FF00101C2F80C1270
:1041B0000022C3F80425082004F0F4FF134A00236A
:1041C000FF21995401331D2BFBD1114B114D0122BD
:1041D0001A600020104A042301461468002CFCD009
:1041E0002C681160013B44EA0020F6D10B4B012200
:1041F0001A6004F00DFFBDE8384001F0D7B800BFE9
:10420000907C01200080004000E00140B8050020C3
:1042100000D0004008D5004000D1004004D000404C
:10422000F8B506460948094F0C4604F0D7FD84420C
:10423000A8BF04463546AB1B9C4205DD384604F05A
:10424000D3FD05F8010BF6E72046F8BD907C012070
:104250000146014804F087BD907C012010B5054C53
:10426000204604F08DFD20464FF4E131BDE81040BA
:1042700004F074BD907C0120C3070CD4064B1B686E
:10428000834208D8054B1B68984204D850F8043C78
:10429000002B18BF18467047E0050020DC05002001
:1042A0000B4908B50122002341F823200133642B78
:1042B000FAD1084B1A60084B084A1846002107F04B
:1042C00067F9074B40F8043F064B186008BD00BF74
:1042D000688E012008000020E405002070670100BE
:1042E000A09D0500D8050020034B044A1A60044B2A
:1042F000044A1A60FFF7D4BFE0050020E40500205F
:10430000DC050020546D0120044B1B681868C0F3C5
:104310000F10023820EAE070704700BFD805002077
:1043200000B59BB00246054901A807F08BFC01A827
:1043300002F057FA02F066FDFCE700BF9BD10000D7
:10434000C30713D4042802D812D00B48704703685F
:1043500003F00F03042B01D104307047092B09D05F
:10436000064A0748032B18BF104670470548704798
:10437000054870470548704758CC000086D10000BA
:104380008FD1000075D100005ECC00007FD100000D
:10439000064B074900201A6843F8040CC2F30F12B9
:1043A000023203EB82038B42F5D37047E80500200D
:1043B000546D01202F4B304A1868304B2DE9F041E5
:1043C0001C682F4D136803F00F01072928D81368C4
:1043D000C3F30F13023302EB8302AA42F2D329493B
:1043E000002251F82200FFF747FF41F82200013276
:1043F000642AF6D1244A1068FFF73EFF1060234A72
:10440000106810B1FFF738FF1060214B214C1E6877
:104410000021F0274FF03C08B14214DBBDE8F081E9
:10442000C3F30F1302EB83039A42D0D01968CE076F
:1044300007D4884205D28C4203D351F8041C01B141
:104440001960043BF0E707FB01F31A191B5D0BB978
:104450000131E1E71269551E08FB012204EB8202DB
:104460001832002DF4DB52F8040DFFF705FF013D73
:104470001060F6E7E0050020E8050020DC050020DC
:10448000546D0120688E012008000020546D012029
:10449000AC050020107D0120C307F0B540D4214BAE
:1044A0001C68A0423CD3204B1D68A84238D850F865
:1044B000043CABBB03680246C3F30F13012673B978
:1044C000904242F8046C2BD0116851F8043C51F82A
:1044D0002370176041F82320013B0A46EFE752F8AA
:1044E0002310CF0702EB830C18D48C4216D88D42D0
:1044F00014D351F8047C8FB90F6807F00F0EBEF18A
:10450000070F08D9CCF8007042F8043C0B680A6029
:10451000C3F30F13E1E741F8046CD0E7013BCEE7AA
:10452000F0BD00BFE0050020DC0500200D4930B5DE
:104530000D4C0B461A6853F8045CC2F30F12901C22
:1045400065B18B4214BF0A46002243F8042C01EBEC
:10455000800103EB8003A342ECD330BD12011A604B
:10456000F7E700BFE8050020546D0120144B2DE94A
:10457000F041144C1E464FF000083268C2F30F178A
:1045800012070FD07D1C9E424FEA850505D01846C4
:104590002A46314606F0E3FF03465A1904352B44F8
:1045A000C2F80080023706EB8706A642E5D3E41A7C
:1045B000A410013C044A24011C601360BDE8F08192
:1045C000E8050020546D0120D80500202DE9F041B8
:1045D0009AB0FFF7DFFB214D0746002455F8240071
:1045E0000134FFF759FF642CF8D11D4B1868FFF711
:1045F00053FF1C4B186808B1FFF74EFF1A4DDFF848
:1046000074800026D8F800309E4218DBFFF78EFF3A
:10461000FFF7D0FEFFF7AAFFFFF7BCFB134B1449CF
:104620001B681B68C3F30F13C21B023B01A807F0F2
:1046300009FB01A802F0D5F81AB0BDE8F0812B788B
:1046400013B90136F035DDE72C69013C002CF8DBAD
:1046500005EB84039869FFF71FFFF6E7688E0120DA
:1046600008000020546D0120107D0120D805002095
:1046700055D10000AC0500202DE9F8431B4C236800
:104680001B684D1CC3F30F139D4206468846174610
:10469000A1460CDBFFF79AFF23681B68C3F30F13D7
:1046A0009D4204DB0A20BDE8F843FDF7CDB808F1D0
:1046B0000202D9F800009B1A1B0140F822300023A7
:1046C00040F8043C06F00F06034646EA081694003C
:1046D00043F8046B0119083CC9F800101C44A342BC
:1046E00001D3BDE8F88343F8047BF8E7D805002040
:1046F000F8B510F0010704460E462CD1174B1B6885
:10470000834228D8164B1B68834224D9154D286054
:104710000068012200F00F00FFF7AEFF2C682F6049
:104720000546C0B12146043051F8042BC2F30F12E4
:10473000B242A8BF3246920006F006FFFFF728FEFD
:1047400044F8045CFFF736FE2268074B44F8047C0B
:10475000134023602C462046F8BD00BFE005002032
:10476000DC050020546D0120F0FF0F00011D002228
:10477000042091FBF0F1FFF77FBF38B505460846EE
:104780000C46FFF7F3FF50B1C21C2B46591B8C425D
:1047900006DC002CACBF0419041C0023237138BDB7
:1047A00013F8011B02F8011FF0E7F0B502289BB0D7
:1047B0000C4604DC1C20FDF747F81BB0F0BD086870
:1047C000C20706D4042804D9036803F00F03042B9E
:1047D00001D00E20EFE74B6813F00107F9D1042B4D
:1047E000F7D91B6803F00F03042BF2D18B68DB07AA
:1047F00001D40D20DFE7FFF7A3FD06466068FFF751
:104800009FFDA5681AAC014604F8647D6D10304622
:1048100003F0D7FD29466423224603F034FE2046E8
:1048200007F056FA01462046FFF7A7FFC5E700004C
:1048300010B50446ADF5806D10B9FFF797FF0BE09A
:1048400003F0E5FC0138062827D8DFE800F0080867
:1048500010172804230000200DF5806D10BD2046A0
:1048600003F04FFD011B2046FFF787FFF4E72046CA
:1048700003F0FBFC400040F00100EDE769464FF417
:104880008062204603F00BFD684607F021FA0146DE
:104890006846E9E704210348E6E70020CDE7042065
:1048A000DAE700BFF4D10000022838B50C4604DC7A
:1048B0001C20BDE83840FCF7C7BF0868C10706D414
:1048C000042804D9036803F00F03042B01D00E2041
:1048D000EFE76368DA07FAD4042BF8D91B6803F012
:1048E0000F03042BF3D1A368DB0701D40D20E0E70D
:1048F000FFF726FD05466068FFF722FDA468014624
:104900006410284603F05DFD214603F099FDBDE8E3
:104910003840FFF78DBF012838B50C4604DC1C2059
:10492000BDE83840FCF790BF0868C10706D40428EA
:1049300004D9036803F00F03042B01D00E20EFE726
:104940006368DA07FAD4042BF8D91B6803F00F0365
:10495000042BF3D1FFF7F4FC05466068FFF7F0FC89
:104960000146284603F02DFD03F0A9FD400040F06C
:10497000010038BD012870B505460C4604DC1C203A
:10498000BDE87040FCF760BF0868C10706D4042882
:1049900004D9036803F00F03042B01D00E20EFE7C6
:1049A0006368DA07FAD4042BF8D91B6803F00F0305
:1049B000042BF3D1FFF7C4FC06466068FFF7C0FC88
:1049C000022D014615D0A468E30712D564103046C5
:1049D00003F0F7FC054603F01AFC012812D1002C65
:1049E00002DD0135012C07D12846BDE87040FFF7F4
:1049F0001FBF4FF0FF34EAE7284603F091FC013C6B
:104A00000546EFE70228EFD1002CEDDD0135012C42
:104A1000EAD000221146284603F0ACFC03F080FCEB
:104A2000013C0546F3E7086808B5C30706D4042827
:104A300004D9036803F00F03042B04D00E20BDE853
:104A40000840FCF701BFFFF77BFC0378232B08BF6E
:104A500001301022002107F0FFF900F10053B3F1FB
:104A6000804F01D31420EAE7400040F0010008BD68
:104A700010B510F0010402D04410204610BD0428E7
:104A800012D9026802F00F02042A07D1FFF758FC7E
:104A90000A222146BDE8104007F0DEB9032A03D1FF
:104AA0000A2221460430F5E70D20FCF7CDFEE4E7AD
:104AB00008B50868FFF7DCFF07EE900AB8EEE77A62
:104AC000DFED0A7A67EE277A17EE900A06F09EF974
:104AD00004F0C4FD0022064B06F0F0F904F074FD6A
:104AE00006F09CFC400040F0010008BDD3023739BD
:104AF0000000D04004282DE9F0410C4604DC1C20C5
:104B0000BDE8F041FCF7A0BE0868FFF7B1FF07461B
:104B10006068FFF7ADFF0646A068FFF7A9FF0546EE
:104B2000E068FFF7A5FF80462069FFF7A1FFAE42CE
:104B300001D11F20E4E7BF1BA0EB08007843AD1BA9
:104B400090FBF5F04044400040F00100BDE8F081EA
:104B5000024A0348082101F07DBB00BFB4D1000028
:104B6000ACD10000002070471E20FCF76DBE1E2057
:104B7000FCF76ABE1E20FCF767BE1E20FCF764BE71
:104B80001E20FCF761BE1E20FCF75EBE1E20FCF757
:104B90005BBE1E20FCF758BE1E20FCF755BE1E2033
:104BA000FCF752BE1E20FCF74FBE1E20FCF74CBE89
:104BB0001E20FCF749BE1E20FCF746BE1E20FCF757
:104BC00043BE1E20FCF740BE1E20FCF73DBE1E204B
:104BD000FCF73ABE1E20FCF737BE1E20FCF734BEA1
:104BE0001E20FCF731BE1E20FCF72EBE1E20FCF757
:104BF0002BBE1E20FCF728BE1E20FCF725BE1E2063
:104C0000FCF722BE1E20FCF71FBE1E20FCF71CBEB8
:104C10001E20FCF719BE0000024A03481E2101F0C5
:104C200019BB00BF48D2000038D30000034B01225B
:104C30001A60034B18689040104370477C6D012048
:104C4000586D01202DE9F043EFF31084012304F0A7
:104C5000010483F31088164A164912680E68013A57
:104C60009340154A1568154A12684FF002094FF033
:104C70000E0C4FF00D0E4FF00608A3B118422A603B
:104C80000AD0774639000139FDDC326047463900E9
:104C90000139FDDC5B08F0E74F4639000139FDDCE6
:104CA00032606746F3E784F31088BDE8F08300BF05
:104CB00020000020606D0120646D01206C6D0120DA
:104CC00070B5084E084D002456F824000021FFF767
:104CD0007BF855F8240000210134FFF775F8052C06
:104CE000F2D170BDC8D400001CD800002DE9F041FD
:104CF000134E144D144F0024002156F82400FFF7E2
:104D000063F855F8248001214046FFF75DF8B8F1BB
:104D1000220F10D857F828200C4B202AB8BF4FF08C
:104D2000A04302F01F0203EB8203D3F8002742F4F2
:104D30004072C3F800270134052CDDD1BDE8F081B5
:104D4000C8D400001CD8000010E30000000300508D
:104D50002DE9F3413B4D4FF441732C68ADF804301D
:104D60000A238DF80630BCBBFFF7AAFFDFF8E4800A
:104D7000264658F8267001213846FFF725F80136F7
:104D80000021384604F046FB052EF2D100260DF135
:104D9000040816F8087001213846FFF715F80136A7
:104DA0000121384604F036FB032EF2D10021042005
:104DB000FFF70AF800213046FFF706F800210A2025
:104DC000FFF702F801232B60FEF7E4FF1E4B18608B
:104DD000204602B0BDE8F0811B4B1C68FEF7DAFFED
:104DE000844298BF001BB0F57A6F29DB022004F0E3
:104DF000DFF9042004F0EEF90446032004F0EAF998
:104E000007460A2004F0E6F90646012004F0D0F92E
:104E1000012004F0DFF9E0193044C0F532600323CB
:104E2000023090FBF3F0094B0028BCBF00221A604F
:104E3000074AA8BF186000232B6013600124C7E74E
:104E40000024C5E7746D0120806D0120586D01209C
:104E50007C6D01201CD8000008B5054B00221A60AB
:104E6000044B1B680BB103F071F9002008BD00BFB3
:104E7000786D0120F47A012010B5041E1CDA00249C
:104E80001049114B114A0B6004331360104B53F857
:104E900024301F2B81BF0F4808600F49116003F0B9
:104EA0001F024FF0010303FA02F38CBF0C310B49D0
:104EB0000B4A0B60136010BDFEF784FFA042DEDDDD
:104EC000DEE700BF646D012008050050606D012021
:104ED00010E30000080800500C08005018050050AE
:104EE0006C6D012008B50B68DA074CBF5B104FF002
:104EF000FF3301280DDD4A68042A14BF182220223E
:104F0000054918460A60FEF783FFFFF7B5FF00204A
:104F100008BD1822F4E700BF20000020002808B5D3
:104F20000CDD0B68042B084B14BF012200221A6011
:104F300006D0FFF7C5FE054B00221A60002008BD11
:104F4000FFF7D4FEFAE700BF706D0120586D012015
:104F500010B510F0010402D04410204610BD042802
:104F600012D9026802F00F02042A07D1FFF7E8F90C
:104F70000A222146BDE8104006F06EBF032A03D185
:104F80000A2221460430F5E70D20FCF75DFCE4E73A
:104F9000086810F0010370B51CD0FFF7D9FF034675
:104FA000203B5E2B27D8154C03EB83030022012105
:104FB00010462344052A1AD09E5C052410252E4253
:104FC00018BF4018013C4FEA41014FEA6505F6D190
:104FD0000132EFE70428E3D9026802F00F01042947
:104FE000DED1C2F30F13002BDAD00379D8E74000EB
:104FF00040F0010070BD0120FCE700BFDCD40000E0
:1050000038B508680D46FFF7A3FF04466868FFF748
:105010009FFF621E042A014612D8431E042B0FD89C
:10502000084803EB830313440568012202FA03F3E3
:105030002B430360044B1B6813B1204603F087F831
:10504000002038BD786D0120F47A012038B5086859
:105050000D46FFF77DFF04466868FFF779FF621E83
:10506000042A014614D8431E042B11D8094803EB27
:1050700083031344012202FA03F3026822EA0302C3
:10508000054B02601B681BB10022204603F05FF84D
:10509000002038BD786D0120F47A01202DE9F04F11
:1050A000054685B008680C46FFF752FF022D0190B7
:1050B0003CDD6068FFF74CFF0746A068FFF748FF3C
:1050C0000446231DDFF8C8A00293661E4FF00108B6
:1050D000029B9E4206F1010935D006EB8602531E63
:1050E00007F1050B3D460393AB4522D0042E19D89A
:1050F0006A1E042A16D8039B019ADAF8000059198F
:10510000224B4FF0010C18EA020E0CFA01F11B6859
:1051100011D00143CAF8001023B16246494628461F
:1051200003F015F84FEA48080135DDE7012427466A
:10513000C7E74E46CCE720EA0101CAF80010002B71
:10514000F0D07246EAE73D1D042D1BD8012C19D181
:10515000DFF83C80DFF834900026D8F8003004FAFD
:1051600005F223EA0203C8F80030D9F8003001360E
:1051700023B100223146781D02F0E9FF052E05F12A
:105180000505EAD1002005B0BDE8F08FF47A0120D2
:10519000786D01202DE9F843394B1B680C461BB98B
:1051A0004FF0FF30FFF768FE206810F001083AD199
:1051B000042838D9036803F00F03092B33D10746BD
:1051C000304D57F8044F304E641040F25969A045F5
:1051D00052DA57F8040FFFF7BBFEC0F30742C0F3E3
:1051E00007235B43524393FBF9FC92FBF9F32A68D4
:1051F000202AC1B208BFC0F305604FEA032308BFED
:1052000056F8202043EA0C4301FB01F191FBF9F130
:1052100043EA010308BF42EA03231846FFF712FDE1
:1052200008F10108D3E7FFF793FEC0F30742C0F38C
:10523000072340F259655B43524393FBF5F492FB1D
:10524000F5F3104A1268202AC1B204BF0E4AC0F317
:1052500005604FEA032308BF52F8202043EA0443C5
:1052600001FB01F191FBF5F143EA010308BF42EABA
:1052700003231846FFF7E6FC0020BDE8F88300BFD3
:105280006C6D012020000020B8D60000086808B529
:10529000C30703D5FFF75CFE054B1860054B1B6881
:1052A0001BB1034B186802F053FF002008BD00BF7C
:1052B000786D0120F47A01202DE9F843334B1C6806
:1052C000002C59D1324E326852B9324B1B683BB96F
:1052D000314B1B68002B4FD0BDE8F843FFF738BDBA
:1052E0002E4D2B6863B92C4B1B68002B40D1294AEB
:1052F000336810681146002840D10B60FFF7F6FCB8
:105300002B68274EDFF88C90264F002BCCBF03F183
:10531000FF330423002156F82300FEF755FD2A68C9
:10532000214B53F8228057F8240004EB840101EB51
:105330000803D9F80010194101F00101013404F00B
:1053400069F8052CEFD12B68012156F82300FEF7F0
:105350003BFD2B68002156F8230004F05BF82B6816
:10536000013393FBF4F404EB84041C1B2C6003E076
:10537000FFF7EEFC0028BAD1BDE8F883002BBCD1C2
:105380001360BDE8F843FFF79BBC00BF706D0120C0
:10539000786D0120686D01207C6D01205C6D01201D
:1053A000C8D400001CD80000B8D700004FF0FF3070
:1053B000FFF762BD024A03480A2100F04BBF00BF5D
:1053C000CCD7000030D800004FF0805310B51A69D8
:1053D000094B0224C3F8044522F00302884203D398
:1053E0000022C3F8042510BDD3F80044002CFBD0E4
:1053F000C3F808051044F1E700E00140002815BF9C
:105400004FF4D2214FF4B4214FF4B4204FF496203E
:10541000FFF7DABF00280CBF4FF496234FF4B423F4
:105420001868030E532B0CBF20F07F4000207047FC
:10543000064B0122C3F80425D3F80024002AFBD030
:1054400000220160C3F80425704700BF00E001405E
:10545000002821F07F4141F0A6410CBF4FF4962077
:105460004FF4B420FFF7E4BF0A4B30B50124C3F872
:105470000445002903DC0022C3F8042530BD52F89E
:10548000044BD3F80054002DFBD040F8044B0139F5
:10549000EFE700BF00E0014038B54C680234054634
:1054A0000A462146FFF7E0FF05EB840038BD000007
:1054B000124B1B68002B0BBF4FF4B4224FF4D222C7
:1054C0004FF496234FF4B42328B91A1DDB79522BDD
:1054D00008BF1046704782420DD9C378522B0AD1BB
:1054E0004368023300EB8300824204D9C378522B15
:1054F00018BF002070470020704700BF846E012055
:105500002DE9F0410020B4B0FFF7D2FF0024DFF80E
:10551000A4800546274626464DBB224D2868FFF746
:1055200079FF3B463246CDE900401F4902A806F00C
:1055300089FB02A801F055F91C4B1A682B68002B57
:105540000CBF4FF496234FF4B423D21A4FF470419A
:1055500064235343009193FBF1F302A8144906F02E
:1055600071FB02A801F03DF934B0BDE8F081696833
:105570002A6801918B1C1F44D1B2C2F307239C42BD
:10558000C2F30742009102A84146B8BF1C4606F08C
:1055900059FB02A801F025F92846FFF789FF0136DB
:1055A0000546B9E7846E01204AD90000886E0120C3
:1055B000F4D8000036D9000070B50020FFF72AFFAC
:1055C00005460120FFF726FF0C4B1E68B6FA86F44D
:1055D00085424FEA5414B8BF054620461C60FFF7C9
:1055E0000DFF074A074B002E18BF1346064A691CD9
:1055F0002046BDE870401360FFF72ABF846E01208B
:1056000004B0040004A00500886E012070B50020DD
:10561000FFF700FF02460120FFF7FCFE1F4E204C63
:10562000054672B968B94FF4D2214FF49620FFF7BE
:10563000CBFE01212846FFF70BFF1A4B3560236094
:1056400029E0AA4208DD00233360164B23604FF4A3
:10565000B4212368002017E001233360124B23603C
:105660004FF4D221F5E7120E522A08D000B1236080
:105670000E4801F0B6F8BDE87040FFF79DBF5A68CC
:10568000023203EB820301208B4205D21A68551CBB
:10569000E9D10028D3D170BD2160FCE7846E0120E0
:1056A000886E012004B0040004A005000FD900009A
:1056B00010B50020FFF7FCFE014608B9084610BDF2
:1056C0008478FFF7F5FEDA2C08BF0146F5E7000005
:1056D00038B500214FF4FF621B4805F059FFFFF772
:1056E000E7FF1949002490B91848174C0123F0210D
:1056F00001FB030212F8F05C2DB112F8EF5C54F8D4
:10570000355042F8E85C01330B2BF1D138BD03680A
:10571000C3F307420A2A0BD1C3F30722FF2A04D09E
:1057200001EBC20541F832002B71FFF7C1FEDAE749
:10573000132AFAD1C3F30723FF2B1EBF01EBC302C9
:1057400041F833401471F0E770860120107D01208C
:1057500000B59BB0FFF75AFFFFF7BAFF00230B49D4
:105760001A4651F8330000B101320133FF2BF8D152
:10577000074901A806F066FA01A801F032F80548C9
:1057800001F02FF81BB05DF804FB00BF708601200C
:105790007FD9000093D900002DE9F04F4FF48072BB
:1057A0009FB0604C6048002105F0F2FE4FF480721B
:1057B00000215E4805F0ECFED4F80090B9FA89F8B3
:1057C0004FEA58184046FFF719FEA246584B594C6D
:1057D0000020B9F1000F08BF1C46FFF769FF06461D
:1057E00048BB4846FFF716FE534D411C4046FFF7A5
:1057F0002FFECAF800802C60FFF76AFFFEF72EFD2F
:10580000DAF800302A68002B0CBF4FF496234FF4CF
:10581000B423D21A4FF4704164235343009193FB95
:10582000F1F305A8454906F00DFA05A800F0D9FFE7
:105830001FB0BDE8F08F3568C5F30743A3F10A0236
:10584000092AC5F3072546D8374B595D91BB10226D
:105850003B48DFF8ECB005F09BFE37463A68C2F3F0
:1058600007218D4209D1C2F307410B2926D0132904
:105870002BD00A2901D1CBF800703846FFF718FE6B
:1058800007460028EAD12E4F396881B12046FFF73C
:1058900003FE0123044657F8231029B12046039341
:1058A000FFF7FAFD039B04460133042BF3D11E4A94
:1058B000012353553046FFF7FBFD90E7D2B2022A91
:1058C000DBDC0BEB82025760D7E710220021584641
:1058D00005F05EFED1E7A3F11502082AEAD8134AC3
:1058E000525D002AE6D1152B0CBF3146002130460F
:1058F0000368C3F30742152A0ED01D2A08BF0021F2
:10590000FFF7D6FD0028F3D119B12046FFF7C4FDFB
:1059100004460123054ACCE7C3F307239D4208BF91
:105920000146EDE7846E0120846D01208C6E01201C
:1059300004A0050004B00400886E0120D9D800003E
:10594000F88F0120FFF728BF2DE9F84FDFF8A8B046
:10595000274F03339246042293FBF2F6DBF8003024
:10596000B41C002B3B684FEA84040CBF4FF4B422F4
:105970004FF4D22223449A4281460D46B84614D2AF
:10598000FFF70AFFDBF80030002B3B680CBF4FF439
:10599000B4224FF4D22223449A4206D2154800F092
:1059A00020FF00273846BDE8F88F2D025FFA8AF104
:1059B00041F0A441ADB2D8F800700D434FEA09415F
:1059C00001F47F0129433846FFF732FD07F108054E
:1059D0003146381DC8F80050FFF72AFD1EB10A9A5B
:1059E0002846FFF741FD083C2544C8F80050D9E798
:1059F000886E0120B3D80000846E01207047704784
:105A00000A4B0022C3F8002101225A60D3F800217A
:105A1000002AFBD00022C3F80C2101229A60044B1B
:105A20000222C3F880211A60704700BF00100040B6
:105A300000E100E0074B0222C3F88020064B002261
:105A4000C3F8102101221A61D3F81021002AFBD0DB
:105A5000704700BF00E100E00010004008B50449B5
:105A60000A780AB1FFF7E6FF0020087008BD00BF02
:105A70008D6F0120024B1868400040F00100704714
:105A800010700120024B1868400040F00100704780
:105A9000240000201FB5064B06491A6801A806F02D
:105AA000D1F8082101A8FEF768FE05B05DF804FBF7
:105AB0001470012024DA00001FB54FF0805306490E
:105AC0001A6E01A806F0BEF8082101A8FEF755FEDF
:105AD00005B05DF804FB00BF24DA000010B5054CEA
:105AE000204606F0F5F801462046BDE81040FEF7D6
:105AF00044BE00BF19700120104B1B685A1C10B522
:105B000014D0CBB1012B13D0022B13D0042B13D004
:105B10000B4C0C4A052B08BF1446204606F0D8F85B
:105B200001462046BDE81040FEF727BE064CF4E7CC
:105B3000044CF2E7054CF0E7054CEEE728000020A6
:105B40002EDA000034DA000029DA00001BD0000051
:105B500014D0000070B504460D461646FEF722F933
:105B60004FF0805301221B6E6270E270020AA27134
:105B7000020CE2711A0A002160716372000EA272B7
:105B80001A0C1B0E2670A17025712072E27223730D
:105B900070BD000010B521480278002A3DD14FF0B9
:105BA0008043C3F8002101221A60D3F80021002AA3
:105BB000FBD01B4B1B4C00220721C3F80C25C3F85C
:105BC00008151949C3F81025C3F81C15C3F8242576
:105BD0000121C3F82C250822C3F83015C3F8142579
:105BE000C3F818450224C3F834454FF6FF74C3F8D0
:105BF0003C450E4CC3F838451824C3F85445C3F847
:105C00000423D3F8002242F01002C3F80022084A0D
:105C1000C3F80425FFF7F4FE017010BD8D6F01205D
:105C20000010004020000402746962752110010018
:105C30008E6F012013B50A4A0A4B07280446CDE9A6
:105C400000230BD8084B1B780BB9FFF7A3FF02AB5F
:105C50001C44064B14F9082CC3F80C2502B010BDE7
:105C6000E2ECF0F4F8FC00048D6F0120001000401D
:105C7000F8B5104B1B7804460BB9FFF78BFF0E4E9F
:105C80003378ABB10D4A1278D21A02F003010C4AF4
:105C900002EB411202F1200710685168254603C546
:105CA0000832BA422C46F7D1013B33700120F8BDCF
:105CB0001846FCE78D6F0120187001208C6F0120C1
:105CC0008E6F012030B5002889B02ADD0D6815F0EF
:105CD000010426D1042D26D92B6803F00F03092BCC
:105CE00021D16B683F2B1EDD6846FFF7C1FFB0B1C5
:105CF0009DF800200435A242A8BF1DF8043004F12D
:105D00000104A6BF5B0043F001030123202C45F8EA
:105D1000043FF0D1054BDDF809201A60042009B0DA
:105D200030BD0020FBE72046F9E700BF14700120DA
:105D300030B5384B1B788BB00BB9FFF72BFF02A89F
:105D4000FFF796FF10B900200BB030BD9DF808306A
:105D50000B2BF8D99DF80930012BF4D19DF80B30AD
:105D6000012BF0D12C4D2D4C2D4ADDF811100023C4
:105D70002B6023709DF80C3013602A4A116023B900
:105D8000DDF815302B6000230FE0012B11D1DDF879
:105D900015309DF819202B600DF11A010E23934246
:105DA000A8BF134600229A4230D10022E2540420B8
:105DB000CAE7022B05D19DF8152012230DF116011B
:105DC000EDE7042B0DD10AAA6B4652F8130D51686A
:105DD00003C3DDE9000103F069FB05F01FFB286048
:105DE000D1E7052BCFD10AAA6B4652F8130D5168A3
:105DF00003C3DDE9000103F059FB05F00FFB9DF83B
:105E00001D2028600A230DF11E01C8E7885CA054FC
:105E10000132C8E78D6F0120107001201970012038
:105E2000280000201470012010B5154B1B78044683
:105E30000BB9FFF7AFFEFFF7FDFD124B0022C3F8D1
:105E40000445C3F8002101221A60D3F80021002A7A
:105E5000FBD00022C3F80C2101229A60094AD2F833
:105E60000C31002BFBD0084B1978084B03EB411386
:105E7000C2F80435FFF7DEFDBDE81040FFF7C0BDF6
:105E80008D6F0120001000408C6F01208E6F01206B
:105E900000B5002889B01DDD0B6813F0010219D18F
:105EA000042B17D9196801F00F01092912D159687B
:105EB0003F290FDD043353F8040F10F0010118BF20
:105EC000C0F347010DF802100132202AF3D16846D1
:105ED000FFF7AAFF002009B05DF804FB002810B509
:105EE00011DD0C68E3070ED56410532C0BD8074B5B
:105EF0001B780BB9FFF74EFEFFF79CFD044BC3F870
:105F00000845FFF77DFD002010BD00BF8D6F01200B
:105F100000100040002810B50DDD0C68E3070AD51D
:105F20006410FF2C07D8054B1B780BB9FFF732FE26
:105F3000034BC3F82445002010BD00BF8D6F012026
:105F400000100040002808B505DD0868C30702D529
:105F50004010FFF76FFE002008BD70B5002888B024
:105F600020DD086810F001041CD104281AD9036848
:105F700003F00F03042B15D1FEF7E2F9064605F0F6
:105F8000A7FE122828BF1220054600F10D020221AB
:105F90006846FFF7DFFD8DF80D50A54205DC684629
:105FA000FFF742FF002008B070BD0DEB0403325D27
:105FB0009A730134F1E72DE9F041012888B00D46CC
:105FC00030DD086810F001042CD104282AD90368B8
:105FD00003F00F03042B25D14B68DB0722D5FEF716
:105FE000AFF9804605F074FE6D680E2828BF0E20BC
:105FF0006E10074600F1110201216846FFF7AAFD65
:106000006B128DF80D606D14360E8DF80E308DF814
:106010000F508DF810608DF81170A74206DC6846AD
:10602000FFF702FF002008B0BDE8F0810DEB04038C
:1060300018F804209A740134EFE730B5002889B0CD
:1060400016DD0C68E30713D56510684610220021A1
:10605000FFF780FD63128DF80D5064142D0E684615
:106060008DF80E308DF80F408DF81050FFF7DCFEE4
:10607000002009B030BD0000174BD3F8002122B139
:106080000022C3F8002101229A60D3F80C2102B348
:106090000021C3F80C11D3F80024012A0F4A19D1AA
:1060A000D3F848355B4213600D4A1378032B9CBF2D
:1060B000013313700B4A1378013303F00303137099
:1060C000094A02EB4313044AC2F80435024B012289
:1060D0009A6070471160F9E700100040240000202A
:1060E000187001208C6F01208E6F012008B50A4BBB
:1060F0001B787BB1FFF79EFC08490723C1F80835E0
:10610000FFF77EFC0023C1F824350620BDE80840D7
:10611000FFF790BD08BD00BF8D6F0120001000404B
:10612000024A0348102100F095B800BFA4D900002E
:106130009BD90000044A05491368C8540133C3F3CE
:1061400009031360704700BF4C7401204C7001209C
:1061500070B51249124A0B68834202DC00230B60BF
:1061600018E0845CA4F1FA06012E00F1010506D8BE
:10617000AB4210DDAC5C14B1283C9F2C01D8284602
:10618000EAE70446151A165D2E550134A342FADCDF
:10619000181A086070BD1470FAE700BF5878012023
:1061A0005874012008B5FDF7F5FD074B1A688242C7
:1061B00084BF00221A601B68C01A44F6206398420C
:1061C00094BF0020012008BD4470012010B5FFF7E6
:1061D0006FFA044608B9204610BD83781D2B08BF0E
:1061E0000446FFF765F9F5E7F8B50C4C0C4E0D4F7A
:1061F000002523683268934203D0F85CFEF728F844
:1062000028B91DB1FDF7CEFD074B1860F8BD236816
:106210000133C3F3090323600125EAE75074012029
:106220004C7401204C7001204870012070B5074E5D
:10623000074D044633682A689B1ADB43C3F30903FE
:10624000A34200DB70BDFFF7CFFFF3E74C740120E2
:1062500050740120F0B5074D2B680B2B08DC064F5E
:106260000C245C433E19C6E90112013338512B60FE
:10627000F0BD00BF54740120089001202DE9F04FBB
:10628000B3B0044605F024FD012803D8002033B044
:10629000BDE8F08F23785B2BF8D101382518235CFB
:1062A0005D2BF3D101343A21204605F0FAFC064675
:1062B0000028EBD0071B002FE8DD21463A46684650
:1062C00005F020FD32AB711C00241F446D1AA5425D
:1062D00007F8C84CDADD2A4619A805F013FD32ABE1
:1062E0001D44134B134ED3F8009005F8644C4FF047
:1062F0000C0AA145CADD0AFB04F36946985903EB71
:10630000060805F0DBFC054618B9D8E901874545C4
:1063100001DB0134EDE719A957F8350007EBC50B90
:1063200005F0CCFC10B9DBF80400B0E70135EEE76E
:10633000547401200890012008B5FBF7BFF8FFF75F
:1063400039F8FBF7E1F8FDF7FDFEFEF701FCFEF77B
:1063500063FCFFF7E5FE01F08BF901F0CFFE01F0E1
:10636000F9FEBDE8084002F02FB9000008B54FF46F
:1063700016620021034805F00BF9034B00221A6056
:1063800008BD00BF107D0120AC050020174B53F85D
:106390003000836803F07F031C2B70B50D46144654
:1063A00001D0002070BDC36803F07F02042AF8D139
:1063B000026902F07F02192AF3D11B0A00EB830065
:1063C0001030FDF7BDFF0378064633B105F080FCC1
:1063D000A042E6D10023A34201DB0120E2E7F15C09
:1063E000EA5C9142DDD10133F5E700BF7086012000
:1063F00008B5FDF7D7FC074B1A68824284BF00221C
:106400001A601B68C01AB0F5FA6F2CBF002001207B
:1064100008BD00BF48700120064B074A1B68126880
:106420009B1ADB43C3F309038342D4BF002001203E
:10643000704700BF4C74012050740120F8B5074626
:106440000E4614461D4673B90320FFF7E5FF10B34F
:10645000FA20FFF76FFEF8B2FFF76CFEF0B2BDE86E
:10646000F840FFF767BE501DFFF7D6FF98B1FB203D
:10647000FFF760FEF8B2FFF75DFEF0B2FFF75AFEDD
:10648000E0B2FFF757FEC4F30720FFF753FE2E4696
:10649000731B9C4200DCF8BD16F8010BFFF74AFEA7
:1064A000F6E70000F8B50C4E0C4D0024F0273368D9
:1064B000A34203DCBDE8F840FFF758BF07FB04F335
:1064C00059195B5D2BB100231A4649781120FFF75B
:1064D000B5FF0134EBE700BFAC050020107D0120C3
:1064E000F8B50E4C0E4E07460025BC4205F10105DD
:1064F00011D0237853B100231A4661781120FFF799
:106500009DFFF0220021204605F042F80A2D04F1FB
:10651000F004EAD1F8BD3560F8E700BF107D012036
:10652000AC0500202DE9F04F12F00106ADF54F7DCE
:1065300082468B4617D001238DF8143042FA03F3BC
:1065400054128DF8153052141B0E8DF817208DF84B
:1065500018308DF8164005AB0522FFF76FFF0DF5DB
:106560004F7DBDE8F08F042A2CD9116801F00F038C
:10657000042B38D105AD022310462B70FDF7E0FE49
:10658000044605F0A5FBB0F5487F034604F1FF3152
:10659000A8BF4FF448739E4206F101020DD1B0F539
:1065A000487F06D96D4B19889B78ADF832138DF86A
:1065B00034332B4659465046CFE7164611F8012F83
:1065C000AA55E8E740F0C680A2F1040CDCF1000215
:1065D0004FF0030342EB0C028DF814308DF81520B8
:1065E00005AB0222E6E7092B40F091801546042313
:1065F0008DF8143055F8043F4FEA6308B8F1200FC6
:106600008DF815804FEA6323A8BF4FF020088DF85E
:1066100016308DF8178006AC03220521B04502DC48
:1066200005ABE21AC6E755F8040F10F0010706D1D2
:10663000042847D9036803F00F03022B0DD14FF054
:10664000010323704310637047121B0E4014A770A0
:10665000E070237105340136E0E7042B30D1234686
:106660004FF0020C03F802CBCDE901210093039314
:10667000FDF766FE814605F02BFB0C28DDE90121C4
:106680000AD8009B6070874201D1DC19E3E719F852
:106690000740DC550137F6E723460C2003F8010FCD
:1066A00009F1FF3009F1080910F8017F03F8017FB3
:1066B0004845F9D12E23E372237363730E34CAE77E
:1066C000012B08D12346071F03F8022B784278419B
:1066D00060701C46BFE7092B09D10423237043686F
:1066E000581060705B12A370E7700434B3E7032B9B
:1066F0000AD121700368C3F30F10C3F34173C3EBD6
:10670000800363701B12EEE727700134A3E7032BAD
:106710007FF425AF05238DF81430C1F30F13C1F3B7
:106720004171C1EB830164294FEA21238DF81510D3
:10673000A8BF64218DF816308DF8171003328E42F1
:1067400005AB01DB0A1D35E7334412F8010F187160
:106750000136F4E7002A7FF402AF35E768CC000089
:106760000F4970B5F022002402FB04135D788542C6
:1067700003D001340A2CF7D170BDF0221846002155
:1067800004F006FF074A1368013BA34200D11460DE
:10679000002329461A461120BDE87040FFF74EBE7F
:1067A000107D0120AC05002030B5B3B032AC02231F
:1067B000054604F8C83D05F08BFAC72828BFC72056
:1067C000691E0023984207DC421C2346FE21142048
:1067D000FFF734FE33B030BD013311F8012FE2541E
:1067E000F0E770B5B2B00446FFF702FEC0B132ADBB
:1067F0000223204605F8C83D05F06AFAC72828BFDD
:10680000C7200646013C0023B3420BDB06F13200F1
:10681000FFF70CFD2B46721CFF211420FFF70EFE24
:1068200032B070BD013314F8012FEA54ECE70000D8
:106830002DE9F04F0128B9B08146884603DC1B20C2
:10684000FBF702F857E00868C20729D4042827D9C3
:10685000036803F00F03042B22D1FDF771FD0546F9
:10686000D8F80400C3071DD404281BD9036803F01B
:106870000F03042B16D1FDF763FD0646204B1B6862
:1068800003930027039BBB420EDC00962B461D4A58
:10689000C82106A805F0A2F906A8FFF7A2FFCEE7D7
:1068A000194DDDE7184EE9E70C237B43174A2946CB
:1068B000985803EB020B05F001FA044618B9DBE91E
:1068C000013A9C4201DB0137DCE70AEBC4023146A6
:1068D0005AF834000593049205F0F0F9DDE9042339
:1068E000834658B9536808F10801A9F10200984796
:1068F000074BC3F800B039B0BDE8F08F0134E0E7D2
:106900005474012005DB0000ABD100000890012089
:10691000546D01202DE9F0411F4F204AD7F8008027
:1069200005460023F02098450EDC0024F02000FBF3
:1069300004F15318565C8EB101340A2CF7D1184873
:10694000BDE8F041FFF74DBF00FB03F15418647838
:10695000AC4201D1515CE9B90133E4E7F0223146A0
:10696000184604F015FE0F49457051F83510857032
:106970000222A0450270C0E90212C0E9046601DCEF
:1069800001343C60002329461A461020BDE8F0413E
:10699000FFF754BDBDE8F081AC050020107D01205B
:1069A0004DDF00007086012070B5FFF77BFD094EBA
:1069B000FF246FF0070505FB046393F8FC37043BE5
:1069C000012B03D8E043C0B2FFF7A4FF013CF2D192
:1069D00070BD00BF708601202DE9F04106460F46CC
:1069E000FDF7CBFE0D4BDFF838801860002408EB74
:1069F000C4031B79062B01D0032B09D1E5B23A461B
:106A000031462846FFF7C2FC10B12846FFF782FF47
:106A10000134FF2CEBD1BDE8F08100BF080000205D
:106A200070860120F8B5094F0546FF246FF0070670
:106A300006FB047393F8FC37AB4203D1E043C0B2CA
:106A4000FFF768FF013CF3D1F8BD00BF708601205D
:106A50002DE9F84FFDF79EF9584B1A68824284BF22
:106A600000221A601A6842F20F71821A8A420BD908
:106A70005349186000235A181279073A022A0FD98D
:106A80000833B3F5FF6FF6D1BDE8F88F0720FFF7A5
:106A9000C9FF8AF800802EE00820FFF7C3FF3FE01F
:106AA000FDF780F9002814BF044601240020FDF7FB
:106AB00021FA81460020FDF731FA424D424E074649
:106AC000B9F1000F17D02B68002B70D133682C6000
:106AD000002B6FD0DFF8F8B0DFF8F0A09BF80030A3
:106AE0004FF00108002BD1D10920FFF79BFF8AF856
:106AF00000808BF80080AFB133689BB92B6834609D
:106B00001BB3DFF8C8B0DFF8C8A09BF800304FF027
:106B10000108002BC0D10920FFF784FF8BF800800B
:106B20008AF800802B6883B1284A1178904661B9B1
:106B30009C4238BF2C602B68E31A312B05D9072003
:106B4000FFF770FF012388F80030326882B1204BD4
:106B50001978984661B9A24288BF34603368E41A54
:106B6000312C05D90820FFF75DFF012388F800309C
:106B70002B685BB1B9F1000F08D1144C227812B91F
:106B80000720FFF74FFF00232B6023703368002B93
:106B90003FF47AAF002F7FF477AF0D4C227812B913
:106BA0000820FFF73FFF0023336023706CE7002FBE
:106BB000A2D1B9E7002FA1D1B4E700BF40700120F6
:106BC000708601203070012038700120347001205F
:106BD0003C70012013B50446FFF764FCFEF70FFF7D
:106BE00000230093134B1B6813B96846FDF764F943
:106BF00002A9042341F8043D0120FEF78FF900218A
:106C00000846FEF729F9FEF757FBFFF76FFAFDF785
:106C100099F9FDF773FAFDF78DFAFEF7C7FBFDF75B
:106C2000E1F824B1FDF73CFB0348FFF7DAFD02B0C1
:106C300010BD00BFF47A01203EDF000000230146B2
:106C40001A461120FFF7FABB07B513128DF8012081
:106C50008DF802301314120E8DF800108DF80330E9
:106C60008DF8042001466B4605221320FFF7E6FB52
:106C700003B05DF804FB0A4601461220FFF752BC40
:106C800070B505460C46FFF7B3FB58B104F132006E
:106C9000FFF7CCFA2B46224600211B20BDE87040AE
:106CA000FFF7CCBB70BD10B4144603460A4614204F
:106CB00021465DF8044BFFF7C1BB000030B5084C1E
:106CC00001444FF0FF33884201D3D84330BD10F860
:106CD000015BDAB26A4054F8222082EA1323F2E719
:106CE00020DB0000FE2837B5044614D80B4B53F8C0
:106CF000300080B1416808308900FFF7DFFF02AD46
:106D000045F8040D0920FFF791FA2B46042221468D
:106D10001720FFF793FB03B030BD00BF7086012042
:106D2000254AF8B500231846174652F8331001B12A
:106D300001300133FF2BF8D100EB80040A20FFF76C
:106D400075FAFB20FFF7F6F92720FFF7F3F900208B
:106D5000FFF7F0F9E0B2FFF7EDF9C4F30720FFF712
:106D6000E9F9164B00241E68FA2396FBF3F657F850
:106D70003400E0B1416808308900FFF79FFF054605
:106D80000520FFF753FAE0B2FFF7D4F9E8B2FFF7B6
:106D9000D1F9C5F30720FFF7CDF9C5F30740FFF799
:106DA000C9F9280EFFF7C6F9304602F04FF9013451
:106DB000FF2CDCD1F8BD00BF70860120040000204C
:106DC000F8B50746FFF702FA4FF0FF3504460CB955
:106DD0002846F8BD2668C6F30743152B0CD104F1ED
:106DE0000801384604F06AFF08B9C6F307252046B3
:106DF000FEF75EFB0446EAE71D2B08BF4FF0FF35A8
:106E0000F5E700002DE9F04FAB4CDFF8CC829DB0E8
:106E1000FFF7EAF92068C0F580614044FDF700FA09
:106E2000236818442060464688B1FCF7B3FFA34BA3
:106E3000186098F80030FA2B40F050812368022B3C
:106E400008DCFFF7AFF910B10120FFF781F91DB0A1
:106E5000BDE8F08F98F8010098F80240831E242BBB
:106E600000F22081DFE813F0250039003D004100E9
:106E700044004D001E0157008C0096009D00B30099
:106E8000F4000B011E011E011E011E011E011E0148
:106E90001E011E011E011E0119011E011E011E01FF
:106EA0001E011E011E011E011E011E011E011E01EA
:106EB0009A00FF2C0FD02046FFF752FC804A002397
:106EC00042F8343002EBC4022146137113200093C0
:106ED0001A46FEF739FD0320B7E72046FFF71AFDF3
:106EE000F9E72046FFF73CFCF5E7FFF75DFDF2E729
:106EF000FFF7D8FA0020FFF76DFE7248FFF771FC2C
:106F0000E9E7632CE7D8704B214653F8242015207D
:106F1000FFF708FBDFE7FFF759F96FF007080446B2
:106F2000002CD8D02768C7F30743152B04D0204680
:106F3000FEF7BEFA0446F3E704F10806304604F013
:106F4000C7FE05460530FFF771F9FB20FFF7F2F8A1
:106F50001D20FFF7EFF8C7F30720FFF7EBF8E8B2C3
:106F6000FFF7E8F8C5F30720FFF7E4F8A8EB0407FC
:106F7000F3199D42DBDD16F8010BFFF7DBF8F7E7AD
:106F8000002300931A4619461D20FEF7DDFCFDF78D
:106F900087F9A0E72046FFF7A5FE9CE7FFF7C0FEB4
:106FA00099E7FCF70BFF494A00906421484B03A87E
:106FB00004F014FE022303A88DF80C3004F088FEC0
:106FC00003AB024600211620FFF738FA83E7414B56
:106FD000DFF8EC801F680025FA2397FBF3F758F8D9
:106FE000354008EBC50354B3D4F8049093F804B0CB
:106FF0004FEA8906B01DFFF719F9FB20FFF79AF851
:10700000012006F1010AFFF795F8E8B2FFF792F8C0
:107010005FFA8AF0FFF78EF8CAF30720FFF78AF8C5
:107020005846FFF787F808342644A6420BD8FFF7E6
:10703000DBF809FB07F002F009F8FFF7D5F8013596
:10704000FF2DCCD147E714F8010BFFF773F8ECE7FD
:107050000024FFF727FA2346224621460094DA202F
:10706000FEF772FC21464FF4FF62154804F090FAD7
:10707000FDF716F921462046FDF7EEFE2BE7012C21
:1070800002D1FEF73DFA26E7022C02D1FEF75AFCA8
:1070900021E70120FFF79EFD1DE700231A46214648
:1070A0001A2091E7A0F1C803052B3FF614AF002288
:1070B0001146FAF733FA0EE75878012044700120A0
:1070C0007086012020DF0000688E012037DF00007D
:1070D00032DF00000400002058740120FB2B7FF4F5
:1070E000B3AE2268042A7FF7ACAEB8F8037040F262
:1070F000F6339F423FF7A8AE3B1D9A427FF7A1AE01
:1071000018F80330FE2B7FF49FAE98F8010098F832
:1071100002401B2807F1FF356BD01CD807284FD041
:10712000082826D001281BD1FF2C12D02046FFF7BB
:1071300017FB98F80550534B00932146BB1E2A4677
:107140000A20FEF701FC504B43F8340003EBC40463
:107150002571781D79E61D285FD050D31E2874D084
:10716000A0F1C803052BF4D8484A2946FAF7D6F906
:10717000EFE7632CEDD898F80530022B0CD0032BE9
:1071800014D0012BE5D1D8F80630414A5B0043F01A
:10719000010342F82430DCE7002DDADDB91E39485E
:1071A000FDF7EBFA3A4B43F82400D2E798F80630A3
:1071B000002B374B0CBF0022042243F82420C8E7E1
:1071C000632DC6DC2A46314903A804F0BDF91CAB87
:1071D0001D4403A8002305F8643CFFF7F1FD0028D7
:1071E000B7DB2B4B214653F820201520FFF79AF9E7
:1071F000AFE7294608F10500FFF7EEFBA9E7FF2CF2
:10720000A7D098F80520022AA3D81E4B0093214648
:10721000BB1E0B20FEF798FB9BE7632DA8BF6325E1
:10722000002303A99D420BDC1CAA25EAE573134445
:10723000002203F8642C152000916B1C2146E9E71D
:10724000F2185279CA540133ECE7022C13D0032C04
:1072500014D0012C7FF47DAF002D7FF77AAF98F822
:1072600005301BB1322BA8BF32231C4664235C437C
:10727000084B1C606DE7FEF7C1FB6AE7FEF7BFFB3A
:1072800067E700BF5E740120708601205D740120F5
:10729000688E012004000020084B01221A60084A71
:1072A0001368002BFCD0074B1868042390FBF3F005
:1072B0000638400040F00100704700BF00C00040A9
:1072C00000C1004008C500400120704710B5064CC1
:1072D000204601F08FFA0549204601F0F1FA044BEF
:1072E00001221A6010BD00BF187B0120801A060021
:1072F0005C78012010B5064C204601F07BFA054968
:10730000204601F0DDFA044B01221A6010BD00BFD7
:10731000D47B0120801A0600607801201FB500216F
:107320000E20FCF751FD01210F20FCF74DFD01213E
:107330000D20FCF749FD1D4801F0B4F91C4B1D4917
:107340001B681D4A8B4212780FD84FF000730193CF
:10735000002303938DF8082004AB13E90E001348B3
:1073600005B05DF804EB01F0B3B914498B4202D8C3
:107370004FF08063EBE712498B4202D84FF0006375
:10738000E5E710498B4202D84FF08053DFE70E4902
:107390008B4202D84FF00053D9E70C498B4294BF7F
:1073A0004FF080434FF00043D1E700BFF87A01204F
:1073B0003000002048E801002C00002090D003009D
:1073C00020A1070040420F0080841E0000093D00FC
:1073D000002814DD0B68DA0711D50D4A5B1001286F
:1073E00013600C4A09D04B68D90706D55B10022BF5
:1073F00009D0032B09D0012B03D0022313600020F6
:1074000070470023FAE70323F8E70123F6E700BFFC
:10741000300000202C000020002810B50EDD0C6884
:10742000E3070BD56410012C08DD054B1B680BB975
:10743000FFF74CFF2146034801F042FA002010BD3F
:107440005C780120187B012008682DE9F843C30708
:1074500004D40D20BDE8F843FAF7F6B94010FCF764
:10746000D7FC051E12DBFCF7ADFCA8420EDB0221A7
:107470002846FCF7A9FC4FF4FA620121284601F0E6
:107480001DFE28B901462846FCF79EFC002036E088
:10749000DFF8748000244FF00109002707264FF41D
:1074A0007A720121284601F009FE0028EED0282832
:1074B000C4BF09FA06F31F4316F1FF36EFD204F8F2
:1074C00008700134052CE8D100212846FCF77CFC2B
:1074D000012206210920FDF7CFF80028D6D0034667
:1074E0000B2243F8042F074900F1180411F8012F6B
:1074F000520042F0010243F8042FA342F6D1BDE846
:10750000F88300BF63780120647801200028F8B573
:1075100021DD0C6814F001061DD1042C1BD9236851
:1075200003F00F02032A16D1C3F30F15C3F34173FF
:10753000C3EB8505FFF7F2FE084F0334B54207DDC4
:1075400014F8011F384601F0D0F801362070F5E735
:10755000024801F0C9F80020F8BD00BFF87A012008
:1075600010B50468E30704D40D20BDE81040FAF715
:107570006BB96410FF2C01D91720F6E7FFF7CEFE98
:10758000E1B2044801F0B1F8024801F0ADF8002082
:1075900010BD00BFF87A012038B5074DFFF7BEFED9
:1075A0000021284601F0A1F80446284601F09CF885
:1075B000600040F0010038BDF87A0120274A82B00F
:1075C00001210023ADF80630C2F8F015C2F800150D
:1075D00019461A0102F1804202F5E0420133082BFC
:1075E000C2F81415C2F81015F3D11C4B4FF4E06229
:1075F000C3F818250422C3F81425C3F810250DF18B
:107600000602C3F82C260122C3F830261A60D3F8EC
:107610000021002AFBD00022C3F8002101225A6079
:107620000E4B1A46D3F804110029FBD00021C3F8F1
:10763000041101219960D2F81431002BFBD00020F5
:10764000C2F81401C2F80005BDF806301BB283422F
:10765000C8BFA3F50B70400002B070470070004037
:1076600008B5FFF7ABFF400040F0010008BD000087
:10767000024A03480F21FEF7EDBD00BF64DF0000A2
:10768000DCDF00000C4B1B6870B506460D46144647
:107690000BB9FFF71BFEF1B2084801F08FF9E9B210
:1076A000064801F06FF8E1B2044801F06BF80348B6
:1076B000BDE8704001F0EDB95C780120187B012035
:1076C00008B50368D90705D54168CA0702D582689D
:1076D000D00704D40D20BDE80840FAF7B5B858101B
:1076E000802801D91520F6E74910FF2901D9162075
:1076F000F1E75210FF2A01D91720ECE7FFF7C2FF8C
:10770000002008BD0C4B1B6870B506460D4614469C
:107710000BB9FFF7EFFDF1B2084801F04FF9E9B2FC
:10772000064801F02FF8E1B2044801F02BF80348B5
:10773000BDE8704001F0ADB960780120D47B012034
:1077400001282DE9F0415EDD0D68EA075BD52F4B7E
:107750004C681B686D100BB9FFF7B8FDE9B22C48F7
:1077600001F02CF914F0010613D06410FF2C02D99B
:107770001720FAF769F8E1B2254801F003F8244828
:1077800001F087F918B12320FAF75EF80020BDE870
:10779000F081042CF3D9236803F00F02092A1AD1CF
:1077A00054F8047FDFF868807F10B742E7DD54F8B3
:1077B000045FEB070BD56D10FF2D02D91720FAF7E8
:1077C00043F8E9B2404600F0DDFF0136EDE717204F
:1077D000FAF73AF8F9E7032AD1D1261DC4F1FF24BC
:1077E000C3F30F1504F57F04C3F34173084FC3EBD4
:1077F0008505FC343319AB42C1DA16F8011B384653
:1078000000F0C0FFF6E70120C1E700BF5C7801206F
:10781000187B012038B5134B1B6804460D460BB985
:10782000FFF754FDE4B221460F4801F0C7F8E9B272
:107830000D4800F0A7FF00210B4801F0C9F808B17E
:10784000404238BD01222146074801F0B4F80648FD
:1078500000F08FFF0028F4D00348BDE8384000F066
:107860008BBF00BF5C780120187B012008B503683E
:10787000D90702D54168CA0704D40D20BDE80840E5
:10788000F9F7E2BF5810802801D91520F6E7491012
:10789000FF2901D91620F1E7FFF7BCFF400040F0B7
:1078A000010008BD38B5124B1B6804460D460BB9E4
:1078B000FFF720FDE4B221460E4801F07FF8E9B25F
:1078C0000C4800F05FFF0B4801F0E3F808B14042BC
:1078D00038BD01222146074801F06DF8054800F047
:1078E00048FF0028F4D00348BDE8384000F044BF0A
:1078F00060780120D47B012038B50D211D20FFF7D1
:10790000D1FF5A28174C0CD1012222702A211D20A8
:10791000FFF7F8FE022001F099FB134B01221A60D9
:1079200038BD0F211920FFF7BDFF332805D10223F1
:1079300023708F2220211920EAE70D211E20FFF756
:10794000B1FFC7280AD1032500222A211E20257055
:10795000FFF7D8FE2A462A211E20D9E700232370EC
:10796000D8E700BF340000206C780120002838B52B
:1079700004DC1C20BDE83840F9F766BF0B6813F043
:10798000010401D10D20F5E75B10012B2ADD022B4C
:1079900003D0052BB4BF02240324194B1B680BB979
:1079A000FFF7AAFF174B93F90050022D1CD0032DAF
:1079B0001ED0012D11D1032C08BF022400222A2140
:1079C0001D20FFF79FFE22460E211D20FFF79AFE85
:1079D0002A462A211D20FFF795FE022001F036FBE2
:1079E000002038BD0024D8E7220123211920F2E726
:1079F000032C14BF224602220E211E20EBE700BFFB
:107A00006C78012034000020204B1B6810B5044620
:107A10000BB9FFF771FF1E4B93F90030022B0AD010
:107A2000032B25D0012B26D121461D20FFF73AFF3D
:107A30004FF0FF3405E0012C13D129211920FFF765
:107A400031FF7F28C8BFA0F580706FF07E03984299
:107A5000B8BF1846C82358437F2390FBF3F0604318
:107A600010BD032C0BD12B211920DFE72D21FBE7C3
:107A700021461E20DAE74FF0FF340020EAE7052C0C
:107A8000F4D04FF0FF340020DFE700BF6C78012016
:107A90003400002008B50120FFF7B6FF400040F099
:107AA000010008BD08B50320FFF7AEFF400040F01D
:107AB000010008BD08B50520FFF7A6FF400040F013
:107AC000010008BD38B5134B1B6813B90120FFF73F
:107AD0009BFF114B93F90030013301D1FFF70CFFED
:107AE0000120FFF791FF04460320FFF78DFF0546B5
:107AF0000520FFF789FF6D4304FB045400FB0040A1
:107B000003F072F901F0EEFD03F088FC400040F054
:107B1000010038BD6C78012034000020234B1B6825
:107B200070B506460BB9FFF7E5FB214C94F9001040
:107B300000291BDA0F211920FFF7B4FE332811D1D9
:107B40001C4B68221A701C4B1E2500221A706021E3
:107B50000C2228462570FFF7D5FD02226121284618
:107B6000FFF7D0FD94F9001000291EDBC9B21348BD
:107B7000124D00F023FF0F4B1048197800F002FE61
:107B80000E4800F086FF21780C48062200F013FF13
:107B9000741E0536284600F0ECFD30B1284600F092
:107BA000EBFD04F8010FB442F4D170BD6078012000
:107BB000350000203700002036000020D47B012053
:107BC00073B5002368460093ADF80430FFF7A6FFB5
:107BD000FFF718F91C4B9DF8015093F900609DF8D0
:107BE00002009DF800309DF803409DF804209DF8A8
:107BF000051006B345EA032344EA00201BB200B295
:107C000041EA0222114991F90010102912B202BF73
:107C1000DB105210C010002BB8BF5B420028B8BF69
:107C20004042002A1844B8BF52421044400040F07D
:107C3000010002B070BD43EA052340EA04201BB2F4
:107C400000B242EA0122DDE73600002035000020C4
:107C50000128F8B535DD0F68FB0732D54D6815F002
:107C600001062ED1042D2CD92B6803F00F03092B0C
:107C700027D16C68144B64101B68202CA8BF2024EB
:107C80000BB9FFF723FBC7F3470122460F480F4FFD
:107C900000F091FE0435A64211DA0C4800F069FDAF
:107CA00018B9700040F00100F8BD384600F064FDDE
:107CB000400040F0010045F8040F0136EBE760009A
:107CC000F0E70120F0E700BF5C780120187B01207D
:107CD0000A4B0B4A30B5D3F834450A4BA34208BFD0
:107CE0001346013B0246FF24151AA94205DD13F88D
:107CF000015F02F8015B1C70F6E730BD00800240B6
:107D00007478012074790120064B01225A60DA60F0
:107D1000D3F85821002AFBD00022C3F80025024BDB
:107D20001A607047008002407078012038B52C4BF3
:107D30001B680D4623B92520BDE83840F9F784BDFE
:107D4000012801DC1C20F7E70C68E10709D4042CAA
:107D500009D9236803F00F03DA1E012A05D924206C
:107D6000EAE70223F8E70123F6E76A68D20701D4BD
:107D70001120E1E7042B0CD12046FCF7E1FA03F0D7
:107D8000A7FF6A685210013A01D4824209DB12202F
:107D9000D2E72068C0F30F12C0F34170C0EB82003D
:107DA000EFE71049D1F82031C3B1801A80280E4A7C
:107DB000A8BF802004340023834204DA14F8015B56
:107DC0009D540133F8E70023C1F84805C1F820317C
:107DD00001238B60400040F0010038BD1846F9E7F0
:107DE0007078012000800240747A012070B5174D30
:107DF000174CD5F83435174E9C4214BF23463346F2
:107E00004FF480721846FF2103F0C2FB4FF48073D9
:107E1000C5F83405C5F838350023C5F80831012305
:107E20002B60D5F83405844208BF344604F1FF00C6
:107E3000A21E0178FF2900F1FF3301D19A4202D13D
:107E4000001B013070BD1846F3E700BF0080024000
:107E50007479012074780120002838B504DC1C20D6
:107E6000BDE83840F9F7F0BC0D68EB0706D4042DE7
:107E700004D92B6803F00F03032B01D02420EFE774
:107E8000124B1B680BB92520EAE7114BD3F80831D8
:107E90000BB9012038BDFFF7A9FF041EF9D001DAA4
:107EA0001B20DDE7284650F8043BC3F30F12C3F351
:107EB0004173C3EB82039C4228BF1C462146FFF757
:107EC00007FF600040F00100E4E700BF7078012088
:107ED000008002400028F8B504DC1C20BDE8F84012
:107EE000F9F7B2BC0968CB0701D40D20F6E71E4DA7
:107EF0001E4C2B68491023B1D4F800350BB1FFF7A5
:107F000003FF1B4B1A68C4F814255B68C4F80C35D2
:107F10004FF486734B43C4F82435164B4FF48072EC
:107F2000FF21184603F034FB4FF48073C4F8340586
:107F3000C4F83835104BC4F844358023C4F84835AC
:107F40002023C4F80032002601270823C4F8003596
:107F50000520C4F808612760C4F84865A76001F0EF
:107F600075F82F603046F8BD70780120008002401F
:107F700010E3000074780120747A012070B5124E6D
:107F800004460D46002D14DDD6F8203193B1802D26
:107F900010DC0E4B621914F8011B03F8011FA242FA
:107FA000F9D1094B0022C3F84855C3F8202101221A
:107FB0009A6070BDFDF780F9FEF74AFDFEF722FFDB
:107FC000012001F043F8DDE700800240737A0120D0
:107FD00006490A6808B52AB1054BD3F800350BB13C
:107FE000FFF792FE0020086008BD00BF70780120F6
:107FF0000080024038B51C4B1B6823B92520BDE822
:108000003840F9F721BC194BD3F8083113B9184D92
:10801000284638BDFFF7EAFE041EF8D001DA1B201F
:10802000EDE7E11C002289100320FCF725FB054643
:1080300008B90A20E3E721460430FFF749FEEB07C1
:10804000E6D4042DE4D92A6802F00F03032BDFD114
:1080500004F00303C3F104035B0703F0C04322F001
:10806000C04213432B60D3E77078012000800240A8
:1080700038000020002837B504DC1C20F9F7E4FBA9
:1080800003B030BD1C4B1B680BB92520F6E7086810
:1080900010F001040CD04310FF2B01D92820EDE78C
:1080A00002A8012100F8013DFFF768FF0020E7E783
:1080B000042813D9036803F00F02042A10D1FCF737
:1080C0003FF9054603F004FE8028014603D9262027
:1080D000F9F7BAFBEAE72846FFF750FF2046CFE75B
:1080E000032AFBD1C3F30F11C3F34173C3EB810127
:1080F0008029ECDC0430EFE770780120024A034865
:108100000621FEF7A7B800BF88E00000B8E0000035
:108110000020704701207047002070470020704702
:1081200000207047012070470020704700207047F2
:1081300000207047002070470020704700207047E3
:10814000002070470020704700207047704770473C
:1081500070470000024A03480F21FEF77BB800BFBA
:10816000D8E0000050E100000246104601320378DA
:10817000013B1F2BF9D9704708B5FFF7F5FF0378CE
:10818000002B39D0222B00F1010011D1037823B14B
:10819000222B00F1010204D11046BDE80840FFF790
:1081A000E3BF5C2B02D1437803B1821C1046EDE79C
:1081B0003A2BF2D02C2BF0D07B2B0BD1FFF7D4FF36
:1081C0000378002BE9D07D2B01D10130E5E7FFF7E3
:1081D000D3FFF5E75B2B10D00246104612F8013BA7
:1081E000002BDAD0202BD8DD2C2B05D003F0DF01BB
:1081F0005D2901D0222BF0D108BDFFF7B5FF037830
:10820000002BCAD05D2BE0D0FFF7B6FFF7E708B52B
:10821000F0B1FFF7A9FF0378222B1AD07B2B1AD0DD
:108220005B2B1AD0A3F13002092A05D92D2B05D1D9
:108230004278303A092A07D8032009E0742B0ED07F
:10824000662B0ED06E2B0ED0181C18BF012040429A
:1082500008BD0420FCE70220FAE70120F8E705202A
:10826000F6E70620F4E70720F2E738B5FFF77CFFD2
:1082700003782D2B11D101304FF0FF34431E002124
:108280000A2501E005FB012113F8012F303AD0B295
:108290000928F7D904FB01F038BD0124EEE710B539
:1082A0001446FFF761FF0378222B02D000230B70E6
:1082B00010BD621E01300378222BF7D0002BF5D0C1
:1082C0005C2B07D0441C002AF0DD01F8013B013A89
:1082D0002046F0E74378622B00F1020409D0662BB8
:1082E00009D06E2B09D0722B09D0742B08BF09233B
:1082F000E9E70823E7E70C23E5E70A23E3E70D2393
:10830000E1E710B50446FFF737FF0346A3421846DE
:1083100005D90278013A1F2A03F1FF33F6D910BDBF
:1083200008B590B1037883B1FFF71EFF037803F01F
:10833000DF035D2B09D0FFF71FFF03782C2B08BF4D
:108340000130BDE80840FFF70FBF002008BD38B579
:108350000D1E0DDD03785B2B0AD10130FFF704FF02
:108360000124A54205D0FFF7DBFF10B10134F8E787
:10837000002038BD38B5154609B100230B70F8B19F
:108380000378E3B1FFF7F0FE03782C2B044603D10A
:108390000130FFF7E9FE044623787D2B0FD019B199
:1083A0002A462046FFF77BFF2046FFF7E5FE0378CD
:1083B0003A2B05D10130BDE83840FFF7D5BE00208B
:1083C00038BD2DE9F0410D469AB004462F789FB391
:1083D0002E21284603F065FC804690B1461B303FB5
:1083E000092F13D82846FFF740FF01462046FFF724
:1083F000AEFF044604B3B8F1000F1DD0013635447A
:10840000E4E7284603F064FC0646E8E723787B2B84
:1084100011D1601C642201A9FFF7ACFF044658B1DA
:108420003246294601A803F05BFC0028E2D0204632
:10843000FFF7A2FEEEE7002420461AB0BDE8F08167
:1084400038B50D1E04461CDDFFF7E1FE012807D1FB
:10845000601C012D00D138BDFFF762FF013DF8E738
:1084600002280ED100221146601CFFF783FF012D68
:10847000F1D0FFF755FF00221146FFF77BFF013DCA
:10848000F5E70020E7E7F8B50C1E074615461E463F
:1084900013DDFFF7BCFE02280FD132462946781CB7
:1084A000FFF768FF012C00D1F8BDFFF739FF324616
:1084B0002946FFF75FFF013CF4E70020F4E710B521
:1084C0000446C8B1FFF750FE03787B2B0AD1013078
:1084D000002400221146FFF74DFF68B1FFF74CFE64
:1084E0000134F6E75B2B06D101300024FFF718FFBB
:1084F00010B10134FAE70024204610BD002870B501
:1085000014DD0D68EB0711D56D10013DFDF7D0F8B6
:1085100000264FF0FF3460B916B3304603F0D8FBA5
:1085200001463046BDE87040FCF727B94FF0FF35F3
:10853000ECE70368C3F30742152A0BD1C3F3072303
:108540009C42B8BF1C469D4201D100F10806FCF7D1
:10855000AFFFE0E71D2A04BF00264FF0FF34F6E727
:10856000601C400040F0010070BD000010B50868BC
:108570000C46FBF7E5FEFEF723FC0028A2BF034BE9
:10858000626843F82020002010BD00BF688E0120E3
:1085900008B50868FBF7D4FEFEF712FC0028AABF56
:1085A000024B012053F8200008BD00BF688E012057
:1085B00008B50868FBF7C4FEFEF702FC0028ACBF54
:1085C0000420002008BD0000024A03480421FDF7F2
:1085D00041BE00BFECE10000E6E1000008B5FBF79A
:1085E000BBFDFBF781FEFDF7A7FE0448FEF7F9F897
:1085F000FDF7AEF8BDE80840FEF7D6B93BE2000053
:10860000FAF702BF38B50025057329B90B4B0C4AA0
:108610000C48252102F02AFF01600B4951F8222065
:10862000027151F8233083719DF8103051F82330D6
:1086300043710223C371856038BD00BF53E200005F
:10864000B2E2000061E2000010E30000037B23B906
:1086500043738373036101230373704784B00DF187
:10866000100C0CE90E009DF8081002680023012987
:10867000C2F80035039B12D00BD303290CD0C2F8EB
:108680005435019BC2F824350123C2F8003504B0EB
:10869000704743F00203F2E743F00403EFE743F0CF
:1086A0000603ECE710B5FFF7D1FF03688279C3F842
:1086B00008254279C3F80C250279C3F81025034B2D
:1086C000BDE810400ECBFFF7C9BF00BF0C7B0120F7
:1086D00010B485B001AC84E80E0094E80E0005B03B
:1086E0005DF8044BFFF7BABF70470368C3F81C1569
:1086F000D3F80821002AFBD0D3F818050022C3F8CC
:108700000821C0B27047000007B5094B09490A4863
:108710004FF080421A6000229A6002221A710F23E1
:1087200000930E220D23FFF76DFF03B05DF804FBED
:108730000C7B012000300240F87A01202DE9F8433B
:1087400080460D46174601EB02090C464C45A4EB4A
:1087500005060BD0D8F8003014F8011B1B68404602
:1087600098470028F2D13046BDE8F8833E46FAE744
:108770007047203000F03CBA203000F02BBA203097
:1087800000F03CBA38B5437F0D460BB9002038BD28
:1087900000F16804204600F039FA0028F6D120469E
:1087A000294600F008FA0120F1E700002DE9F04128
:1087B0001E4600254FF47A73C0E901530C4B044662
:1087C00040F8203B8846174600F0ECF904F16800B9
:1087D00000F0E8F99DF8183063769DF81C30267695
:1087E000C4E90487A37665772046BDE8F08100BF21
:1087F000F8E20000F0B5837E2E4C2F4D0121C176AA
:1088000054F82320437E54F8233012F0200F14BF75
:108810002F464FF0A04702F01F0213F0200F03F085
:108820001F0308BF4FF0A04502F5E07203F5E073A7
:1088300040F20C6647F8226045F8236003694FF068
:10884000CC72C3F8242503690622C3F80025827E72
:10885000036954F82220C3F80825427E036954F8BE
:108860002220C3F80C2590F91830144A5C0903F053
:108870001F03994004F1600342F8231090F9183067
:10888000002BBDBF03F00F0302F6FC32D2189B1879
:10889000B5BF40234022137683F8002390F91830A7
:1088A0000122590903F01F0302FA03F3034A42F8B5
:1088B0002130F0BD10E300000003005000E100E0B3
:1088C000C37EA3B103690022C3F800250A4B994275
:1088D0000ED90A4B994294BF4FF080614FF0C861A6
:1088E0000369C3F8241503690622C3F800257047FD
:1088F0004FF0CC71F4E700BFA086010090D00300D8
:108900002DE9F041044688461F461546002A50D0FE
:1089100000F12006304600F059F92369C3F8888534
:10892000236901221A622369C3F834652369C3F8F5
:10893000385523691A602269D2F84C311BB9D2F834
:108940002431002BF8D00023C2F84C312269D2F830
:108950005C311BB9D2F82431002BF8D00023C2F8C7
:108960005C3122696FB9D2F8243153B90123D36144
:108970002369D3F84821002AFBD00022C3F84821FC
:1089800009E0012353612369D3F80421002AFBD0B5
:108990000022C3F804212369D3F8242112B1002254
:1089A000C3F824212369D3F83C052066C0B2BDE892
:1089B000F0811046FBE70123FFF7A2BF10B5044684
:1089C00080F8B010683000F001F90123637710BD22
:1089D000F8B500234377036990F8B020C3F88825E1
:1089E000036901261E62036900F168050446C3F8A5
:1089F000445528460F4600F0FBF82369C3F84805A4
:108A000023699E602369D3F850211AB9D3F8242131
:108A1000002AF8D00022C3F85021284600F0E8F8D8
:108A2000236930B1D3F860211AB9D3F82421002A80
:108A3000F8D00022C3F8602123696FB9D3F824214C
:108A400052B90122DA612369D3F84821002AFBD008
:108A50000022C3F8482109E001225A612369D3F8B2
:108A60000421002AFBD00022C3F804212369D3F893
:108A7000240168B10022C3F824212369D3F8C40477
:108A8000C3F8C404022803D004280CBF0320042028
:108A9000F8BD0121FFF79CBF70B54369D3F864218D
:108AA000044692B10022012500F12006C3F864219A
:108AB0000577304600F08AF86369C3F83465636966
:108AC0004022C3F8382563691D636369D3F86821C0
:108AD000DAB10025C3F8685104F168060123637711
:108AE0002577304600F072F8D4F8B43003B19847D7
:108AF000636965773046C3F8446500F079F86369C7
:108B0000C3F84805636901225A636369D3F80421F5
:108B100062B10022C3F80421237F3BB16369D3F81B
:108B20003C05D4F8B830206603B198476369D3F8A0
:108B3000242152B10022C3F824216369D3F8D02440
:108B4000C3F8D024636901225A6170BD0148FFF760
:108B5000A3BF00BF187B01200148FFF79DBF00BFE6
:108B6000D47B012007B514231322CDE900324FF046
:108B70004022114604230848FFF718FE074A084818
:108B80001E231F21CDE9003103231146FFF70EFEFE
:108B900003B05DF804FB00BF187B012000300040EB
:108BA000D47B012008B54022002102F0F1FC002214
:108BB000C0E9102208BD026C10B5531C446C03F0D0
:108BC0003F039C421CBF8154036410BD0023C0E9D5
:108BD00010337047D0E9102393421FBFC25C0133AA
:108BE00003F03F03436414BF10464FF0FF3070475B
:108BF000D0E91030181A48BF40307047D0E9102330
:108C0000934214BFC05C4FF0FF307047036C406C60
:108C1000013303F03F031B1A5842584170470000CC
:108C20000649074A074B9B1A03DD043BC858D0503E
:108C3000FBDC00F013F8F7F703FB0000B8E70000D7
:108C40000000002044020020FEE7FEE7FEE7FEE70A
:108C5000FEE7FEE7FEE7FEE7FEE7FEE7394B1A68B0
:108C60000D2A08D14FF080420021C2F80C11C2F841
:108C70001011C2F838151B680D2B46D14FF08052E9
:108C8000314BD2F80414C3F82015D2F80814C3F8F5
:108C90002415D2F80C14C3F82815D2F81014C3F810
:108CA0002C15D2F81414C3F83015D2F81814C3F8E0
:108CB0003415D2F81C14C3F84015D2F82014C3F8A8
:108CC0004415D2F82414C3F84815D2F82814C3F870
:108CD0004C15D2F82C14C3F85015D2F83014C3F840
:108CE0005415D2F83414C3F86015D2F83814C3F808
:108CF0006415D2F83C14C3F86815D2F84014C3F8D0
:108D00006C15D2F84424C3F870250E4B1B680D2B4C
:108D100009D14FF08043D3F80024D20744BF6FF04D
:108D20000102C3F80024094AD2F8883043F47003E2
:108D3000C2F88830BFF34F8FBFF36F8F044B054AE3
:108D40001A6070473001001000C0004000ED00E0E4
:108D50003C0000200090D0030120704703681322DC
:108D6000DB69184770470369C3F81C150369D3F81A
:108D70001C21002AFBD00022C3F81C2101207047CF
:108D800010B490F95C30144C59090122203103F0E1
:108D90001F0302FA03F344F8213003695DF8044B22
:108DA0000421C3F8081303695A600369DA60036990
:108DB0000022C3F8002502694FF0FF33C2F80C35DA
:108DC0000269C2F814350269C2F808350269143024
:108DD000C2F81035FFF7FABE00E100E01430FFF7EB
:108DE00007BF1430FFF70ABF1430FFF7F3BE0000CF
:108DF000036990F85E2010B5C3F80C25036990F85C
:108E00005D20C3F8142590F861200369012A01BF91
:108E100090F85F40C3F81045036990F8604006BFC2
:108E2000C3F8084503690022B1F5966FC3F86C25B5
:108E300069D9B1F5166F69D9B1F5965F69D9B1F500
:108E4000165F68D9B1F5615F67D9B1F5964F66D9FC
:108E5000B1F5E14F65D9B1F5164F64D9B1F5614F60
:108E600064D9B1F5963F64D9B1F5E13F63D9B1F565
:108E7000613F63D9364B994263D9B1F5E12F63D98C
:108E8000B1F5612F94BF4FF070634FF080530269CA
:108E9000C2F8243503690422C3F8002501690023C0
:108EA000C1F808310169C1F81C31016901230B6067
:108EB00001698B600169C1F8042390F95C205109B4
:108EC00002F01F0293406031224A42F8213090F9AB
:108ED0005C30002BBDBF03F00F0302F6FC32D2184A
:108EE0009B18B5BF60236022137683F8002390F9A6
:108EF0005C300122590903F01F0302FA03F3154AFB
:108F000042F8213010BD4FF49E23C0E74FF41D23DB
:108F1000BDE7114BBBE7114BB9E7114BB7E7114B5D
:108F2000B5E7114BB3E74FF41D03B0E74FF46B0304
:108F3000ADE70E4BABE74FF0EB73A8E74FF06C7368
:108F4000A5E74FF08063A2E74FF0E8639FE700BF1B
:108F500090D0030000E100E000B0130000502700B3
:108F600000F03A0000A04E0000C0750000903A01E9
:108F70002DE9F0411E4600254FF47A73C0E90153F4
:108F80000D4B044640F8143B17468846FFF70AFE8F
:108F90000A4AC4F8108084F85C7052F8263084F8CD
:108FA0005D309DF8183052F8233084F85E3084F834
:108FB00061502046BDE8F081A4E3000010E300000A
:108FC00010B50369D3F8082104464AB1D3F818153F
:108FD0001430C9B2FFF7EFFD23690022C3F808215E
:108FE00010BD00000148FFF7EBBF00BF907C0120DF
:108FF00007B5222300930222212303490348FFF7E8
:10900000B7FF03B05DF804FB00200040907C012016
:1090100008B102F08BBD70470A4B19680A4B30B596
:10902000D3F804050C060D0A44EA00024FF47A71E5
:109030002B46A2FB014501FB0355E00B40EA4540EE
:1090400030BD00BFF47C01200010014038B504465B
:1090500048B1FFF7E1FF054600F01AF8FFF7DCFF23
:10906000401BA042F8D338BD074B0022C3F80421AF
:1090700082B0D3F80431054A0193019B1368013390
:10908000DBB2136002B0704700100140F47C012095
:109090007047704708B500F067F8FFF7FAFF012046
:1090A000FFF7D4FFFFF79AFA034CFFF7A9FA002C59
:1090B000FBD0AFF30080F8E70000000038B5174B95
:1090C000174D53F82030174813F0200F4FF00104CC
:1090D00003F01F0304FA03F408BF4FF0A040002977
:1090E0002B681149B3FBF1F300F5A26002FB03F317
:1090F00021464FF00A02B3FBF2F314BF22460022CE
:1091000000F014F842F2107358434FF47A722B684F
:10911000B3FBF2F3B0FBF3F038BD00BF10E3000087
:109120003C0000200003005040420F0030B50468AE
:109130000C40944206D1013B002BF8D112E0013BD8
:10914000002B0FD004680C409442F8D1002405682D
:109150000D40954204D101349C42F8D1002002E038
:10916000201C00E0181C30BD0D4BE02283F81123B9
:109170004FF40032C3F880211A604FF0804301227F
:10918000C3F818259A6003F588330021C3F8081541
:109190000221C3F80413C3F844131A60704700BFD8
:1091A00000E100E0014B1860704700BF580000204C
:1091B0000228064A064B1BBF002111600121012233
:1091C00012BF1A6011601860704700BF007D012057
:1091D00054000020222837B50CD84B4B53F82030D0
:1091E000052B00F0828007D8032B12D07BD8022BEE
:1091F00000F08180002074E01D2B78D003D81C2B58
:10920000F8D1052206E01E2B73D01F2BF2D10822C5
:1092100000E002223D4B196808296EDD0A296FDD46
:109220000D29B5BF0C240E24022303233848C0F8AF
:10923000F0350123C0F8003500200546030103F195
:10924000804303F5E04301300828C3F81455C3F800
:109250001055F3D12F4B18682F4B1B6800021B03CE
:1092600003F4805300F4E0601843294BC3F8180559
:10927000C3F81425C3F810250DF10602C3F82C26F7
:109280000122C3F830261A60D3F80021002AFBD04F
:109290000022C3F8002101225A601D4B1A46D3F860
:1092A00004010028FBD00020C3F8040101209860CD
:1092B000D2F81431002BFBD00023C2F81431BDF9D1
:1092C00006209A42124AB8BFADF80630A142C2F851
:1092D0000035BDF9060004D035BF611A091BC8402E
:1092E000884003B030BD032294E7042292E70622AF
:1092F00090E707228EE701228CE70824002395E7F8
:109300000A24012392E700BF10E300005000002070
:109310000070004054000020007D0120222830B55C
:109320003CD8224B53F82000214B00221D4653F815
:109330002240B4F1FF3F32D11E4C45F822006FEAC3
:1093400041411D4D1D4B246853F822306FEA5141B5
:1093500025F81210012101FA04F4C3F86005013C5C
:10936000C3F8640505EB4202C3F86805C3F86C0551
:109370000020C3F80015C3F80C05C3F80405C3F8B2
:109380000845C3F81405C3F81005C3F82025C3F831
:109390002415C3F82815C3F82C05996030BD844204
:1093A000CAD00132042AC2D1F8E700BF10E300009E
:1093B0004000002058000020F87C0120CCE3000091
:1093C000222815D8114B124A53F8203013F0200FE1
:1093D00008BF4FF0A04203F01F03032908D8DFE8BD
:1093E00001F00210080C03F5E073002142F823108D
:1093F000704703F5E0730C21F8E703F5E0730421EF
:10940000F4E703F5E0730321F0E700BF10E3000089
:1094100000030050222813D80A4B53F820000A4BAF
:1094200010F0200F4FF0010200F01F0008BF4FF0B6
:10943000A043824011B9C3F80C257047C3F8082532
:10944000704700BF10E3000000030050222810D82E
:10945000094B0A4A53F8203013F0200F08BF4FF091
:10946000A04203F01F03D2F81005D84000F001001D
:1094700070470020704700BF10E300000003005059
:109480002DE9F04106460D4601EB02080C46444525
:10949000A4EB050707D0336814F8011B1B6830469E
:1094A00098470028F3D13846BDE8F0812DE9F04116
:1094B000C1F30A57A7F2FF35132D82B002460B46BF
:1094C0000C464FEAD178064633DC002D4EDB3C4992
:1094D000294103EA0100104326D049080B4052EA13
:1094E00003060CD04FF48023132D24EA010143FA24
:1094F00005F444EA01040CBF4FF000460026314950
:1095000001EBC8082346D8E90045324620462946E3
:1095100001F01EFBCDE9000122462B46DDE90001EA
:1095200001F014FB02460B461046194602B0BDE896
:10953000F081332D07DDB5F5806FF5D101F008FB23
:1095400002460B46F0E7A7F213474FF0FF31F94010
:109550000842E9D049080842D1D04FF0804320EAC0
:10956000010143FA07F741EA0706C8E721F0004185
:109570000143D9D0C3F3130101434E420E43114DB1
:109580005C0C360B640406F4002305EBC80243EAC6
:109590000401D2E900450B4602462946204601F067
:1095A000D7FACDE9000122462B46DDE9000101F0A2
:1095B000CDFA21F00041024641EAC873B4E700BF8A
:1095C000FFFF0F00E0E30000F8B5C1F30A57A7F270
:1095D000FF35132D02460B460C4610DC002D29DB0F
:1095E0008C461D4929410B422AD04FF400242C41BE
:1095F000644424EA0104002621463046F8BD332D98
:1096000005DDB5F5806F1ED010461946F8BDA7F2EE
:1096100013474FF0FF3121FA07F73842F4D0012306
:10962000C5F1330503FA05F5461928BFE41826EA03
:109630000706E1E7013501F0004407D00026DBE72B
:109640000028D2D1E0E701F083FAF8BD44F07F545E
:1096500044F440140026CFE7FFFF0F0030B51F4A47
:1096600021F00043934287B01CDD1D4A934205DD83
:1096700002460B4601F06AFA07B030BD02AA00F0BC
:109680008FF800F003000128DDE9042312D002283E
:109690001CD0A0B1DDE9020100F066FB01F1004140
:1096A00007B030BD002300930022002301F084F8AE
:1096B00007B030BDDDE9020100F056FBDCE7012414
:1096C000DDE90201009401F077F8D5E70124DDE936
:1096D0000201009401F070F8E0E700BFFB21E93FD0
:1096E000FFFFEF7F2DE9F04F8BB004460D4600F0F1
:1096F00079FA294B93F900A0BAF1FF3F06460F46CD
:1097000012D022462B462046294601F071FE8346A0
:1097100050B94FF000084FF0000920462946424654
:109720004B4601F03DFE20B9304639460BB0BDE84E
:10973000F08F0122194BCDF820B00092CDE90445FD
:10974000CDE902450193BAF1000F17D042464B46CE
:109750004046494601F0DCFCBAF1020FCDE90601B2
:109760000ED101F0A1FE21230360089B73B9DDE94E
:109770000667304639460BB0BDE8F08FCDE9068963
:10978000684601F055F90028EFD1EAE701F08CFEB8
:10979000089B0360EBE700BF5C000020F0E30000E3
:1097A0002DE9F047CA4B21F000479F4290B0804618
:1097B000894640F38F80C74B9F420C46924626DC79
:1097C0000029B9A3D3E9002340F38F8001F0BEF94B
:1097D000C14B9F4204460D4600F04781B4A3D3E934
:1097E000002301F0B3F902460B46CAE900232046E4
:1097F000294601F0ABF9AEA3D3E9002301F0A6F9A5
:109800000125CAE90201284610B0BDE8F087B34B34
:109810009F4240F38980B24B9F4200F31C813D156B
:10982000A5F21645A7EB055319461F46064601F05B
:10983000F5FD01F0D9FA8046894642464B4630464E
:109840003946CDE90A8901F081F90022A54B01F0E2
:1098500035FB8946804601F0E1FD01F0C5FA064678
:109860000F4632463B4640464946CDE90C6701F07B
:109870006DF900229B4B01F021FB00220023CDE972
:109880000E0101F083FD002800F0608100233046C6
:109890003946002201F07AFD002814BF012302237B
:1098A000914A019202212A4600910AA8514600F0ED
:1098B00083FB002C054614DADAF80420DAF80C30C1
:1098C00002F1004203F100434542CAF80420CAF8FD
:1098D0000C3006E000200021C2E90089C2E9020143
:1098E0000025284610B0BDE8F08701F031F97A4B29
:1098F0009F4204460D4600F00B816DA3D3E900237F
:1099000001F026F902460B46CAE900232946204603
:1099100001F01CF966A3D3E9002301F019F94FF017
:10992000FF35CAE90201DCE700F0FCFF62A3D3E9DE
:1099300000238046894601F0C1FA00226B4B01F0FA
:1099400007F901F06BFD054601F04EFA56A3D3E985
:109950000023CDE9060101F0B1FA02460B4640466C
:10996000494601F0F3F852A3D3E900238046894623
:10997000DDE90601CDE9028901F0A0FA1F2D0246BA
:109980000B46CDE9042340F3B380DDE90423DDE990
:10999000020101F0DBF8804689463F15C9F30A53FE
:1099A000FB1A102B40F3B18045A3D3E90023DDE976
:1099B000060101F083FA8046894602460B46DDE93E
:1099C000020101F0C3F802460B46DDE90201CDE9D0
:1099D000082301F0BBF842464B4601F0B7F83AA322
:1099E000D3E9002380468946DDE9060101F066FAE5
:1099F00042464B4601F0AAF80B46CDE90401024667
:109A0000DDE9080101F0A2F8C1F30A53FF1A312F72
:109A10008046894600F39C809DED087BCAE9008959
:109A20008DED027B42464B46DDE9020101F08EF8E6
:109A3000DDE9042301F08AF8002CCAE90201BFF62F
:109A400050AF09F1004401F100436D42CAE90084BE
:109A5000CAE9020345E702460B4601F077F8002504
:109A6000CAE90201CAE900013BE715A3D3E90023D3
:109A700001F06CF814A3D3E900230D46044601F06D
:109A800065F802460B46CAE900232946204601F044
:109A90005DF80DA3D3E9002301F058F80125CAE9C8
:109AA00002011EE7AFF3008000004054FB21F93FA4
:109AB0003163621A61B4D03D83C8C96D305FE43F41
:109AC0000000601A61B4D03D7370032E8A19A33B65
:109AD000FB21E93F7BD90240FB21F93FFB213941C2
:109AE000FFFFEF7F0000704178E400000000E03FDE
:109AF0004046494601F02AF8394B6A1E804653F821
:109B00002230BB4289463FF448AFCAE9008989E761
:109B10002BA3D3E9002301F01BF82BA3D3E90023E7
:109B20000D46044601F014F802460B46CAE900232C
:109B30002946204601F00AF823A3D3E9002301F0C7
:109B400007F84FF0FF35CAE90201CAE60323A7E68A
:109B50001FA3D3E90023DDE9060101F0AFF90646B2
:109B60000F4602460B46DDE9080100F0EFFF804694
:109B7000894602460B46DDE90801CDE9028900F07D
:109B8000E5FF32463B4600F0E1FF13A3D3E9002393
:109B900006460F46DDE9060101F090F932463B46E4
:109BA00000F0D4FF02460B4640464946CDE9042367
:109BB00000F0CCFF80468946A7E700BFAFF30080E6
:109BC0000000601A61B4D03D7370032E8A19A33B64
:109BD0000000002E8A19A33BC14920259A837B39B6
:109BE000F8E300005E4A8A432DE9F04104460D4641
:109BF00000F0958000290B460646844656DD0F1579
:109C000000F0A580C3F31303A7F2FF3743F48013DA
:109C10004FEADC72F80702EB43034FEA4C0504D528
:109C2000ED0F05EB43034FEA8C0500267F10B44689
:109C300016224FF400110CEB010098424FEAD57444
:109C40004FEA450503DC1B1A00EB010C0E44013AF8
:109C500004EB43034FEA5101EDD110469646202410
:109C60004FF0004209E051D05B00013C03EBD5739B
:109C70004FEA52024FEA450537D0634502EB0E0129
:109C8000F1DD002901EB020E0ADBE046A3EB0C0339
:109C9000A94288BF03F1FF336D1A1044C446E3E7BD
:109CA000BEF1000FF1DB0CF10108EFE721F00042FB
:109CB000024329D0002942D10146CA0A153B490571
:109CC000002AFAD012F4801001D044E0604652001D
:109CD000D40200F1010CF9D5CCF1200401FA0CFCFE
:109CE000E1401F1A41EA02038CE72B4321D14408CB
:109CF000731003F17F53F20703F5001348BF44F0DC
:109D0000004403EB07512046BDE8F081A942ABD8DF
:109D1000002901EB020EC3DB98460023BCE7024694
:109D20000B4601F0CBF822462B4600F011FFBDE8B0
:109D3000F081411C16BF421C01365408D8E7024688
:109D400000F004FF02460B4601F0E2F9DCE71A4698
:109D500031463B46B6E78C4620244FF0FF30BFE744
:109D60000000F07F000000002DE9F04F21F00048D6
:109D7000B8F1795F85B006460F4692469B466BDA8E
:109D800001F04CFB002800F0E18032463B463046B3
:109D9000394601F093F874A3D3E9002304460D4635
:109DA00001F08CF872A3D3E9002300F0D1FE224623
:109DB0002B4601F083F870A3D3E9002300F0C6FE20
:109DC00022462B4601F07AF86DA3D3E9002300F078
:109DD000BFFE22462B4601F071F86BA3D3E90023A6
:109DE00000F0B4FE22462B4601F068F868A3D3E9E0
:109DF000002300F0ADFE22462B4601F05FF8CDE9CE
:109E000000010022664B2046294601F057F8DDE9A3
:109E10000023804689462046294601F04FF85246E5
:109E200004460D465B463046394601F047F8024687
:109E30000B462046294600F089FE02460B46404666
:109E4000494600F083FE02460B460020554900F0CB
:109E50007DFE05B0BDE8F08F02460B4601F02EF8FE
:109E600041A3D3E9002304460D4601F027F840A39F
:109E7000D3E9002300F06CFE22462B4601F01EF8C9
:109E80003DA3D3E9002300F061FE22462B4601F0FA
:109E900015F83BA3D3E9002300F05AFE22462B46D7
:109EA00001F00CF838A3D3E9002300F04FFE22465E
:109EB0002B4601F003F836A3D3E9002300F048FE57
:109EC0002B46224600F0FAFF374B9845CDE90001BA
:109ED00097DD364B98453EDCA8F5001300220020A4
:109EE00030499046994600F031FECDE9020100224A
:109EF0002B4B2046294600F0E1FF42464B4600F03E
:109F000025FEDDE90023804689462046294600F0EB
:109F1000D5FF524604460D465B463046394600F0B2
:109F2000CDFF02460B462046294600F00FFE0246B2
:109F30000B464046494600F009FE02460B46DDE965
:109F4000020100F003FE05B0BDE8F08F15490020C6
:109F500005B0BDE8F08F9FED107B4FF000088DED50
:109F6000027BDFF84C90C2E7D43888BEE9FAA8BD7E
:109F7000C4B1B4BD9EEE213EAD529C804F7E923E58
:109F80009015CB19A001FA3E7751C1166CC1563F0E
:109F90004C5555555555A53F000000000000E73FC2
:109FA0000000E03F0000F03F3233D33F0000E93FC4
:109FB0000000D23F000000002DE9F04FADF5197D03
:109FC000BE4CA29EBE4D54F826600793D41E85FB5E
:109FD0000475E417C4EBA50424EAE4741D46631C6D
:109FE000A3EB8303013D02EBC303059373190496AE
:109FF0000994019503900B91A4EB05071AD43B44F7
:10A00000002400255E1C0DF18008DDF88C9208E02C
:10A0100059F8270000F0E8FE0137B742E8E80201EE
:10A0200008D0002FF4DA013720462946B742E8E885
:10A030000201F6D1049B002B079B4FEAC303029356
:10A040002ADB039A20A902EB030801EB0309049B16
:10A0500072AA02EBC30B0DF5E07A019B002B4FF0C7
:10A0600000064FF0000711DB039C4D4675E9022303
:10A07000F4E8020100F022FF02460B463046394662
:10A0800000F066FD444506460F46EFD1EAE8026758
:10A09000DA4509F10809E0D1DDE902040499204418
:10A0A0008B0082460BA8A3F10802C31808930CABDF
:10A0B00013440A938B4698AB03EBCB03BBF1000F21
:10A0C00053E9284529DD70AB03EBCB080DF13009CE
:10A0D00000227C4B2046294600F0F0FE01F09EF95C
:10A0E00000F082FE0022784B06460F4600F0E6FEA6
:10A0F00002460B462046294600F028FD01F08EF965
:10A1000078E9022349F8040B3946304600F020FD77
:10A1100070AB984504460D46DAD1DDF81490204620
:10A1200029464A4600F088FC00224FF07F5304463F
:10A130000D4600F0C3FE00F0FBFB0022634B00F075
:10A14000BDFE02460B462046294600F0FFFC0D46A8
:10A15000044601F063F9804600F046FE0B460246D5
:10A160002946204600F0F2FC4B46002B06460F46DF
:10A1700040F3E1800BF1FF320CA9C9F1180351F84B
:10A18000225045FA03F101FA03F30CA8EB1A40F848
:10A190002230C9F11705884443FA05F5002D2CDD5E
:10A1A000BBF1000F08F1010840F381820C9C002CE8
:10A1B00040F0A780BBF1010F0AD00CA9012251F891
:10A1C000044F531C002C40F09E809B451A46F6D14C
:10A1D000059B002B0EDD012B00F0D980022B09D14D
:10A1E0000BF1FF320CAB0CA953F82230C3F315036B
:10A1F00041F82230022D00F0AF80002200233046CB
:10A20000394601F0C3F8002800F05382049B0BF19B
:10A21000FF394B4510DC0BF180430CAA013B089839
:10A2200002EB8303002253F80419834242EA01023D
:10A23000F9D1002A40F0B680049B0CAA013B52F8E9
:10A240002330002B40F0A1800A9A012352F8041910
:10A2500001330029FAD05B440BF1010999450693BB
:10A260004CDC099A079909EB020801EB0B0508F190
:10A27000804802EB030BA39B08F1FF3803EB88082F
:10A2800070AB03EBC909A39B20A903EB8B0301EB84
:10A29000C505029358F8040F00F0A6FD0B4601997E
:10A2A0000246002905F1080BC5E900234FF000061E
:10A2B0004FF000071CDB039C0CE000BFC0E5000072
:10A2C000ABAAAA2A0000703E0000704100002040A6
:10A2D00075E90223F4E8020100F0F0FD02460B46A6
:10A2E0003046394600F034FC544506460F46EFD15F
:10A2F000029B9845E9E802675D46CBD1DDF818B0CE
:10A30000D9E6012300220CA9C4F180749B4541F8D1
:10A3100022400EDD51F8232001EB8B0001EB83037B
:10A320006FF07F4100E01A688A1A43F8042B8342D9
:10A33000F9D101244CE706D10BF1FF330CAA52F8F6
:10A340002350ED152AE700227B4B01F03DF8002851
:10A3500040F0A381054650E732463B46002077494E
:10A3600000F0F4FB06460F46002C3FF446AF059A7A
:10A370007249002000F060FB02460B463046394629
:10A3800000F0E4FB06460F4637E7012363E70BF1D5
:10A39000FF320CAB0CA953F82230C3F3160341F87B
:10A3A000223027E70CAB059A53F82930183ACDE94B
:10A3B000068505926BB909F18043013B0CA901EBBD
:10A3C000830353F8041909F1FF39183A0029F8D02A
:10A3D0000592059A5949002000F02EFBB9F1000FB3
:10A3E00004460D46C0F2C0814FEAC90370AA02EBD1
:10A3F000030808930CAB03EB8906DFF844B14FF078
:10A40000000A08F10807043656F8040D00F0ECFCC9
:10A4100022462B4600F052FD5B4667E90201524698
:10A420002046294600F04AFD0CAB9E4204460D46EC
:10A43000EAD148AB03930193CDF8149009F10103DD
:10A44000DDF810900293C3464FF0000AB9F1000FF7
:10A45000C0F22A81DFF8EC805D4635A3D3E9002302
:10A4600000260027002403E0544510DCF8E802230E
:10A47000F5E8020100F022FD02460B46304639465F
:10A4800000F066FB0134A14506460F46ECDA019B5D
:10A49000E3E802670193029B0AF1010A9A45ABF1D6
:10A4A000080BD3D1A29BDDF81490032B39D8DFE839
:10A4B00013F0D900060006004D0048AB0393B9F134
:10A4C000000F4FF000004FF0000109DB039D05EB8A
:10A4D000C904083474E9022300F03AFBA542F9D11B
:10A4E000079B002B40F01E810B9BC3E900010B462C
:10A4F00003990246D1E9000100F028FBB9F1000FF1
:10A500000CDD4AAD01240134F5E8022300F020FB04
:10A51000A145F8DA079B002B40F014810B9BC3E99F
:10A520000201069B03F007000DF5197DBDE8F08FD1
:10A5300000000040FB21F93F0000E03F0000F03F39
:10A540000000703E88E5000048AB0393B9F1000FAE
:10A5500040F32781039ACDF810904FEAC903019385
:10A56000D318D3E900AB09F10053013B02EBC90852
:10A570000293914678E9026752465B463046394677
:10A5800000F0E6FA04460D4602460B4630463946D0
:10A5900000F0DCFA52465B4600F0DAFAC145A2460A
:10A5A000AB46C8E90201C8E90045E3D1DDF81090E7
:10A5B000B9F1010F40F3F580019B039A029913440E
:10A5C000C900D3E9006701F1080A019192440DF531
:10A5D000947B7AE9028932463B464046494600F080
:10A5E000B7FA04460D4602460B464046494600F07F
:10A5F000ADFA32463B4600F0ABFAD34526462F462D
:10A60000CAE90201CAE90045E3D1019C039B103469
:10A61000002000211C4403F1100574E9022300F01E
:10A6200097FAA542F9D1039C079ED4E90023D4E907
:10A630000245002E00F08A8003F1004701F100433B
:10A640000B99C1E90403069B2646944605F1004494
:10A6500003F00700C1E900C7C1E902640DF5197DE7
:10A66000BDE8F08F089C039D0834002000212C4495
:10A6700074E9022300F06CFAA542F9D1079B13B1EB
:10A6800001F1004319460B9BC3E90001069B03F04F
:10A6900007000DF5197DBDE8F08FBBF1000F08F143
:10A6A000010874DD022581E500260027EFE600247D
:10A6B0008EE5CDE90685059D304639466A4200F0B3
:10A6C000BBF90022384B06460F4600F07DFE00B372
:10A6D0000022364B3046394600F0F0FB00F09EFE7B
:10A6E000044600F081FB00222F4B00F0E7FB0B46F5
:10A6F00002463946304600F029FA00F08FFE0BF191
:10A7000001090CAB183543F82B00059543F8294097
:10A710005FE63046394600F081FE0CABD94643F87F
:10A720002B0056E60B9C01F10043C4E900030B46E5
:10A7300003990246D1E9000100F008FAB9F1000FCF
:10A740003FF7DFAE01F100431946E7E60B9EC6E98D
:10A750000023069BC6E9040103F00700C6E9024591
:10A760000DF5197DBDE8F08FA29B032B3FF6D9AE06
:10A7700001A252F823F000BF89A70000BBA400008B
:10A78000BBA4000049A500000020002176E7324666
:10A790003B460020064900F0D9F9022506460F463F
:10A7A0002BE5002000213EE7000070410000703ED4
:10A7B0000000F03F000000002DE9F04F21F00046BE
:10A7C000B6F1795F85B004460D469046994604DAA5
:10A7D00000F024FE002800F0858022462B4620460B
:10A7E000294600F06BFB06460F4602460B46204604
:10A7F000294600F063FB41A3D3E9002382468B4640
:10A800003046394600F05AFB3EA3D3E9002300F05E
:10A810009DF932463B4600F051FB3CA3D3E90023AF
:10A8200000F096F932463B4600F048FB39A3D3E9E5
:10A83000002300F08BF932463B4600F03FFB37A384
:10A84000D3E9002300F084F90E9BCDE900019BB30E
:10A850000022294B4046494600F030FBDDE9002349
:10A86000CDE902015046594600F028FB02460B464E
:10A87000DDE9020100F06AF932463B4600F01EFBBA
:10A8800042464B4600F062F919A3D3E9002306467D
:10A890000F465046594600F011FB02460B46304623
:10A8A000394600F055F902460B462046294600F08D
:10A8B0004DF905B0BDE8F08F02460B4630463946EB
:10A8C00000F0FCFA0AA3D3E9002300F03FF9524656
:10A8D0005B4600F0F3FA22462B4600F039F905B04A
:10A8E000BDE8F08F2046294605B0BDE8F08F00BFD7
:10A8F000495555555555C53F0000E03F7CD5CF5AC9
:10A900003AD9E53DEB9C2B8AE6E55A3E7DFEB157F0
:10A91000E31DC73ED561C119A0012A3FA6F8101159
:10A920001111813F21F000431946704700000000DB
:10A930002DE9F041C1F30A57A7F2FF35132D024666
:10A940000B460C46884606461DDC002D3CDB364F88
:10A950002F4101EA070C5CEA000C19D030A3D3E9BF
:10A96000002300F0F5F80022002300F037FDC8B303
:10A97000002C04DA4FF4801343FA05F5A84428EAC2
:10A98000070400262EE0332D06DDB5F5806F2DD0AF
:10A9900010461946BDE8F081A7F213474FF0FF3C7F
:10A9A0002CFA07F70742F3D01DA3D3E9002300F0E8
:10A9B000CFF80022002300F011FD98B1002C21DB1C
:10A9C00026EA070644460DE015A3D3E9002300F06C
:10A9D000BFF80022002300F001FD18B1002C08DBB5
:10A9E0000026344621463046BDE8F08100F0B0F83C
:10A9F000D0E724F000430D4A1E43002E18BF144632
:10AA00000026EFE7142D08D00123C5F1340503FA21
:10AA100005F5AE1928BF9844D2E704F10108CFE745
:10AA20009C7500883CE4377EFFFF0F000000F0BFFC
:10AA30000020704700000000F8B5C1F30A53044637
:10AA40000D460E4617460BBB21F000460346334326
:10AA50001BD0354B002200F031FA344B9F420446A4
:10AA60000D4635DBC1F30A530E46363B3B4440F2FC
:10AA7000FE72934232DC002B11DD26F0FF4626F4F5
:10AA8000E00646EA035520462946F8BD40F2FF722B
:10AA90009342EBD102460B4600F05AF8F8BD13F191
:10AAA000350F28DA4CF250339F4222462B460ADDFE
:10AAB00019A1D1E9000100F03DF817A3D3E9002363
:10AAC00000F0FCF9F8BD16A1D1E9000100F032F860
:10AAD00013A3D3E9002300F0F1F9F8BD22462B4679
:10AAE0000DA1D1E9000100F025F80BA3D3E9002363
:10AAF00000F0E4F9F8BD26F0FF4626F4E006363310
:10AB000046EA0355204629460022094B00F0D6F9B3
:10AB1000F8BD00BFAFF300809C7500883CE4377E31
:10AB200059F3F8C21F6EA50100005043B03CFFFF6F
:10AB30000000903C03F0004321F0004242EA030190
:10AB4000704700BF81F0004102E000BF83F0004386
:10AB500030B54FEA41044FEA430594EA050F08BFB8
:10AB600090EA020F1FBF54EA000C55EA020C7FEA7C
:10AB7000645C7FEA655C00F0E2804FEA5454D4EBF9
:10AB80005555B8BF6D420CDD2C4480EA020281EAC3
:10AB9000030382EA000083EA010180EA020281EAFB
:10ABA0000303362D88BF30BD11F0004F4FEA01314D
:10ABB0004FF4801C4CEA113102D0404261EB41015C
:10ABC00013F0004F4FEA03334CEA133302D05242E2
:10ABD00063EB430394EA050F00F0A780A4F101049E
:10ABE000D5F1200E0DDB02FA0EFC22FA05F28018D8
:10ABF00041F1000103FA0EF2801843FA05F35941BE
:10AC00000EE0A5F120050EF1200E012A03FA0EFC3C
:10AC100028BF4CF0020C43FA05F3C01851EBE37166
:10AC200001F0004507D54FF0000EDCF1000C7EEB83
:10AC300000006EEB0101B1F5801F1BD3B1F5001FC1
:10AC40000CD349085FEA30004FEA3C0C04F10104E0
:10AC50004FEA445212F5800F80F09A80BCF1004F09
:10AC600008BF5FEA500C50F1000041EB045141EA8B
:10AC7000050130BD5FEA4C0C404141EB010111F48C
:10AC8000801FA4F10104E9D191F0000F04BF014637
:10AC90000020B1FA81F308BF2033A3F10B03B3F115
:10ACA00020020CDA0C3208DD02F1140CC2F10C02A5
:10ACB00001FA0CF021FA02F10CE002F11402D8BF03
:10ACC000C2F1200C01FA02F120FA0CFCDCBF41EACF
:10ACD0000C019040E41AA2BF01EB0451294330BD9E
:10ACE0006FEA04041F3C1CDA0C340EDC04F114047B
:10ACF000C4F1200220FA04F001FA02F340EA030052
:10AD000021FA04F345EA030130BDC4F10C04C4F197
:10AD1000200220FA02F001FA04F340EA0300294677
:10AD200030BD21FA04F0294630BD94F0000F83F4C1
:10AD3000801306BF81F480110134013D4EE77FEAA4
:10AD4000645C18BF7FEA655C29D094EA050F08BFF0
:10AD500090EA020F05D054EA000C04BF19461046D1
:10AD600030BD91EA030F1EBF0021002030BD5FEA15
:10AD7000545C05D14000494128BF41F0004130BD3D
:10AD800014F580043CBF01F5801130BD01F0004591
:10AD900045F0FE4141F470014FF0000030BD7FEA04
:10ADA000645C1ABF194610467FEA655C1CBF0B46FF
:10ADB000024650EA013406BF52EA033591EA030F16
:10ADC00041F4002130BD00BF90F0000F04BF00210E
:10ADD000704730B54FF4806404F132044FF0000541
:10ADE0004FF0000150E700BF90F0000F04BF0021BA
:10ADF000704730B54FF4806404F1320410F0004520
:10AE000048BF40424FF000013EE700BF42004FEA1A
:10AE1000E2014FEA31014FEA02701FBF12F07F4397
:10AE200093F07F4F81F06051704732F07F4208BF4E
:10AE3000704793F07F4F04BF41F40021704730B555
:10AE40004FF4607401F0004521F000411CE700BFA1
:10AE500050EA010208BF704730B54FF000050AE024
:10AE600050EA010208BF704730B511F0004502D525
:10AE7000404261EB41014FF4806404F132045FEA27
:10AE8000915C3FF4D8AE4FF003025FEADC0C18BFD0
:10AE900003325FEADC0C18BF033202EBDC02C2F1C2
:10AEA000200300FA03FC20FA02F001FA03FE40EA54
:10AEB0000E0021FA02F11444BDE600BF70B54FF058
:10AEC000FF0C4CF4E06C1CEA11541DBF1CEA135536
:10AED00094EA0C0F95EA0C0F00F0DEF82C4481EA9E
:10AEE000030621EA4C5123EA4C5350EA013518BFBE
:10AEF00052EA033541F4801143F4801338D0A0FBAB
:10AF000002CE4FF00005E1FB02E506F00042E0FB57
:10AF100003E54FF00006E1FB03569CF0000F18BF5D
:10AF20004EF0010EA4F1FF04B6F5007F64F5407405
:10AF300004D25FEA4E0E6D4146EB060642EAC62198
:10AF400041EA55514FEAC52040EA5E504FEACE2E05
:10AF5000B4F1FD0C88BFBCF5E06F1ED8BEF1004F08
:10AF600008BF5FEA500E50F1000041EB045170BD84
:10AF700006F0004646EA010140EA020081EA0301C8
:10AF8000B4EB5C04C2BFD4EB0C0541EA045170BDC4
:10AF900041F480114FF0000E013C00F3AB8014F13E
:10AFA000360FDEBF002001F0004170BDC4F1000487
:10AFB000203C35DA0C341BDC04F11404C4F1200508
:10AFC00000FA05F320FA04F001FA05F240EA020063
:10AFD00001F0004221F0004110EBD37021FA04F699
:10AFE00042EB06015EEA430E08BF20EAD37070BD53
:10AFF000C4F10C04C4F1200500FA04F320FA05F0B2
:10B0000001FA04F240EA020001F0004110EBD370B3
:10B0100041F100015EEA430E08BF20EAD37070BD23
:10B02000C4F1200500FA05F24EEA020E20FA04F3FC
:10B0300001FA05F243EA020321FA04F001F00041AB
:10B0400021FA04F220EA020000EBD3705EEA430E1C
:10B0500008BF20EAD37070BD94F0000F0FD101F04B
:10B060000046400041EB010111F4801F08BF013C84
:10B07000F7D041EA060195F0000F18BF704703F0C2
:10B080000046520043EB030313F4801F08BF013D49
:10B09000F7D043EA0603704794EA0C0F0CEA135505
:10B0A00018BF95EA0C0F0CD050EA410618BF52EABF
:10B0B0004306D1D181EA030101F000414FF00000C5
:10B0C00070BD50EA410606BF1046194652EA4306D3
:10B0D00019D094EA0C0F02D150EA013613D195EA47
:10B0E0000C0F05D152EA03361CBF104619460AD18F
:10B0F00081EA030101F0004141F0FE4141F4700199
:10B100004FF0000070BD41F0FE4141F4780170BD88
:10B1100070B54FF0FF0C4CF4E06C1CEA11541DBFED
:10B120001CEA135594EA0C0F95EA0C0F00F0A7F8EF
:10B13000A4EB050481EA030E52EA03354FEA01311C
:10B1400000F088804FEA03334FF0805545EA13132F
:10B1500043EA12634FEA022245EA111545EA1065F7
:10B160004FEA00260EF000419D4208BF964244F18E
:10B17000FD0404F5407402D25B084FEA3202B61AAD
:10B1800065EB03055B084FEA32024FF480104FF481
:10B19000002CB6EB020E75EB030E22BFB61A7546F5
:10B1A00040EA0C005B084FEA3202B6EB020E75EB88
:10B1B000030E22BFB61A754640EA5C005B084FEAF0
:10B1C0003202B6EB020E75EB030E22BFB61A7546BD
:10B1D00040EA9C005B084FEA3202B6EB020E75EBC8
:10B1E000030E22BFB61A754640EADC0055EA060E89
:10B1F00018D04FEA051545EA16754FEA06164FEACC
:10B20000C30343EA52734FEAC2025FEA1C1CC0D177
:10B2100011F4801F0BD141EA00014FF000004FF004
:10B22000004CB6E711F4801F04BF01430020B4F1C5
:10B23000FD0C88BFBCF5E06F3FF6AFAEB5EB030C7D
:10B2400004BFB6EB020C5FEA500C50F1000041EB7A
:10B25000045170BD0EF0004E4EEA113114EB5C0447
:10B26000C2BFD4EB0C0541EA045170BD41F480111A
:10B270004FF0000E013C90E645EA060E8DE60CEA22
:10B28000135594EA0C0F08BF95EA0C0F3FF43BAF3F
:10B2900094EA0C0F0AD150EA01347FF434AF95EAF6
:10B2A0000C0F7FF425AF104619462CE795EA0C0FDA
:10B2B00006D152EA03353FF4FDAE1046194622E7A7
:10B2C00050EA410618BF52EA43067FF4C5AE50EA81
:10B2D00041047FF40DAF52EA43057FF4EBAE12E771
:10B2E0004FF0FF3C06E000BF4FF0010C02E000BF52
:10B2F0004FF0010C4DF804CD4FEA410C7FEA6C5C35
:10B300004FEA430C18BF7FEA6C5C1BD001B050EAD7
:10B31000410C0CBF52EA430C91EA030F02BF90EAC2
:10B32000020F0020704710F1000F91EA030F58BF81
:10B33000994208BF90422CBFD8176FEAE37040F0E3
:10B34000010070474FEA410C7FEA6C5C02D150EA81
:10B35000013C07D14FEA430C7FEA6C5CD6D152EA3C
:10B36000033CD3D05DF8040B704700BF8446104601
:10B3700062468C461946634600E000BF01B5FFF700
:10B38000B7FF002848BF10F1000F01BD4DF808EDD0
:10B39000FFF7F4FF0CBF012000205DF808FB00BFA1
:10B3A0004DF808EDFFF7EAFF34BF012000205DF8FB
:10B3B00008FB00BF4DF808EDFFF7E0FF94BF012048
:10B3C00000205DF808FB00BF4DF808EDFFF7CEFF49
:10B3D00094BF012000205DF808FB00BF4DF808ED88
:10B3E000FFF7C4FF34BF012000205DF808FB00BF59
:10B3F0004FEA410C7FEA6C5C02D150EA013C0AD171
:10B400004FEA430C7FEA6C5C02D152EA033C02D162
:10B410004FF0000070474FF0010070474FEA4102C3
:10B4200012F5001215D211D56FF47873B3EB625296
:10B4300012D94FEAC12343F0004343EA505311F0BD
:10B44000004F23FA02F018BF404270474FF000004F
:10B45000704750EA013005D111F0004008BF6FF08D
:10B46000004070474FF00000704700BF1FB51C46FA
:10B47000094B1B680546D86852B1084B0091CDE9CD
:10B48000013207492B46224600F028F800F0BAFDA9
:10B49000044B1A46F2E700BF60000020D0E5000030
:10B4A000DDE50000ABD10000014B1868704700BF1C
:10B4B0006000002008B5074B044613B10021AFF32C
:10B4C0000080054B1868836A03B19847204601F055
:10B4D00071FB00BF000000000CE600000EB403B5D5
:10B4E000014603AB054853F8042B0068019300F0B4
:10B4F00081F802B05DF804EB03B0704760000020F3
:10B5000070B50D4E0D4CA41BA4100025A54209D109
:10B510000B4E0C4C01F050FBA41BA4100025A542BF
:10B5200005D170BD56F8253098470135EEE756F83D
:10B53000253098470135F2E7300200203002002024
:10B54000300200204002002010B5431E0A44914200
:10B5500000D110BD11F8014B03F8014FF7E7884205
:10B5600010B501EB020307D8421E99420AD011F828
:10B57000014B02F8014FF8E78342F5D98118D21A3E
:10B58000D34200D110BD13F8014D01F8014DF7E78A
:10B5900002440346934200D1704703F8011BF9E7C8
:10B5A0009368013B002B10B4936008DA9469A342BE
:10B5B00001DB0A2903D15DF8044B00F063BC13687A
:10B5C000581C1060197008465DF8044B7047F8B5B8
:10B5D00006460F461446D518AC4201D1002007E0BC
:10B5E0003A4614F8011B3046FFF7DAFF431CF3D14B
:10B5F000F8BD00002DE9F04F9DB00C4617460393AF
:10B60000064618B183690BB900F0F4FD7B4B9C42F0
:10B6100057D17468A38918075DD52369002B5AD0C8
:10B620000023099320238DF8293030238DF82A3008
:10B630004FF0010BB846454615F8013B0BB1252BE1
:10B6400054D1B8EB070A0BD053463A462146304650
:10B65000FFF7BDFF013000F0C280099B53440993FE
:10B6600098F80030002B00F0BA8000234FF0FF3232
:10B67000CDE90523049307938DF853301A93A84618
:10B68000052218F8011B5E4800F0C2FE049B78BB3F
:10B69000D90644BF20228DF853201A0744BF2B221D
:10B6A0008DF853202A782A2A2AD0079AA846002003
:10B6B0000A25414611F8013B303B092B69D960B39B
:10B6C00024E0504B9C4201D1B468A3E74E4B9C420E
:10B6D00008BFF4689EE72146304600F025FC0028AC
:10B6E0009ED04FF0FF301DB0BDE8F08FA846A2E716
:10B6F000434A801A0BFA00F0184304904546BEE70F
:10B70000039A111D12680391002A01DB079204E0DD
:10B71000524243F002030792049398F800302E2B14
:10B720000ED198F801302A2B38D1039B1A1D1B68C3
:10B730000392002BB8BF4FF0FF3308F102080593C6
:10B74000324D98F800100322284600F061FE40B107
:10B750004023401B03FA00F0049B034308F1010857
:10B76000049398F800102A488DF82810062208F152
:10B77000010700F04DFE002837D0264B1BBB039B72
:10B78000073323F0070308330393099B4B440993C2
:10B7900050E705FB0232012088468AE7002308F1C2
:10B7A0000108059319460A25404610F8012B303A46
:10B7B000092A03D9002BC3D00591C1E705FB01215C
:10B7C00001238046F0E703AB00932246124B04A905
:10B7D0003046AFF30080B0F1FF3F8146D5D1A38959
:10B7E0005B063FF57EAF09987DE703AB00932246E9
:10B7F000094B04A9304600F087F8ECE764E6000046
:10B8000010E6000084E6000044E6000016E60000B2
:10B810001AE6000000000000CFB500002DE9F04757
:10B8200091461F468A680B69DDF820809342B8BFB5
:10B830001346C9F8003091F8432006460C4612B171
:10B840000133C9F800302368990642BFD9F80030A7
:10B850000233C9F80030256815F0060507D104F158
:10B86000190AE368D9F800209B1AAB4228DC94F847
:10B8700043302268003318BF012392062DD404F10F
:10B88000430239463046C047013020D02368E5687E
:10B89000D9F8002003F00603042B08BFAD1AA368F3
:10B8A00022690CBF25EAE57500259342C4BF9B1AA7
:10B8B000ED184FF000091A344D451AD1002008E068
:10B8C0000123524639463046C047013003D14FF07C
:10B8D000FF30BDE8F0870135C3E7E1185A1C30207E
:10B8E00081F84300224494F8451082F84310023353
:10B8F000C5E70123224639463046C0470130E6D02D
:10B9000009F10109D8E700002DE9F04301F1430CEA
:10B910000C46097E85B06E291746064698460C9A55
:10B9200000F0B38022D8632936D00AD8002900F06D
:10B93000B980582900F0838004F1420584F8421050
:10B9400032E0642901D06929F6D120681368050620
:10B9500003F104012AD51B681160002B03DA2D22A4
:10B960005B4284F843206F480A2239E0732900F0D3
:10B970009D8008D86F2920D07029DDD1236843F03D
:10B980002003236003E0752917D07829D4D17823C8
:10B9900084F84530644855E01368191D1B68116030
:10B9A00004F1420584F8423001238CE01B681160E9
:10B9B00010F0400F18BF1BB2CFE713682568181DA1
:10B9C0001060280601D51B6802E06806FBD51B88BD
:10B9D00054486F2914BF0A220822002184F843101A
:10B9E0006568A560002DC0F29580216821F00401F2
:10B9F0002160002B3DD1002D40F08E806546082A45
:10BA00000BD12368DB0708D5236962689A42DEBF41
:10BA1000302305F8013C05F1FF35ACEB050323614C
:10BA2000CDF800803B4603AA21463046FFF7F6FEDC
:10BA300001304DD14FF0FF3005B0BDE8F0833948FB
:10BA400084F84510136821681D1D1B6815600A06DF
:10BA50000BD5CA0744BF41F0200121601BB9226801
:10BA600022F0200222601022B7E74D0648BF9BB2A9
:10BA7000EFE76546B3FBF2F102FB1133C35C05F857
:10BA8000013D0B460029F5D1B9E7136825686169C6
:10BA9000181D106028061B6801D5196002E06A06AF
:10BAA000FBD51980002323616546B9E71368191D8A
:10BAB00011601D6862680021284600F0A9FC08B1E9
:10BAC000401B606063682361002384F84330A7E76C
:10BAD00023692A4639463046C0470130AAD0236838
:10BAE0009B0713D4E068039B9842B8BF1846A3E7AE
:10BAF00001234A4639463046C04701309AD00135C5
:10BB0000E368039A9B1AAB42F2DCEBE7002504F1F1
:10BB10001909F5E7002BACD1037884F8423004F121
:10BB200042056CE721E6000032E6000038B50D4B17
:10BB30001C68A36B05467BB9182000F04DFC0A4A2F
:10BB40000A4BA063C0E90023094B83600B23838168
:10BB500001220023C0E90423A36B00221D615A6166
:10BB600038BD00BF600000200E33CDAB34126DE64F
:10BB7000ECDE050038B5134B1C68A36B7BB91820AD
:10BB800000F02AFC104A114BA063C0E90023104BBF
:10BB900083600B23838101220023C0E90423A16B6E
:10BBA0000C480A694B690C4C504304FB0300A2FB90
:10BBB00004230344541C43F10005C1E9044525F066
:10BBC000004038BD600000200E33CDAB34126DE66E
:10BBD000ECDE05002DF451582D7F954C0CB430B59A
:10BBE000174B0C1E9DB01D6808DA8B232B604FF09D
:10BBF000FF301DB0BDE8304002B070474FF4027313
:10BC0000ADF8143014BF04F1FF33234604930793B7
:10BC10004FF6FF7302900690ADF81630209A21ABD4
:10BC200002A92846019300F06BFD431CBCBF8B2387
:10BC30002B60002CDDD0029B00221A70D9E700BFD8
:10BC4000600000200EB400B59CB01DAB02900690C1
:10BC50006FF00041094807910491094953F8042BFA
:10BC600005910068019302A900F04AFD029B0022A1
:10BC70001A701CB05DF804EB03B070476000002040
:10BC80000802FFFF10B503461A785C1C3AB9013B65
:10BC900011F8012B03F8012F002AF9D110BD23461A
:10BCA000F2E7C9B2034610F8012B1AB18A42F9D162
:10BCB00018467047002918BF0023F9E710F8012B38
:10BCC00011F8013B012A28BF9A42F7D0D01A7047D9
:10BCD000034613F8012B002AFBD1181A01387047CC
:10BCE00010B56AB10139841810F8013B11F8012F21
:10BCF000934203D1A04201D0002BF5D1981A10BD78
:10BD00001046FCE770B50139044602B970BD234600
:10BD100011F8015F03F8015B561E2DB91444A342CC
:10BD2000F4D003F8015BFAE71C463246EDE7F0B5C4
:10BD300003787BB1044623782046661C7BB14A1EFB
:10BD4000631E12F8015F4DB113F8017FAF42344614
:10BD5000F7D0F0E70B78002B18BF0020F0BD184695
:10BD6000FCE72DE9F0478046894692461E460F467D
:10BD70003D46089815F8014B00F0C6FA2044437878
:10BD800013F0080332D12D2C32D17C78BD1C012256
:10BD9000002E5DD0102E09D1302C07D12B7803F066
:10BDA000DF03582B4FD16C7810260235002A14BFC0
:10BDB0004FF000416FF000410027B1FBF6FC384620
:10BDC00006FB1C1EA4F13003092B17D81C46A64203
:10BDD00023DD7B1C07D084451CD301D1A64519DB8C
:10BDE00000FB0640012715F8014BEBE72F46BFE7A4
:10BDF0002B2C04BFBD1C7C781A46C9E7A4F1410373
:10BE0000192B01D8373CE2E7A4F16103192B04D8C0
:10BE1000573CDCE74FF0FF37E5E77B1C08D12223D6
:10BE2000C8F800300846BAF1000F07D1BDE8F08726
:10BE300002B14042BAF1000FF8D00FB105F1FF395D
:10BE4000CAF80090F2E73024002EAFD10826ADE703
:10BE5000302CA3D00A26A9E7084B37B51C68084D3B
:10BE6000236A002B08BF2B46009313460A4601465F
:10BE70002046FFF776FF03B030BD00BF6000002012
:10BE8000C4000020F8B50E461446054618B1836973
:10BE90000BB900F0AFF9214B9C422AD16C68A36921
:10BEA000A360A3891A072ED5236963B32369206889
:10BEB000C01A6369F6B28342374604DC214628463D
:10BEC00000F02EF928BBA368013BA36023685A1C2D
:10BED00022601E7063690130834204D0A389DB07AE
:10BEE00019D50A2E17D12146284600F019F990B12C
:10BEF0000FE00B4B9C4201D1AC68D0E7094B9C4250
:10BF000008BFEC68CBE72146284600F00DF8002872
:10BF1000CCD04FF0FF373846F8BD00BF64E60000D4
:10BF200084E6000044E60000324B70B51D6806460A
:10BF30000C4625B1AB6913B9284600F05BF92E4BCE
:10BF40009C420FD16C68B4F90C309AB215072CD40E
:10BF5000D00611D40922326043F04003A3814FF090
:10BF6000FF303EE0254B9C4201D1AC68EBE7244B0F
:10BF70009C4208BFEC68E6E7510712D5616B41B1FE
:10BF800004F14403994202D0304600F091FA0023B4
:10BF90006363A38923F02403A381002363602369DF
:10BFA0002360A38943F00803A38123694BB9A389C4
:10BFB00003F42073B3F5007F03D02146304600F030
:10BFC000CBF9A28912F001030CD00023A3606369AE
:10BFD0005B42A361236953B9B4F90C3013F08000BC
:10BFE000BAD170BD920758BF6369A360F2E7002021
:10BFF000F7E700BF6000002064E6000084E6000070
:10C0000044E6000008B5062000F0A8FC012000F07E
:10C01000D1FD00008A892DE9F041054610070C4644
:10C0200058D44B68002B05DC0B6C002B02DC002085
:10C03000BDE8F081E66A002EF9D0002312F48052A8
:10C040002F68216A2B6032D0606DA3895A0705D50D
:10C050006368C01A636B0BB1236CC01A00230246DD
:10C06000E66A216A2846B047431CA38906D129689D
:10C070001D2948D8294ACA40D60744D50022626003
:10C08000D9042269226004D5421C01D12B6803B96E
:10C090006065616B2F600029C9D004F144039942A7
:10C0A00002D0284600F004FA00206063C0E70123B4
:10C0B0002846B047411CC8D12B68002BC5D01D2B8A
:10C0C00001D0162B01D12F60B1E7A38943F04003C3
:10C0D000A381ADE70F69002FA9D093070E6808BFB1
:10C0E0004B690F6018BF0023A6EB07088B60B8F1FF
:10C0F000000F9CDD43463A46216AA66A2846B047AF
:10C10000002806DCA38943F04003A3814FF0FF30F1
:10C110008EE70744A8EB0008E9E700BF01004020D4
:10C1200038B50B6905460C46DBB118B183690BB90C
:10C1300000F060F80C4B9C4209D16C68B4F90C30EB
:10C140007BB121462846BDE83840FFF763BF074B67
:10C150009C4201D1AC68F1E7054B9C4208BFEC68FA
:10C16000ECE7002038BD00BF64E6000084E6000074
:10C1700044E60000002310B50446C0E900338360A4
:10C1800081814366C281C0E9043383611946082274
:10C190005C30FFF7FDF9054B6362054BA362054B6D
:10C1A000E362054B2462236310BD00BF95C9000004
:10C1B000B7C90000EFC9000013CA0000014900F030
:10C1C00085B800BF21C1000070B54A1E68255543DF
:10C1D0000E4605F1740100F0B9F9044640B10021A2
:10C1E000C0E900160C30A06005F16802FFF7D0F935
:10C1F000204670BD836910B5044633BBC0E91233D5
:10C200000365124B124A1B688262984204BF0123E5
:10C21000836100F01FF86060204600F01BF8A0600A
:10C22000204600F017F80022E06004216068FFF764
:10C23000A1FF01220921A068FFF79CFF0222122121
:10C24000E068FFF797FF0123A36110BD0CE6000033
:10C25000BDC10000F8B51B4B1E68B369074613B992
:10C260003046FFF7C7FF4836D6E90134013B03D516
:10C27000336833B13668F7E7B4F90C506DB1683400
:10C28000F4E704213846FFF79FFF30600028F1D122
:10C290000C233B6004462046F8BD0B4B6566C4E9A1
:10C2A0000055A560C4E90335C4E9055508222946AF
:10C2B00004F15C00FFF76CF9C4E90D55C4E91255AF
:10C2C000E9E700BF0CE600000100FFFF2DE9F8439D
:10C2D0008046894600F14804002614B93046BDE87E
:10C2E000F883D4E90175013F01D52468F5E7AB89EE
:10C2F000012B07D9B5F90E30013303D0294640464A
:10C30000C84706436835EEE7D0F8EC00704770B5D3
:10C310000E46B1F90E10002996B014461D4607DAF4
:10C3200000232B60B3891A0610D44FF480630EE00B
:10C330006A4600F0A1FB0028F2DB019A02F4704289
:10C34000A2F500535A425A412A60EEE740230020EA
:10C35000236016B070BD00008B8973B59D0706463B
:10C360000C4607D504F14703236023610123636171
:10C3700002B070BD01AB6A46FFF7C9FF00990546E0
:10C38000304600F0E3F848B9B4F90C309A05EFD420
:10C3900023F0030343F00203A381E3E70D4BB362F1
:10C3A000A389206043F08003A381009B6361019B0C
:10C3B00020615BB1B4F90E10304600F06FFB28B17C
:10C3C000A38923F0030343F00103A381A3891D4341
:10C3D000A581CDE7BDC10000024B0146186800F001
:10C3E000B5B800BF6000002082B001B901A942B118
:10C3F0004BB113780B601278101C18BF012002B0EB
:10C4000070471046FBE76FF00100F8E700000000FE
:10C4100001F0FF01102A2BDB10F0070F08D010F8F5
:10C42000013B013A8B422DD010F0070F42B3F6D1F9
:10C43000F0B441EA012141EA014122F007047FF012
:10C4400000070023F0E80256083C85EA010586EA69
:10C45000010685FA47F5A3FA87F586FA47F6A5FAA5
:10C4600087F68EB9EED1F0BC01F0FF0102F00702B1
:10C4700032B110F8013B013A83EA010313B1F8D15C
:10C480000020704701387047002D06BF354603383D
:10C49000073815F0010F07D1013015F4807F02BF76
:10C4A000013015F4C03F0130F0BC0138704700BFC7
:10C4B00038B50546002945D051F8043C0C1F002B27
:10C4C000B8BFE41800F00CFB1F4A1368104633B9DC
:10C4D000636014602846BDE8384000F002BBA34208
:10C4E0000CD921686218934204BF1A685B686360C4
:10C4F00004BF521822600460ECE713465A680AB180
:10C50000A242FAD919685818A0420BD120680144F8
:10C51000581882421960DDD1106852685A6001448F
:10C520001960D7E702D90C232B60D3E720682118C4
:10C530008A4204BF11685268626004BF0918216012
:10C540005C60C7E738BD00BF047D012070B5CD1C1D
:10C5500025F0030508350C2D38BF0C25002D0646A7
:10C5600001DBA94203D90C233360002070BD00F029
:10C57000B7FA214A1468214691B9204C23681BB9A7
:10C58000304600F0B3F920602946304600F0AEF99D
:10C59000431C24D10C233360304600F0A2FAE4E7B8
:10C5A0000B685B1B18D40B2B0FD90B60CD50CC182C
:10C5B000304600F096FA04F10B00231D20F007002E
:10C5C000C31AD3D05A42E250D0E78C424B6816BF10
:10C5D000636013600C46EBE70C464968CCE7C41C6B
:10C5E00024F00304A04205D0211A304600F07EF961
:10C5F0000130CFD02560DBE7047D0120087D0120DC
:10C60000F8B5074614460E4621B91146BDE8F84074
:10C61000FFF79CBF22B9FFF74BFF25462846F8BD20
:10C6200000F060FAA0420FD221463846FFF78EFF95
:10C6300005460028F2D031462246FEF785FF3146F6
:10C640003846FFF735FFE9E73546E7E72DE9F047DC
:10C650008E689E4282460C469046994637D88A8913
:10C6600012F4906F31D0256809696F1A6569022349
:10C6700005EB450595FBF3F509F101033B449D42AC
:10C6800038BF1D46530530D52946FFF75FFF0646E4
:10C6900050B90C23CAF80030A38943F04003A381AA
:10C6A0004FF0FF30BDE8F0873A462169FEF74CFFB6
:10C6B000A38923F4906343F08003A381266165611D
:10C6C0003E44ED1B2660A5604E464E4500D94E46C1
:10C6D000324641462068FEF742FFA3689B1BA360D9
:10C6E00023681E4426600020DCE72A46FFF788FF07
:10C6F00006460028E2D121695046FFF7D9FEC8E777
:10C700002DE9F04F9DB0804603938B891D060C46A2
:10C7100016460FD50B696BB94021FFF717FF206054
:10C72000206128B90C23C8F800304FF0FF30C7E073
:10C73000402363610023099320238DF8293030239F
:10C740008DF82A304FF0010B37463D4615F8013B76
:10C750000BB1252B3ED1B7EB060A0BD05346324620
:10C7600021464046FFF772FF013000F0A480099B8C
:10C77000534409933B78002B00F09D8000234FF039
:10C78000FF32CDE90523049307938DF853301A93B4
:10C790002F46052217F8011B4F48FFF739FE049B6F
:10C7A000D0B9D90644BF20228DF853201A0744BFC0
:10C7B0002B228DF853202A782A2A15D0079A2F4643
:10C7C00000200A25394611F8013B303B092B4DD991
:10C7D000B8B10FE02F46B8E73F4A801A0BFA00F0D5
:10C7E000184304903D46D3E7039A111D1268039144
:10C7F000002A01DB079204E0524243F00203079251
:10C8000004933B782E2B0CD17B782A2B33D1039BBE
:10C810001A1D1B680392002BB8BF4FF0FF3302377D
:10C8200005932E4D397803222846FFF7F1FD38B1E4
:10C830004023401B03FA00F0049B03430137049399
:10C84000397827488DF8281006227E1CFFF7E0FD76
:10C85000002838D0234B13BB039B073323F0070377
:10C8600008330393099B4B4409936DE705FB0232A0
:10C8700001200F46A6E700230137059319460A2534
:10C88000384610F8012B303A092A03D9002BC8D0BA
:10C890000591C6E705FB012101230746F0E703AB3D
:10C8A00000932246104B04A94046AFF30080B0F13C
:10C8B000FF3F8146D6D1A3895B063FF536AF099885
:10C8C0001DB0BDE8F08F03AB00932246064B04A9D0
:10C8D0004046FFF719F8EAE710E6000016E6000008
:10C8E0001AE60000000000004DC6000038B5064CF6
:10C8F000002305460846236000F046F9431C02D198
:10C90000236803B12B6038BD989001201F2938B5EA
:10C9100004460D4604D9162303604FF0FF3038BD9E
:10C92000426C12B152F821304BB9204600F030F879
:10C930002A4601462046BDE8384000F017B8012BD2
:10C940000AD0591C03D1162303600120E7E7002415
:10C9500042F82540284698470020E0E7024B014670
:10C960001868FFF7D3BF00BF6000002038B5074C40
:10C970000023054608461146236000F0EDF8431CED
:10C9800002D1236803B12B6038BD00BF989001200D
:10C9900000F0D2B810B50C46B1F90E1000F0AAF8AC
:10C9A0000028ABBF636DA3891B1823F48053ACBF71
:10C9B0006365A38110BD2DE9F0411F468B89DB051E
:10C9C00005460C46164605D502230022B1F90E1085
:10C9D00000F074F8A389B4F90E1023F48053A381F6
:10C9E00032463B462846BDE8F04100F023B810B57A
:10C9F0000C46B1F90E1000F061F8431CA38915BF75
:10CA0000606523F4805343F48053A38118BFA3814E
:10CA100010BDB1F90E1000F01FB849B1FF2A85BF53
:10CA20008A2303600A704FF0FF3098BF01207047DF
:10CA30000846704738B5074C05460846114600229F
:10CA400022601A4600F0AEF8431C02D1236803B1FD
:10CA50002B6038BD9890012038B5064C0023054660
:10CA60000846236000F058F8431C02D1236803B144
:10CA70002B6038BD9890012038B5074C002305463F
:10CA800008461146236000F04FF8431C02D123688A
:10CA900003B12B6038BD00BF9890012038B5064C1B
:10CAA000002305460846236000F04EF8431C02D1DF
:10CAB000236803B12B6038BD9890012038B5074C2E
:10CAC000054608461146002222601A4600F04CF83E
:10CAD000431C02D1236803B12B6038BD989001201C
:10CAE0007047704751F8043C181F002BBCBF0B580F
:10CAF000C018704738B5074C054608461146002255
:10CB000022601A4600F038F8431C02D1236803B1B2
:10CB10002B6038BD98900120024B58221A604FF0CC
:10CB2000FF30704798900120024B58221A604FF056
:10CB3000FF30704798900120024B58221A604FF046
:10CB4000FF30704798900120024B58221A60002055
:10CB5000704700BF98900120024B58221A604FF096
:10CB6000FF30704798900120024B58221A604FF016
:10CB7000FF30704798900120024B58221A604FF006
:10CB8000FF30704798900120044A05491368002B34
:10CB900008BF0B4618441060184670470C7D0120F2
:10CBA000A0900120024B58221A604FF0FF307047CE
:10CBB00098900120FEE700BFF8B500BFF8BC08BCA4
:10CBC0009E467047F8B500BFF8BC08BC9E4670474B
:10CBD00064617461000000006CCC00001D03000063
:10CBE00075CC0000CD0B00007BCC00000D040000D4
:10CBF00083CC0000890C00008ACC0000B50D000039
:10CC00008FCC00001906000095CC0000F107000051
:10CC1000A0CC000077040000A5CC0000F10F0000BC
:10CC2000B1CC00004F030000BBCC0000F90A0000AB
:10CC3000C9CC000095070000D6CC00007D0900009B
:10CC4000E2CC00005D07000072616E646F6D0061F0
:10CC50006C6C006C6173740066616C736500747257
:10CC6000756500252E3135732E2E2E006D616B6596
:10CC70004C6973740072616E6765006164644C6135
:10CC800073740064656C657465006A6F696E007327
:10CC9000706C697400636F707946726F6D546F00C9
:10CCA00066696E64006A6F696E537472696E677349
:10CCB00000756E69636F6465417400756E69636FBA
:10CCC0006465537472696E67006E65774279746546
:10CCD0004172726179006173427974654172726167
:10CCE0007900667265654D656D6F727900000000B0
:10CCF0005DCD0000D114000062CD0000EB140000F7
:10CD000083CC0000EF14000068CD0000D5140000B3
:10CD100072CD0000F31400007BCD0000F71400007A
:10CD200085CD0000FB1400008ECD0000FF14000034
:10CD300099CD000003150000A5CD0000D914000016
:10CD4000AECD0000E3140000B8CD0000DD140000FB
:10CD5000C3CD0000E714000066696C65006F706564
:10CD60006E00636C6F736500656E644F6646696C38
:10CD70006500726561644C696E650072656164424C
:10CD8000797465730072656164496E746F006170D7
:10CD900070656E644C696E6500617070656E6442AA
:10CDA000797465730066696C6553697A650073749C
:10CDB0006172744C697374006E657874496E4C6965
:10CDC00073740073797374656D496E666F0000004B
:10CDD000F418000004190000181900008C19000054
:10CDE000BE190000EE190000201A0000421A0000CF
:10CDF000821A0000BC1A00000C1B00004A1B000035
:10CE0000AA1B0000EA1B00000A1C00003E1C0000D8
:10CE10007E1C0000A01C0000CA1C0000F41C0000C6
:10CE2000D8320000B81D0000801E0000F21E000075
:10CE30003C1F0000A01F0000BC1F0000DA1F000004
:10CE40001821000058210000CA210000F82100002C
:10CE50002822000056220000BA2200001E230000F3
:10CE600080230000E223000056240000D0240000AC
:10CE70003025000090250000C62500000A2600008D
:10CE80005026000096260000E82600003E270000FD
:10CE90007C2700000C2800004028000086280000A5
:10CEA000CC280000122900004C2900009229000023
:10CEB000D8290000342B0000CA1C00003E1C0000D2
:10CEC0004C2A0000F4180000802A0000A62A000066
:10CED000DA2A0000002B0000F4180000F41800000B
:10CEE000F4180000F4180000AA2B0000E62B000044
:10CEF000262C0000762C00009C2C00000A2D00003F
:10CF0000542D0000842D0000F4180000F4180000D7
:10CF1000A22D0000D42D0000062E00003A2E0000A5
:10CF20005E2E0000BC2E0000E02E0000022F00004C
:10CF3000242F0000562F0000882F0000AC2F000087
:10CF4000D02F00000230000026300000F41800004E
:10CF5000F4180000F4180000F4180000F4180000A1
:10CF6000583000007E300000A4300000CA300000BD
:10CF7000F030000024310000583100008C310000F6
:10CF8000C0310000E63100000C32000040320000E9
:10CF9000F4180000F4180000F4180000F418000061
:10CFA000F4180000F4180000F4180000F418000051
:10CFB000F4180000F4180000F4180000F418000041
:10CFC000663200006632000092330000C233000077
:10CFD0005B2564206974656D206C6973745D00283D
:10CFE00025642062797465732900286F626A65631D
:10CFF0007420747970653A20256429005374616344
:10D000006B20756E646572666C6F7700626F6F6C13
:10D0100065616E006E756D62657200737472696E23
:10D0200067006C6973740062797465206172726163
:10D03000790000000700000003000000CDD00000D0
:10D04000E1340000D5D000008D350000DED00000B6
:10D05000793D0000E7D00000E5340000F0D000008A
:10D060007D3D0000F8D000002137000001D1000014
:10D07000D53700000FD100006D3600001AD1000036
:10D08000E93E000025D100003137000030D100001A
:10D09000AD3E00003CD100001936000048D1000030
:10D0A000034000000000000001000000020000003A
:10D0B00003000000040000000A0000001D00000042
:10D0C0006D6963726F3A62697420763200686173C9
:10D0D000546F6E6500706C6179546F6E65006861A5
:10D0E00073536572766F00736574536572766F0063
:10D0F000646163496E697400646163577269746541
:10D1000000736F6674577269746542797465007351
:10D1100071756172655761766500736574557365E5
:10D12000724C454400616E616C6F675265616400CA
:10D13000616E616C6F6757726974650064696769D5
:10D1400074616C52656164006469676974616C57ED
:10D150007269746500474320746F6F6B20256420EB
:10D1600075736563733B206672656520256420775F
:10D170006F726473003C496E74656765723E003C73
:10D180004C6973743E003C4F626A6563743E003CB8
:10D190004279746541727261793E000D0A564D20E4
:10D1A00050616E69633A2025730D0A006D697363DF
:10D1B00000000000F9D10000274A000002D2000060
:10D1C000F54A00000AD20000B14A00000ED2000069
:10D1D000651800001DD200007549000025D200002E
:10D1E000174900002FD20000A94800003BD20000E0
:10D1F000AB4700006E756C6C00686578546F496EC3
:10D20000740072657363616C650073696E006272AD
:10D210006F616463617374546F494445006A736F4E
:10D220006E476574006A736F6E436F756E74006A43
:10D23000736F6E56616C75654174006A736F6E4BE7
:10D2400065794174000000003CD30000654B00008C
:10D2500044D30000694B00004ED300007B4B00001C
:10D2600057D30000814B000062D30000874B0000C1
:10D270006ED300008D4B00007CD30000934B000068
:10D2800084D30000994B00008AD300009F4B00001C
:10D290009FD30000A54B0000B4D30000AB4B0000AF
:10D2A000C0D30000B14B0000D0D30000B74B00004A
:10D2B000DCD30000BD4B0000E9D30000C34B0000ED
:10D2C000F2D30000C94B0000FAD30000CF4B00009E
:10D2D00008D40000D54B000019D40000DB4B00003F
:10D2E0002CD40000E14B00003AD40000E74B0000D2
:10D2F00049D40000ED4B00005CD40000F34B00006B
:10D3000072D40000F94B00007ED40000FF4B0000F7
:10D310008ED40000054C00009DD400000B4C000092
:10D32000ABD40000114C0000B3D400006F4B0000E0
:10D33000BBD40000754B00006E65740068617357C4
:10D340006946690073746172745769466900737441
:10D350006F705769466900776966695374617475BF
:10D3600073006D794950416464726573730073741E
:10D37000617274535349447363616E0067657453FB
:10D38000534944006D794D4143006874747053658E
:10D390007276657247657452657175657374007253
:10D3A0006573706F6E64546F4874747052657175F4
:10D3B0006573740068747470436F6E6E6563740097
:10D3C000687474704973436F6E6E6563746564004E
:10D3D00068747470526571756573740068747470E4
:10D3E000526573706F6E736500756470537461720B
:10D3F000740075647053746F700075647053656E5B
:10D40000645061636B65740075647052656365692F
:10D4100076655061636B65740075647052656D6FFD
:10D420007465495041646472657373007564705229
:10D43000656D6F7465506F727400776562536F63CA
:10D440006B6574537461727400776562536F636BBC
:10D4500065744C6173744576656E740077656253CC
:10D460006F636B657453656E64546F436C69656E6E
:10D4700074004D515454436F6E6E656374004D518A
:10D4800054544973436F6E6E6563746564004D5107
:10D490005454446973636F6E6E656374004D5154E8
:10D4A000544C6173744576656E74004D51545450FC
:10D4B0007562004D515454537562004D515454558A
:10D4C0006E7375620000000004000000030000009D
:10D4D0000A00000007000000060000000000000035
:10D4E0000008080800080A4A4000000A5FEA5FEAEC
:10D4F0000ED92ED36E19324489330C924C924D08BA
:10D500000800000004880808040804848488000ACD
:10D51000448A4000048EC480000000048800000E8D
:10D52000C000000000080001224488100C925252F2
:10D530004C048C84848E1C824C901E1EC244924CDF
:10D5400006CA525FE21FF01EC13E02448ED12E1F5A
:10D55000E24488100ED12ED12E0ED12EC4880008A0
:10D5600000080000048004880244880482000EC081
:10D570000EC008048244880ED126C0040ED135B3F3
:10D580006C0C925ED2521C925C925C0ED010100E0B
:10D590001C9252525C1ED01C901E1ED01C90100E6D
:10D5A000D013712E12525ED2521C8808081C1FE242
:10D5B00042524C1254981492101010101E113B75C8
:10D5C000B131113935B3710C9252524C1C925C90AE
:10D5D000100C92524C861C925C92510ED00C825CC4
:10D5E0001FE4848484125252524C1131312A441166
:10D5F0003135BB7112524C9252112A4484841EC49C
:10D6000088101E0EC808080E10080482410EC2427F
:10D61000424E048A400000000000001F0804800001
:10D6200000000ED2524F10101C925C000ED0100E53
:10D6300002424ED24E0C925C900E06C81C88080E18
:10D64000D24EC24C10101C9252080008080802402A
:10D6500002424C10149814920808080806001B7522
:10D66000B131001C925252000C92524C001C925C40
:10D6700090000ED24EC2000ED010100006C80498C2
:10D6800008080EC807001252524F0011312A4400F8
:10D69000113135BB00124C8C9200112A4498001EA7
:10D6A000C4881E06C48C8486080808080818080C5C
:10D6B000881800000C8360000000000001000000DA
:10D6C000020000000300000004000000050000004C
:10D6D000060000000700000008000000090000002C
:10D6E0000A0000000B0000000C0000000D0000000C
:10D6F0000E0000000F0000001000000012000000EB
:10D700001400000016000000180000001A000000BD
:10D710001C0000001E00000020000000230000008C
:10D7200026000000290000002C0000002F0000004F
:10D7300032000000360000003A0000003E00000009
:10D7400042000000460000004B00000050000000B6
:10D75000550000005A000000610000006800000051
:10D760006F000000760000007D00000084000000D3
:10D770008B0000009200000099000000A000000053
:10D78000A7000000AE000000B5000000BC000000D3
:10D79000C3000000CA000000D1000000D800000053
:10D7A000DF000000E6000000ED000000F4000000D3
:10D7B000FB000000FF00000000000000020000006D
:10D7C00004000000010000000300000038D8000041
:10D7D0002D4C000043D800008D5200004DD80000B1
:10D7E000594E00005AD800000150000061D80000D6
:10D7F0004D5000006AD800009D50000076D800000F
:10D80000914F000087D800001D4F000097D80000FE
:10D8100095510000A4D80000E54E0000150000005E
:10D82000160000001700000018000000190000009A
:10D83000646973706C6179006C696768744C6576B3
:10D84000656C006D62446973706C6179006D62444F
:10D850006973706C61794F6666006D62506C6F74AD
:10D86000006D62556E706C6F74006D62447261770A
:10D870005368617065006D625368617065466F72D0
:10D880004C6574746572006D62456E61626C6544CE
:10D890006973706C6179006E656F506978656C535F
:10D8A000656E64006E656F506978656C5365745081
:10D8B000696E004E6F7420656E6F75676820726FB9
:10D8C0006F6D206576656E20616674657220636F8A
:10D8D0006D70616374696F6E00436F6D7061637426
:10D8E000656420466C61736820636F64652073749F
:10D8F0006F72650A2564206279746573207573659B
:10D900006420282564252529206F6620256400428F
:10D910006164207265636F726420666F756E642047
:10D92000647572696E6720696E697469616C697A81
:10D930006174696F6E0025642025642025642028A9
:10D94000256420776F7264732900256420726563F3
:10D950006F7264732C20256420776F7264732C209F
:10D960006D617849442025642C20636F6D7061637C
:10D9700074696F6E206379636C657320256400524F
:10D980006573746F726564202564207363726970B7
:10D990007473005374617274656400726164696FBA
:10D9A0000000000039DA00005D5A000046DA00008D
:10D9B000315D000056DA0000C55C000064DA00004A
:10D9C000915E00006FDA0000755A00007FDA0000F7
:10D9D000F95A000093DA0000DD5A0000A2DA0000D4
:10D9E0003B600000AEDA0000B75F0000B7DA00006D
:10D9F0005B5F0000C2DA0000DD5E0000CDDA0000EF
:10DA0000155F0000D6DA0000455F0000DFDA000095
:10DA1000855A0000EEDA0000B95A0000F7DA00007B
:10DA2000955A000025303878006E6F6E65006F746F
:10DA300068657200706169720064697361626C6527
:10DA4000526164696F006D657373616765526563E8
:10DA50006569766564007061636B657452656365C2
:10DA6000697665007061636B657453656E640072FE
:10DA700065636569766564496E7465676572007291
:10DA8000656365697665644D65737361676554792F
:10DA90007065007265636569766564537472696E5A
:10DAA000670073656E64496E7465676572007365BF
:10DAB0006E64506169720073656E64537472696E4E
:10DAC00067007365744368616E6E656C007365749E
:10DAD00047726F757000736574506F77657200736D
:10DAE00069676E616C537472656E67746800646513
:10DAF000766963654944006C6173744D6573736145
:10DB00006765494400556E6B6E6F776E2070726961
:10DB10006D6974697665205B25733A25735D000035
:10DB200000000000963007772C610EEEBA5109997B
:10DB300019C46D078FF46A7035A563E9A395649ED7
:10DB40003288DB0EA4B8DC791EE9D5E088D9D297FB
:10DB50002B4CB609BD7CB17E072DB8E7911DBF9057
:10DB60006410B71DF220B06A4871B9F3DE41BE847B
:10DB70007DD4DA1AEBE4DD6D51B5D4F4C785D383D7
:10DB800056986C13C0A86B647AF962FDECC9658A7B
:10DB90004F5C0114D96C0663633D0FFAF50D088DD7
:10DBA000C8206E3B5E10694CE44160D5727167A27B
:10DBB000D1E4033C47D4044BFD850DD26BB50AA5D7
:10DBC000FAA8B5356C98B242D6C9BBDB40F9BCACFB
:10DBD000E36CD832755CDF45CF0DD6DC593DD1AB57
:10DBE000AC30D9263A00DE518051D7C81661D0BF7B
:10DBF000B5F4B42123C4B3569995BACF0FA5BDB8D7
:10DC00009EB802280888055FB2D90CC624E90BB17A
:10DC1000877C6F2F114C6858AB1D61C13D2D66B6D6
:10DC20009041DC760671DB01BC20D2982A10D5EF3A
:10DC30008985B1711FB5B606A5E4BF9F33D4B8E896
:10DC4000A2C9077834F9000F8EA8099618980EE13A
:10DC5000BB0D6A7F2D3D6D08976C6491015C63E696
:10DC6000F4516B6B62616C1CD83065854E0062F2BA
:10DC7000ED95066C7BA5011BC1F4088257C40FF516
:10DC8000C6D9B06550E9B712EAB8BE8B7C88B9FC3A
:10DC9000DF1DDD62492DDA15F37CD38C654CD4FB96
:10DCA0005861B24DCE51B53A7400BCA3E230BBD43A
:10DCB00041A5DF4AD795D83D6DC4D1A4FBF4D6D396
:10DCC0006AE96943FCD96E34468867ADD0B860DA3A
:10DCD000732D0444E51D03335F4C0AAAC97C0DDD96
:10DCE0003C710550AA41022710100BBE86200CC9BA
:10DCF00025B56857B3856F2009D466B99FE461CE16
:10DD00000EF9DE5E98C9D9292298D0B0B4A8D7C739
:10DD1000173DB359810DB42E3B5CBDB7AD6CBAC095
:10DD20002083B8EDB6B3BF9A0CE2B6039AD2B174B1
:10DD30003947D5EAAF77D29D1526DB048316DC730D
:10DD4000120B63E3843B64943E6A6D0DA85A6A7AB1
:10DD50000BCF0EE49DFF099327AE000AB19E077D0D
:10DD600044930FF0D2A3088768F2011EFEC2066931
:10DD70005D5762F7CB67658071366C19E7066B6E8D
:10DD8000761BD4FEE02BD3895A7ADA10CC4ADD67B1
:10DD90006FDFB9F9F9EFBE8E43BEB717D58EB0600D
:10DDA000E8A3D6D67E93D1A1C4C2D83852F2DF4FB1
:10DDB000F167BBD16757BCA6DD06B53F4B36B2480D
:10DDC000DA2B0DD84C1B0AAFF64A0336607A0441B1
:10DDD000C3EF60DF55DF67A8EF8E6E3179BE69460D
:10DDE0008CB361CB1A8366BCA0D26F2536E2685231
:10DDF00095770CCC03470BBBB91602222F2605558D
:10DE0000BE3BBAC5280BBDB2925AB42B046AB35CB0
:10DE1000A7FFD7C231CFD0B58B9ED92C1DAEDE5B0C
:10DE2000B0C2649B26F263EC9CA36A750A936D02F0
:10DE3000A906099C3F360EEB85670772135700054C
:10DE4000824ABF95147AB8E2AE2BB17B381BB60C70
:10DE50009B8ED2920DBED5E5B7EFDC7C21DFDB0BCC
:10DE6000D4D2D38642E2D4F1F8B3DD686E83DA1FF0
:10DE7000CD16BE815B26B9F6E177B06F7747B7184C
:10DE8000E65A0888706A0FFFCA3B06665C0B0111F0
:10DE9000FF9E658F69AE62F8D3FF6B6145CF6C164C
:10DEA00078E20AA0EED20DD75483044EC2B30339F0
:10DEB000612667A7F71660D04D476949DB776E3E4C
:10DEC0004A6AD1AEDC5AD6D9660BDF40F03BD83770
:10DED00053AEBCA9C59EBBDE7FCFB247E9FFB530CC
:10DEE0001CF2BDBD8AC2BACA3093B353A6A3B424F0
:10DEF0000536D0BA9306D7CD2957DE54BF67D9234C
:10DF00002E7A66B3B84A61C4021B685D942B6F2AEF
:10DF100037BE0BB4A18E0CC31BDF055A8DEF022D4B
:10DF2000416C6C207461736B732073746F707065D7
:10DF300064007631373000202573202573004D654D
:10DF40006D6F727920636C6561726564004E6F203D
:10DF500066726565207461736B20656E74726965A5
:10DF600073000000E4DF0000C57A0000F1DF00006C
:10DF700099720000FDDF0000957A000003E00000C8
:10DF8000A57A000009E00000B57A00000FE000006B
:10DF90006D79000025E00000C17B000033E0000047
:10DFA000C97200003DE00000517C000045E0000027
:10DFB000417700004EE00000197400005FE00000AF
:10DFC0000D7500006BE00000D173000074E00000EC
:10DFD000497400007CE000006176000073656E7398
:10DFE0006F727300616363656C65726174696F6EF3
:10DFF0000074656D70657261747572650074696C2A
:10E0000074580074696C74590074696C745A0073A4
:10E010006574416363656C65726F6D65746572529A
:10E02000616E6765006D61676E65746963466965F9
:10E030006C6400746F756368526561640069326373
:10E0400052656164006932635772697465006932B0
:10E0500063536574436C6F636B53706565640073E1
:10E06000706945786368616E6765007370695365B0
:10E070007475700072656164444854006D69637220
:10E080006F70686F6E6500005DCD0000D57E00008A
:10E0900062CD0000D17F0000BFE00000F57F0000EE
:10E0A00085CD0000597E0000C4E0000075800000AE
:10E0B000CAE000002D7D000073657269616C00721A
:10E0C000656164007772697465007772697465428E
:10E0D000797465730000000054E1000011810000B4
:10E0E00062E10000218100006FE100001581000065
:10E0F00078E100002581000082E100002981000014
:10E100008BE100002D81000090E1000031810000D2
:10E1100095E1000035810000A1E100003981000097
:10E12000A8E100003D810000B1E100004181000054
:10E13000B6E1000045810000C1E100004981000016
:10E14000CBE1000019810000D5E100001D81000035
:10E1500074667400656E61626C65446973706C61AD
:10E1600079007365744261636B6C696768740067FA
:10E1700065745769647468006765744865696768A1
:10E180007400736574506978656C006C696E650025
:10E190007265637400726F756E6465645265637452
:10E1A00000636972636C6500747269616E676C65A7
:10E1B000007465787400746674546F756368656480
:10E1C00000746674546F7563685800746674546F95
:10E1D0007563685900746674546F7563685072652E
:10E1E0007373757265007661727300000CE2000053
:10E1F000B185000016E20000918500001FE20000DA
:10E200006D8500002BE20000FD8400007661724500
:10E210007869737473007661724E616D6564007322
:10E2200065745661724E616D6564007661724E610F
:10E230006D65466F72496E6465780057656C636FF3
:10E240006D6520746F204D6963726F426C6F636BF4
:10E25000732100705F73706920213D204E554C4C36
:10E26000002F686F6D652F6769742F2E706C617455
:10E27000666F726D696F2F7061636B616765732F75
:10E280006672616D65776F726B2D61726475696E10
:10E290006F6E6F726469636E7266352F6C6962723D
:10E2A00061726965732F5350492F5350492E637023
:10E2B0007000535049436C6173733A3A5350494369
:10E2C0006C617373284E52465F5350495F547970A6
:10E2D000652A2C2075696E74385F742C2075696E00
:10E2E00074385F742C2075696E74385F742900006F
:10E2F0000000000000000000858700003D8700004E
:10E3000073870000798700007F8700007187000015
:10E310000200000003000000040000001F000000D5
:10E320001C0000000E000000250000000B00000093
:10E330000A000000090000001E0000001700000095
:10E340000C00000011000000010000000D000000A2
:10E3500022000000FFFFFFFFFFFFFFFF1A00000089
:10E360002000000015000000160000000F00000053
:10E37000180000001300000024000000000000004E
:10E38000140000000500000010000000080000005C
:10E390001900000028000000060000000000000036
:10E3A00000000000678D000081940000DD8D0000FA
:10E3B000E98D0000E38D0000658D00005D8D00009B
:10E3C000F18D0000818D0000598D000000C00140DA
:10E3D000001002400020024000D002400000000077
:10E3E000000000000000304300000000000030C3C7
:10E3F0007371727400000000FB21F93FFB2109409A
:10E400007CD91240FB2119407A6A1F407CD92240F6
:10E41000BBFD2540FB2129403A462C407A6A2F401B
:10E420005C4731407CD932409C6B3440BBFD354069
:10E43000DB8F3740FB2139401BB43A403A463C4021
:10E440005AD83D407A6A3F404C7E40405C4741404C
:10E450006C1042407CD942408CA243409C6B4440AB
:10E46000AC344540BBFD4540CBC64640DB8F474002
:10E47000EB584840FB21494083F9A200444E6E000E
:10E48000FC291500D1572700DD34F50062DBC00000
:10E490003C999500419043006351FE00BBDEAB0008
:10E4A000B761C5003A6E2400D24D42004906E00033
:10E4B00009EA2E001C92D100EB1DFE0029B11C00C0
:10E4C000E83EA700F535820044BB2E009CE984009D
:10E4D000B4267000417E5F00D69139005383390025
:10E4E0009CF439008B5F840028F9BD00F81F3B00C5
:10E4F000DEFF97000F980500112FEF000A5A8B00DE
:10E500006D1F6D00CF7E360009CB2700464FB70048
:10E510009E663F002DEA5F00BA277500E5EBC70055
:10E520003D7BF100F739070092528A00FB6BEA004D
:10E530001FB15F00085D8D00300356007BFC460074
:10E54000F0AB6B0020BCCF0036F49A00E3A91D00AD
:10E550005E619100081BE60085996500A0145F00CC
:10E560008D40680080D8FF0027734D0006063100FB
:10E57000CA561500C9A873007BE260006B8CC0000E
:10E5800000000040FB21F93F000000002D44743ED4
:10E59000000000809846F83C0000006051CC783BB9
:10E5A00000000080831BF0390000004020257A38ED
:10E5B000000000802282E336000000001DF3693570
:10E5C000020000000300000004000000060000003C
:10E5D0002C2066756E6374696F6E3A2000617373E8
:10E5E000657274696F6E2022257322206661696CE2
:10E5F00065643A2066696C6520222573222C206CA4
:10E60000696E65202564257325730A006400002067
:10E61000232D302B2000686C4C006566674546470B
:10E62000003031323334353637383941424344458E
:10E6300046003031323334353637383961626364FD
:10E6400065660000000000000000000000000000FF
:10E6500000000000000000000000000000000000BA
:10E6600000000000000000000000000000000000AA
:10E67000000000000000000000000000000000009A
:10E68000000000000000000000000000000000008A
:10E69000000000000000000000000000000000007A
:10E6A00000000000504F5349580000202020202037
:10E6B0002020202028282828282020202020202032
:10E6C0002020202020202020202020881010101022
:10E6D0001010101010101010101010040404040476
:10E6E00004040404041010101010101041414141A2
:10E6F000414101010101010101010101010101018A
:10E70000010101010101101010101010424242429B
:10E710004242020202020202020202020202020259
:10E72000020202020202101010102000000000007D
:10E7300000000000000000000000000000000000D9
:10E7400000000000000000000000000000000000C9
:10E7500000000000000000000000000000000000B9
:10E7600000000000000000000000000000000000A9
:10E770000000000000000000000000000000000099
:10E780000000000000000000000000000000000089
:10E790000000000000000000000000000000000079
:10E7A0000000000000000000000000000000000069
:08E7B000901AFF7F0100000038
:10E7B800FFFFFFFFE803000001000000E803DC059D
:10E7C800DC05DC05DC050000FFFFFFFFFFFFFFFFA6
:10E7D8001800000019FCFFFFFFFFFFFF0200000008
:10E7E80040420F00FFFF01FF030000000090D0032C
:10E7F800FFFFFFFFFFFFFFFFFFFFFFFFFFFFFFFF21
:10E808000A000000010000000800000001000000EC
:10E81800640000200000000064E6000084E60000B8
:10E8280044E60000000000000000000000000000B6
:10E8380000000000000000000000000000000000D0
:10E8480000000000000000000000000000000000C0
:10E8580000000000000000000000000000000000B0
:10E8680000000000000000000000000000000000A0
:10E87800000000004300000000000000000000004D
:10E888000000000000000000000000000000000080
:10E89800000000004300000000000000000000002D
:10E8A8000000000000000000000000000000000060
:10E8B800000000004300000000000000000000000D
:10E8C8000000000000000000000000000000000040
:10E8D80000000000430000000000000000000000ED
:10E8E8000000000000000000000000000000000020
:10E8F80000000000430000000000000000000000CD
:10E9080000000000000000000000000000000000FF
:10E9180000000000430000000000000000000000AC
:10E9280000000000000000000000000000000000DF
:10E93800000000004300000000000000000000008C
:10E9480000000000000000000000000000000000BF
:10E95800000000001BCA0000E9C30000000000001E
:10E96800AAE600006ACC0000ABD10000ABD10000E1
:10E97800ABD10000ABD10000ABD10000ABD100009F
:10E98800ABD10000ABD10000ABD10000FFFFFFFF0F
:10E99800FFFFFFFFFFFFFFFFFFFF000001004153E4
:10E9A800434949000000000000000000000000008A
:10E9B80000000000000000000000000000004153BB
:10E9C800434949000000000000000000000000006A
:10E9D800000000000000000000000000000000002F
:10E9E8002502000009870000658B0000F18F0000F8
:04E9F8000102000018
:0400000300008C214C
:00000001FF
